:100000001CC200004BC2000049C2000047C20000F1
:1000100045C2000043C2000041C200003FC20000D0
:100020003DC200000C946F420C946F420C946F42DE
:1000300035C200000C94794231C200002FC200008A
:100040002DC200002BC2000029C2000027C2000000
:1000500025C2000023C2000021C200000C949D4074
:100060001DC200000C944E3F0C94253F17C20000A7
:1000700015C2000013C2000011C200000FC2000030
:100080000DC200000BC2000009C2000007C2000040
:1000900005C2000003C2000001C200000C948A43A4
:1000A000FDC10000FBC10000F9C10000F7C1000064
:1000B000F5C10000F3C10000F1C10000EFC1000074
:1000C000EDC10000EBC10000E9C100000C94FC3E52
:1000D0000C94D33EE3C100000C94AA3E0C94813EE4
:1000E000DDC10000A51E5E1F7520CE23342B5C22CF
:1000F00071227522342B7A22CE23E723FC23942508
:10010000AC263627F3278928BE29FA2A6F3B723B93
:10011000613B653B6B3BA93B763B7A3B803B843B39
:10012000883B8E3B923B963BA93B9C3BA03BA43B30
:10013000084AD73B3BCE016E84BCBFFDC12F3D6C4E
:1001400074319ABD56833DDA3D00C77F11BED9E4B4
:10015000BB4C3E916BAAAABE000000803F076342E1
:1001600036B79BD8A71A39685618AEBAAB558C1D4E
:100170003CB7CC5763BD6DEDFD753EF6177231BFD0
:10018000000000803F08000000BE922449123EABF0
:10019000AAAA2ABECDCCCC4C3E00000080BEABAAA1
:1001A000AAAA3E00000000BF000000803F0000003F
:1001B0000000084178D3BB4387D1133D190E3CC3DF
:1001C000BD4282AD2B3E68EC8276BED98FE1A93E5E
:1001D0004C80EFFFBE01C4FF7F3F00000000000025
:1001E0004E414E494E495459494E46CDCCCC3D0A1C
:1001F000D7233C17B7D13877CC2B329595E6241FFF
:10020000B14F0A000020410000C84200401C4620B7
:10021000BCBE4CCA1B0E5AAEC59D7400407A10F38A
:100220005A00A0724E18090010A5D4E80000E87624
:1002300048170000E40B54020000CA9A3B0000007B
:10024000E1F505000080969800000040420F000094
:1002500000A08601000000102700000000E8030055
:100260000000006400000000000A0000000000011F
:1002700000000000002C76D888DC674F0823DFC11F
:10028000DFAE59E1B1B796E5E3E453C63AE65199DA
:100290007696E8E6C28426EB898C9B62ED407C6F03
:1002A000FCEFBC9C9F40F2BAA56FA5F490055A2ABA
:1002B000F75C936B6CF9676DC11BFCE0E40D47FEC6
:1002C000F520E6B500D0ED902E03009435770500BB
:1002D00080841E080000204E0A000000C80C333342
:1002E00033330F986E12831141EF8D2114893BE651
:1002F0005516CFFEE6DB18D1844B381BF77C1D90DA
:100300001DA4BBE424203284725E228100C9F12442
:10031000ECA1E53D2700002100240027002A002D44
:10032000003000330001010000040107010A010050
:10033000002200250028002B002E0031003400028E
:10034000010000050108010B010000200023002628
:100350000029002C002F00320000010000030106DC
:10036000010901050505050705080808080202023C
:10037000020A0A0808040404040101010101010140
:10038000010303030303030303040707070C0C0C17
:100390000C0C0C0C0C0202020206060606060606EF
:1003A000060B0B0B0B0B0B0B0B010210202008088C
:1003B00010204010204080020102010804020101C7
:1003C00002040810204080804020100804020180B0
:1003D0000402018040201008040201080402010107
:1003E0000204081020408001020408102040800010
:1003F000000A0B02090C0D0E08070304010000009F
:1004000000000000000000000000000000000000EC
:1004100000000000000000000000001211100000A9
:1004200000000000000000000000000000000000CC
:10043000000000000000B65A9A5A11241FBECFEFE8
:10044000D1E2DEBFCDBF00E00CBF1FE0A0E0B2E014
:10045000E8EAF2ED00E00BBF02C007900D92AC3B62
:10046000B107D9F725E1ACEBBFE001C01D92A93679
:10047000B207E1F712E0CCE1D2E000E006C021973C
:100480000109802FFE010E949466CB31D10780E0E4
:100490000807A9F70E9408510C944369B1CD3F9217
:1004A0004F925F926F927F928F929F92AF92BF9284
:1004B000CF92DF92EF92FF920F931F93CF93DF9330
:1004C000CDB7DEB7EF970FB6F894DEBF0FBECDBF46
:1004D00086ED9FE00E949317892B09F46EC28EED82
:1004E00094E10E94B7410E94E44A60E080E00E94EB
:1004F000B7380E94914028EE33E040E050E00E947F
:100500002263BA01A9012AE0CE0101960E940F3DA3
:10051000BE016F5F7F4FCE0182960E94923D6AE4DA
:1005200074E0CE0182960E943C3CBC018EED94E1C9
:100530000E94B53DCE0182960E94DB3CCE01019621
:100540000E94DB3C4091DA0F5091DB0F6091DC0F91
:100550007091DD0F20E186E892E10E94D83D86E8A7
:1005600092E10E946D3E8091DA0F9091DB0FA09195
:10057000DC0FB091DD0F883025E09207A105B105B1
:1005800009F4F8C108F08DC08934E1E09E07A105A7
:10059000B10509F4F2C1E0F5843421E09207A10528
:1005A000B10509F4DBC1E8F48134E1E09E07A1055F
:1005B000B10509F4C4C138F480349140A105B105F6
:1005C00009F4AEC1DDC1823441E09407A105B10553
:1005D00009F4BEC183349140A105B10509F4BBC142
:1005E000CFC18634F1E09F07A105B10509F4BCC174
:1005F00008F4B7C1873441E09407A105B10509F4B7
:10060000B6C188349140A105B10509F4B3C1B8C1A0
:100610008230F5E09F07A105B10509F499C1E8F41E
:10062000843741E09407A105B10509F444C138F4C9
:1006300082379140A105B10509F448C1A1C18115D6
:1006400025E09207A105B10509F46AC18130954002
:10065000A105B10509F473C193C18530E5E09E079A
:10066000A105B10509F47DC170F4833025E092073E
:10067000A105B10509F46FC184309540A105B1050C
:1006800009F46CC17DC18630E5E09E07A105B10586
:1006900009F46AC187309540A105B10509F467C125
:1006A0006FC18D3B22E492072FEFA207B10509F439
:1006B00028C108F04BC08F3EE0E19E07EFEFAE0788
:1006C000B10509F454C118F5823325E09207A1055C
:1006D000B10509F4FBC038F489309540A105B10596
:1006E00009F44BC14DC18433F5E09F07A105B10565
:1006F00009F4E1C08D3F9240AF4FB10509F040C110
:1007000068E174E08FE194E10E94783CDCC08D3DAB
:1007100042E294074FEFA407B10509F4CCC038F4C6
:10072000873E9841AF4FB10509F41BC129C18F3CE9
:1007300020E392072FEFA207B10509F40FC1873C10
:100740009843AF4FB10509F415C11AC18739E8E6DE
:100750009E07EFEFAE07B10509F4F1C048F58D3AF9
:1007600022E592072FEFA207B10509F4BBC038F4C8
:10077000853B9A44AF4FB10509F4D2C001C1853A17
:10078000FAE59F07FFEFAF07B10509F4F6C08D3911
:100790009246AF4FB10509F0F3C065E174E08FE117
:1007A00094E10E94783C10924A158CEF9FEF80C034
:1007B000873548EA94074FEFA407B105F9F078F4BC
:1007C0008538FAE79F07FFEFAF07B10509F4CCC002
:1007D00087369849AF4FB10509F4BAC0D1C08F34FC
:1007E00040EB94074FEFA407B10509F4B4C08D3373
:1007F000924CAF4FB10509F469C0C2C082E080934A
:100800002F131092321300E010E08CEB9FE00E9457
:100810009317892B69F40F5F1F4F093EF3E01F0701
:1008200039F06EE170E080E090E00E945940EDCF39
:1008300069ED77E086E892E10E94803E4091C00F2A
:100840005091C10F6091C20F7091C30F2AE086E8EA
:1008500092E10E94D83D86E892E10E946D3E80912F
:10086000C00F9091C10FA091C20FB091C30F823001
:10087000E5E09E07A105B10509F4B1C108F0B2C1D8
:10088000833421E09207A105B10509F4B9C108F04C
:10089000BAC18134E1E09E07A105B10509F099C113
:1008A00062E174E089E194E10E94783C89EF9FEF76
:1008B0000E944B1E7CC068E174E08FE194E10E94CD
:1008C000783C10924A158BEF9FEFF2CF6BE174E00A
:1008D0008FE194E10E94783C81E080934A158DEF8E
:1008E0009FEFE6CF6EE174E089E194E10E94783CED
:1008F0006EE174E08FE194E10E94783C8EEF9FEF0F
:10090000D7CF61E274E089E194E10E94783C61E232
:1009100074E08FE194E10E94783C8FEF9FEFC8CFA5
:1009200061E378E089E194E10E94783C61E378E05A
:100930008FE194E10E94783C80E090E0B9CF62E2E0
:1009400074E089E194E10E94783C81E090E0B0CFCE
:1009500082E090E0ADCF83E090E0AACF84E090E029
:10096000A7CF85E090E0A4CF86E090E0A1CF87E01C
:1009700090E09ECF88E090E09BCF89E090E098CF18
:1009800060E070E0CE0101960E94CC35BE016F5F41
:100990007F4F89E194E10E94A23CCE0101960E9422
:1009A000DB3C64E670E080E090E00E94594082E029
:1009B00080932F1310923213CFC06CE57FE08FE14C
:1009C00094E10E94783C1092CD0F6CE57FE08FE1BE
:1009D00094E10E94783C11E086E892E10E94773A27
:1009E0002091CD0F181619060CF038C1211136C10F
:1009F000B1C14091000250910102609102027091D8
:100A0000030222E0CE0182960E94E03C6CE175E098
:100A1000CE0101960E949A3DBE016E5D7F4FCE01D0
:100A200001960E94533C6AE474E00E943C3CBC0185
:100A3000CE0188960E94923DCE0188960E94022F98
:100A4000CE0188960E94DB3CCE0101960E94DB3CE1
:100A5000CE0182960E94DB3C40910C0250910D0227
:100A600060910E0270910F0222E0CE0182960E94E8
:100A7000E03C6CE275E0CE0101960E949A3DBE0119
:100A80006E5D7F4FCE0101960E94533C6AE474E094
:100A90000E943C3CBC01CE0188960E94923DCE0152
:100AA00088960E94022FCE0188960E94DB3CCE01E0
:100AB00001960E94DB3CCE0182960E94DB3C8EEDCB
:100AC00094E10E94B7410E94E44A60E080E00E9405
:100AD000B7380E94914028EE33E040E050E00E9499
:100AE0002263BA01A9012AE0CE0101960E940F3DBE
:100AF000BE016F5F7F4FCE0182960E94923D6AE4F5
:100B000074E0CE0182960E943C3CBC018EED94E1E3
:100B10000E94B53DCE0182960E94DB3CCE0101963B
:100B20000E94DB3C80912314909124148330910522
:100B300008F04DC58130910509F0DCC4E0911F1427
:100B4000F0912014309711F40C946E17F0808F2DD3
:100B50000E9493320E9491400E9491406093D20F74
:100B60007093D30F8093D40F9093D50F24C08091AE
:100B70004A1581110C9418170E9491400091D20FD0
:100B80001091D30F2091D40F3091D50FDC01CB0100
:100B9000801B910BA20BB30B88349E4EA105B105AF
:100BA00050F06091E3146B7F6093E31468608EED06
:100BB00094E10E94AF4180914A15882311F40C946E
:100BC0007B1764E670E080E090E00E9459400C944E
:100BD0007B1782349140A105B10509F0E8CE88EF7A
:100BE0009FEF66CE8F3CE0E39E07EFEFAE07B105C7
:100BF00081F0F8F4833025E09207A105B10599F45E
:100C000087EF9FEF55CE843421E09207A105B1050F
:100C100019F486EF9FEF4CCE81309540A105B105C8
:100C200009F43ECEC4CE84309540A105B10589F3C8
:100C3000BECE8736E8E99E07EFEFAE07B10579F241
:100C40008F34F0EB9F07FFEFAF07B105C9F287398B
:100C50009846AF4FB10509F0AACE22CE222361F00B
:100C60002091CD0F80912314909124142111A6C0BE
:100C7000009709F0A3C0E2C000E010E0EE24E39486
:100C80008CE491E10E94773A18161906D4F58CE4A9
:100C900091E10E94553A8093CC0F8A30A1F08D30BB
:100CA00091F09091CD0F91110EC089831A8241E08D
:100CB00050E0BE016F5F7F4F8FE194E10E940F3CD7
:100CC0000F5F1F4F17C08091231490912414892B1C
:100CD00089F0E092CD0F8CE491E10E94773A1816EA
:100CE000190644F46CE57FE08FE194E10E94783CC2
:100CF0001092CD0F6FE070E080E090E00E945940CC
:100D0000BFCF62E370E080E090E00E945940012B89
:100D100009F4A6CF6DE274E0CE0101960E949A3DDF
:100D20006FE174E1CE0101960E94533CBC0186E85C
:100D300092E10E94703ECE0101960E94DB3C8CE461
:100D400091E10E94053B64E670E080E090E00E9443
:100D5000594086CF86E892E10E94553A8093CC0FA5
:100D60008A3071F08D3061F089831A8241E050E061
:100D7000BE016F5F7F4F8FE194E10E940F3C17C06F
:100D80001093CD0F64E274E0CE0101960E949A3D6B
:100D90006FE174E1CE0101960E94533CBC0186E8EC
:100DA00092E10E94703ECE0101960E94DB3C6AE017
:100DB00070E080E090E00E9459400ECE019709F06B
:100DC00058C06AE474E0CE0101960E949A3DCE01BB
:100DD00001960E946B4A811112C062E374E0CE0159
:100DE00082960E949A3DCE0182960E946B4A11E043
:100DF000811110E0CE0182960E94DB3C01C010E020
:100E0000CE0101960E94DB3C112389F060E070E086
:100E1000CE0101960E94CC35BE016F5F7F4F89E104
:100E200094E10E94A23CCE0101960E94DB3C64E169
:100E300070E080E090E00E9459401BC064E670E0E2
:100E400080E090E00E9459400E949140CB0168EE02
:100E500073E00E948166CB0164E670E00E948166C7
:100E60008236910534F080914A15882311F40C9450
:100E70005F176AE070E080E090E00E945940809146
:100E8000231490912414009711F40C94F3160197F5
:100E9000E1F564E374E0CE0188960E949A3DCE01AC
:100EA00088960E946B4A81110C94751766E374E072
:100EB000CE0182960E949A3DCE0182960E946B4A94
:100EC000811112C066EA79E0CE0101960E949A3D36
:100ED000CE0101960E946B4A11E0811110E0CE0113
:100EE00001960E94DB3C01C010E0CE0182960E9478
:100EF000DB3CCE0188960E94DB3C112331F06FE190
:100F000074E189E194E10E948D3C809123149091D9
:100F100024140497D8F56BE279E0CE0101960E9483
:100F20009A3DCE0101960E946B4A182FCE01019680
:100F30000E94DB3C112351F161E070E0CE0101968B
:100F40000E94CC35CE0101960E94043C0AEF1FEFAF
:100F50002FEF3FEF58016901A61AB70AC80AD90A4C
:100F6000B601A5012AE0CE0182960E943B3DBE015A
:100F70006E5D7F4F89E194E10E94A23CCE01829692
:100F80000E94DB3CCE0101960E94DB3C68E374E0EA
:100F9000CE0182960E949A3DCE0182960E946B4AB3
:100FA000811113C06CE374E0CE0101960E949A3D5A
:100FB000CE0101960E946B4A11E0811101C010E040
:100FC000CE0101960E94DB3C01C011E0CE01829669
:100FD0000E94DB3C112309F472CD60E474E0CE0181
:100FE00001960E949A3DCE0101960E94022FCE01E9
:100FF00001960E94DB3C6091470370914803809109
:10100000490390914A030E94CA6120E030E048EC15
:1010100052E40E941A64AB01BC0122E0CE01829628
:101020000E94E03C6CE474E0CE0101960E949A3D7F
:10103000BE016E5D7F4FCE0101960E94533C6DE66E
:1010400075E00E943C3CBC01CE0188960E94923D16
:10105000CE0188960E94022FCE0188960E94DB3C2A
:10106000CE0101960E94DB3CCE0182960E94DB3CC1
:1010700040914303509144036091450370914603AE
:1010800022E0CE0182960E94E03C61E674E0CE014F
:1010900001960E949A3DBE016E5D7F4FCE01019682
:1010A0000E94533CBC01CE0188960E94923DCE0125
:1010B00088960E94022FCE0188960E94DB3CCE01CA
:1010C00001960E94DB3CCE0182960E94DB3C40915F
:1010D0003F0350914003609141037091420322E02D
:1010E000CE0182960E94E03C6EE774E0CE0101964C
:1010F0000E949A3DBE016E5D7F4FCE0101960E9417
:10110000533CBC01CE0188960E94923DCE01889648
:101110000E94022FCE0188960E94DB3CCE010196F0
:101120000E94DB3CCE0182960E94DB3C4091A603EC
:101130005091A7036091A8037091A90322E0CE010A
:10114000C4960E94E03C4091B2035091B303609179
:10115000B4037091B50323E0CE018E960E94E03C6B
:101160004091AA035091AB036091AC037091AD0321
:1011700022E0CE0188960E94E03C4091AE0350915F
:10118000AF036091B0037091B10323E0CE0182966A
:101190000E94E03C6EE874E0CE0101960E949A3D08
:1011A000BE016E5D7F4FCE0101960E94533C63EA03
:1011B00074E00E943C3CBE01685D7F4F0E94533C3E
:1011C00066EA74E00E943C3CBE01625D7F4F0E9473
:1011D000533C63EA74E00E943C3CBE016C5C7F4F70
:1011E0000E94533C6CEA74E00E943C3CBC01CE017E
:1011F000CA960E94923DCE01CA960E94022FCE014D
:10120000CA960E94DB3CCE0101960E94DB3CCE01D7
:1012100082960E94DB3CCE0188960E94DB3CCE0188
:101220008E960E94DB3CCE01C4960E94DB3C61EBB3
:1012300074E0CE0101960E949A3D68ED74E1CE0102
:1012400001960E94533CBC01CE0182960E94923DC1
:10125000CE0182960E94022FCE0182960E94DB3C34
:10126000CE0101960E94DB3C409187035091880398
:101270006091890370918A0323E0CE0188960E94D1
:10128000E03C20917F033091800340918103509195
:10129000820360E070E080E291E40E94C8651BA2D6
:1012A0001AA21DA21CA21FA21EA28E010F5F1F4F19
:1012B00021E043E00E94FC5CBC01CE0182960E94CA
:1012C000783C62EC74E0C8010E949A3DBE016E5DFC
:1012D0007F4FC8010E94533C65ED74E00E943C3C86
:1012E000BE01685D7F4F0E94533C6BED74E00E942D
:1012F0003C3CBC01CE018E960E94923DCE018E9662
:101300000E94022FCE018E960E94DB3CC8010E94F3
:10131000DB3CCE0182960E94DB3CCE0188960E9487
:10132000DB3C40918303509184036091850370916D
:10133000860323E0CE0188960E94E03C20917B0347
:1013400030917C0340917D0350917E0360E070E01A
:1013500080E291E40E94C8651BA21AA21DA21CA2F1
:101360001FA21EA221E043E00E94FC5CBC01CE0152
:1013700082960E94783C6EED74E0C8010E949A3D0E
:10138000BE016E5D7F4FC8010E94533C65ED74E065
:101390000E943C3CBE01685D7F4F0E94533C6BED58
:1013A00074E00E943C3CBC01CE018E960E94923DAE
:1013B000CE018E960E94022FCE018E960E94DB3CBB
:1013C000C8010E94DB3CCE0182960E94DB3CCE012C
:1013D00088960E94DB3C40913B0350913C03609116
:1013E0003D0370913E0322E0CE0182960E94E03CD4
:1013F00061EF74E0C8010E949A3DBE016E5D7F4FAF
:10140000C8010E94533C67E075E00E943C3CBC016F
:10141000CE0188960E94923DCE0188960E94022FAE
:10142000CE0188960E94DB3CC8010E94DB3CCE01C5
:1014300082960E94DB3CBBE2CB2EB3E0DB2E01E0C8
:1014400010E08FE0E82E8091290390912A03801705
:1014500091070CF4CECAD601AD90BD906D014AE063
:10146000B501CE0188960E94673D4AE0B801CE01E1
:1014700082960E94673D6EE075E0CE0101960E9463
:101480009A3DBE016E5D7F4FCE0101960E94533C96
:1014900067EA7FE00E943C3CBE01685D7F4F0E948E
:1014A000533C66E175E00E943C3CEA9CB001EB9C39
:1014B000700D1124605F7D4F0E943C3CBC01CE0149
:1014C0008E960E94923DCE018E960E94022FCE01F2
:1014D0008E960E94DB3CCE0101960E94DB3CCE0141
:1014E00082960E94DB3CCE0188960E94DB3C0F5F17
:1014F0001F4FA9CF029709F02ACB6BE279E0CE010A
:1015000001960E949A3DCE0101960E946B4A182FC7
:10151000CE0101960E94DB3C112309F418CB809187
:10152000231490912414029740F0E0911F14F0913D
:101530002014309711F0818101C080E01A82198255
:101540001C821B821E821D828AA31BA2BE016E5DAD
:101550007F4FCE0101960E94783CBE016F5F7F4FA6
:1015600089E194E10E94A23CCE0101960E94DB3CFD
:101570008091231490912414892B41F0E0911F1441
:10158000F0912014309711F0F08001C0F12C67E247
:1015900075E0CE0101960E949A3D6FE174E1CE01A3
:1015A00001960E94533C60E87FE00E943C3CBC01F5
:1015B00086E892E10E94B53DCE0101960E94DB3C97
:1015C00069E174E186E892E10E94703EC0CA41E0A0
:1015D00050E060E070E0CE0101960E948C35BE01C3
:1015E0006F5F7F4F87E094E10E94A23CCE0101969D
:1015F0000E94DB3C69E675E0CE0182960E949A3D2E
:10160000CE0182960E946B4A811113C062EA79E092
:10161000CE0101960E949A3DCE0101960E946B4A2E
:1016200011E0811101C010E0CE0101960E94DB3C67
:1016300001C011E0CE0182960E94DB3C112309F427
:10164000CEC062E070E0CE0101960E94CC35BE01B2
:101650006F5F7F4F87E094E10E94A23CCE0101962C
:101660000E94DB3C67E074E186E892E10E94703EF4
:101670000E94FC5020E030E048EC52E40E942962D5
:101680000E94B364AB01BC014093470350934803ED
:101690006093490370934A032AE030E086E892E1C0
:1016A0000E94203E86E892E10E946D3E60914703D1
:1016B000709148038091490390914A038B019C01EA
:1016C00000591F452140310901341C4921053105CC
:1016D000D0F06CE375E0CE0101960E949A3D67E080
:1016E00074E1CE0101960E94533C6FE475E00E94C4
:1016F0003C3CBC018DE094E10E948D3CCE01019602
:101700000E94DB3C4DC019821A821B821C821D8202
:101710001E821F8218860E94CA6120E030E048ECD9
:1017200052E40E941A648E010F5F1F4F22E047E0CF
:101730000E94FC5CBC018DE094E10E94783C6FE566
:1017400075E0CE0182960E949A3D6DE074E1CE0173
:1017500082960E94533C6CE675E00E943C3CBC01C2
:101760008DE094E10E948D3CCE0182960E94DB3C8C
:1017700010923910109238108091470390914803CD
:10178000A0914903B0914A038093B2109093B31093
:10179000A093B410B093B51080E090E00E943E3664
:1017A00064E175E0CE0101960E949A3D6DE074E11E
:1017B000CE0101960E94533CBC01CE0182960E944C
:1017C000923DCE0182960E94022FCE0182960E9407
:1017D000DB3CCE0101960E94DB3C10E001C011E031
:1017E00061E775E0CE0182960E949A3DCE01829615
:1017F0000E946B4A811113C067E775E0CE01019624
:101800000E949A3DCE0101960E946B4A01E081112F
:1018100001C000E0CE0101960E94DB3C01C001E066
:10182000CE0182960E94DB3C002309F4FDC046E015
:1018300050E065E070E0CE0101960E948C35BE015B
:101840006F5F7F4F87E094E10E94A23CCE0101963A
:101850000E94DB3C87E094E10E94043C2B013C01A8
:1018600065E075E0CE0101960E949A3D80912314B7
:10187000909124142D813E817C01E21AF30A2115F6
:10188000310559F1009749F18217930730F1E816B5
:10189000F90620F07C01E1E0EE1AF108C0901F1477
:1018A000D090201489809A80C60133243A940FEF97
:1018B0005601AE0CBF1CA816B90690F0B4010E94E8
:1018C0002969009769F09C012C193D09E216F3067D
:1018D00010F0322E032F0196EECF6FEF7FEF02C094
:1018E000632D702F6F5F7F4FCE0182960E94CC35A3
:1018F000BE016E5D7F4F87E094E10E94A23CCE0165
:1019000082960E94DB3CCE0101960E94DB3C87E080
:1019100094E10E94043CF201EE0FFF1FE75DFC4FD3
:1019200071836083FCE14F0E511C9201220F331F23
:10193000F901EE54FF4E718360836090290370902B
:101940002A03C0902303D090240340912503509193
:101950002603809027039090280360918B03709159
:101960008C034090210350902203E0901F03F090DD
:101970002003ECEBF3E0ABE2AA2EA3E0BA2E21E0C9
:1019800030E06216730654F1D5018D919D915D0191
:101990008430910519F48280938018C08A309105B3
:1019A00019F44281538112C08530910519F4C28027
:1019B000D38010C08630910519F4628173810AC00A
:1019C0008730910519F44280538004C00B9714F0BE
:1019D000E280F3802F5F3F4F3296D3CFD092240323
:1019E000C0922303F0922003E0921F03509222033F
:1019F0004092210370938C0360938B0350932603D2
:101A00004093250390922803809227036FE174E1AD
:101A100086E892E10E94703E1092391010923810C0
:101A200080E090E00E943E366DE775E0CE01829640
:101A30000E949A3DCE0182960E946B4A811113C08A
:101A400061E875E0CE0101960E949A3DCE010196B3
:101A50000E946B4A01E0811101C000E0CE010196B5
:101A60000E94DB3C01C001E0CE0182960E94DB3C7B
:101A7000002309F472C063E070E0CE0101960E9479
:101A8000CC35BE016F5F7F4F87E094E10E94A23C9E
:101A9000CE0101960E94DB3C67E074E186E892E1AA
:101AA0000E94703E109239101092381067E074E175
:101AB00088ED94E10E948D3C8EEC90E1892BE1F061
:101AC0000091DC141091DD140115110519F4109228
:101AD000CE1012C00730110510F007E010E0609141
:101AE000D8147091D914A8018EEC90E10E941A6963
:101AF000F801E253FF4E1082809138109091391016
:101B00000E943E3665E875E0CE0182960E949A3DBD
:101B100068ED74E1CE0182960E94533CBC01CE0177
:101B200001960E94923DCE0182960E94DB3CBE014E
:101B30006F5F7F4F8CE491E10E94B53D68EB7BE0E5
:101B400080E090E00E9459408EEC90E10E94E434E5
:101B5000CE0101960E94DB3C10E06DE875E0CE01FD
:101B600082960E949A3DCE0182960E946B4A811114
:101B700013C061E975E0CE0101960E949A3DCE0145
:101B800001960E946B4A01E0811101C000E0CE0184
:101B900001960E94DB3C01C001E0CE0182960E94CA
:101BA000DB3C002309F4D5C063E070E0CE01019670
:101BB0000E94CC35BE016F5F7F4F87E094E10E94A9
:101BC000A23CCE0101960E94DB3C0E94FC506B01BE
:101BD0007C0110923910109238100E94E7369093D1
:101BE000351080933410892BC9F165E975E0CE0179
:101BF00001960E949A3DCE0101960E948432CE0148
:101C000001960E94DB3C67E074E1CE0101960E94E0
:101C1000923DCE0101960E94022FCE0101960E94B4
:101C2000DB3C66EB75E0CE0101960E949A3DCE0149
:101C300001960E94022FCE0101960E94DB3C60912A
:101C40003F037091400380914103909142030E94B1
:101C5000E73690933510809334107AC060E070E0DE
:101C600082E090E00E94D63680E090E090933510BC
:101C700080933410892B59F163E176E0CE0101960F
:101C80000E949A3DCE0101960E948432CE010196B7
:101C90000E94DB3C67E074E1CE0101960E94923D18
:101CA000CE0101960E94022FCE0101960E94DB3CDC
:101CB00066EB75E0CE0101960E949A3DCE01019639
:101CC0000E94022FCE0101960E94DB3C41C0C092CF
:101CD0003F03D0924003E0924103F092420364E458
:101CE00076E0CE0101960E949A3DCE0101960E94B7
:101CF0008432CE0101960E94DB3C40913F0350911B
:101D00004003609141037091420322E0CE010196AD
:101D10000E94E03CCE0101960E94022FCE01019666
:101D20000E94DB3C80913F0390914003A0914103CE
:101D3000B09142038093BA109093BB10A093BC1053
:101D4000B093BD1080913810909139100E943E36AA
:101D500010E068E576E0CE0182960E949A3DCE01C1
:101D600082960E946B4A811113C06DE576E0CE0128
:101D700001960E949A3DCE0101960E946B4A01E0B5
:101D8000811101C000E0CE0101960E94DB3C01C040
:101D900001E0CE0182960E94DB3C002309F43FC0A3
:101DA00064E070E0CE0101960E94CC35BE016F5F09
:101DB0007F4F87E094E10E94A23CCE0101960E94F1
:101DC000DB3C62E676E0CE0182960E949A3D67E0B7
:101DD00074E1CE0182960E94533CBC01CE01019673
:101DE0000E94923DCE0182960E94DB3CBE016F5F55
:101DF0007F4F8CE491E10E94B53D68EB7BE080E091
:101E000090E00E945940BE016F5F7F4F86E892E1EB
:101E10000E94703ECE0101960E94DB3C10E069E614
:101E200076E0CE0188960E949A3DCE0188960E9467
:101E30006B4A81112BC06CE676E0CE0182960E943F
:101E40009A3DCE0182960E946B4A811113C06FE6C3
:101E500076E0CE0101960E949A3DCE0101960E9445
:101E60006B4A01E0811101C000E0CE0101960E94A1
:101E7000DB3C01C001E0CE0182960E94DB3CCE013A
:101E800088960E94DB3C011105C020C1CE018896D6
:101E90000E94DB3C8AE0A82EB12CC12CD12C76010B
:101EA00088248A9493E0992E6EE170E080E090E0BF
:101EB0000E945940809123030E940F40B4010E9468
:101EC0008166072E000C880B990B0E94CA6120E0E6
:101ED00030E040EA50E40E9429629B01AC01C70156
:101EE000B6010E9454636B017C01B1E0AB1AB108EA
:101EF000D9F620E030E040E251E40E941A646B0120
:101F00007C0162E776E0CE0182960E949A3DCE0186
:101F100082960E946B4A8111E4C766E776E0CE01A3
:101F200001960E949A3DCE0101960E946B4A01E003
:101F3000811101C000E0CE0101960E94DB3CCE0180
:101F400082960E94DB3C002309F43FC020E030E091
:101F500040E650E4C701B6010E9429629B01AC0132
:101F600060E070E080E890E40E945363AB01BC0144
:101F70004093040250930502609306027093070297
:101F800022E0CE0101960E94E03CBE016F5F7F4FD0
:101F90008DE094E10E94A23CCE0101960E94DB3CC0
:101FA0006AE776E0CE0101960E949A3D6DE074E109
:101FB000CE0101960E94533CBC018DE094E10E9449
:101FC0008D3CCE0101960E94DB3C69E876E0CE01B3
:101FD00082960E949A3DCE0182960E946B4A8111A0
:101FE00082C76EE876E0CE0101960E949A3DCE014E
:101FF00001960E946B4A01E0811101C000E0CE0110
:1020000001960E94DB3CCE0182960E94DB3C0023BD
:1020100009F43FC020E030E040E650E4C701B601DB
:102020000E9429629B01AC0160E070E080E291E4D3
:102030000E945363AB01BC01409308025093090214
:1020400060930A0270930B0222E0CE0101960E9477
:10205000E03CBE016F5F7F4F8DE094E10E94A23CA7
:10206000CE0101960E94DB3C63E976E0CE01019649
:102070000E949A3D6DE074E1CE0101960E94533CAE
:10208000BC018DE094E10E948D3CCE0101960E943E
:10209000DB3C64E175E0CE0101960E949A3D6DE063
:1020A00074E1CE0101960E94533CBC01CE018296A0
:1020B0000E94923DCE0182960E94022FCE0182960E
:1020C0000E94DB3CCE0101960E94DB3C63EA76E095
:1020D000CE0101960E949A3DCE0101960E946B4A64
:1020E000082FCE0101960E94DB3C002309F469C051
:1020F0008091231490912414079708F462C066E03D
:1021000070E0CE0101960E94CC35BE016F5F7F4F1B
:1021100087E094E10E94A23CCE0101960E94DB3C44
:102120000E94FC50AB01BC0140930002509301029D
:10213000609302027093030221E0CE0182960E9416
:10214000E03C6CE175E0CE0101960E949A3DBE0133
:102150006E5D7F4FCE0101960E94533C6AE474E0AD
:102160000E943C3CBC018DE094E10E948D3CCE017C
:1021700001960E94DB3CCE0182960E94DB3C6DE022
:1021800074E1CE0101960E94923DCE0101960E941B
:10219000022FCE0101960E94DB3C0E94914028EE66
:1021A00033E040E050E00E942263CA01B9010E947E
:1021B000C8616093CE0F7093CF0F8093D00F909330
:1021C000D10F6AEA76E0CE0101960E949A3DCE01D7
:1021D00001960E946B4A082FCE0101960E94DB3CBB
:1021E000002309F456C0809123149091241407977A
:1021F00008F44FC066E070E0CE0101960E94CC3535
:10220000BE016F5F7F4F87E094E10E94A23CCE0148
:1022100001960E94DB3C0E94FC50AB01BC01409344
:102220000C0250930D0260930E0270930F0221E096
:10223000CE0182960E94E03C6CE275E0CE010196F0
:102240000E949A3DBE016E5D7F4FCE0101960E94B5
:10225000533C6AE474E00E943C3CBC018DE094E194
:102260000E948D3CCE0101960E94DB3CCE018296FD
:102270000E94DB3C6DE074E1CE0101960E94923D2C
:10228000CE0101960E94022FCE0101960E94DB3CF6
:1022900010E061EB76E0CE0182960E949A3DCE017D
:1022A00082960E946B4A811113C065EB76E0CE01E5
:1022B00001960E949A3DCE0101960E946B4A01E070
:1022C000811101C000E0CE0101960E94DB3C01C0FB
:1022D00001E0CE0182960E94DB3C002309F478C025
:1022E00080912703909128030E94382C6093AE03BD
:1022F0007093AF038093B0039093B1036093C610C3
:102300007093C7108093C8109093C91080E090E03C
:10231000A0E8BFE38093AA039093AB03A093AC0320
:10232000B093AD038093BE109093BF10A093C010E4
:10233000B093C11069EB76E086E892E10E94803E9E
:102340006091AE037091AF038091B0039091B1039F
:102350000E94E947109239101092381080E090E006
:102360000E943E364091AE035091AF036091B0039E
:102370007091B10322E0CE0182960E94E03C64EDB0
:1023800076E0CE0101960E949A3DBE016E5D7F4FC0
:10239000CE0101960E94533CBC018DE094E10E9465
:1023A0008D3CCE0101960E94DB3CCE0182960E94BC
:1023B000DB3C6DE074E1CE0101960E94923DCE01BE
:1023C00001960E94022FCE0101960E94DB3C10E094
:1023D0006DED76E0CE0182960E949A3DCE01829606
:1023E0000E946B4A811113C063EE76E0CE01019624
:1023F0000E949A3DCE0101960E946B4A01E0811134
:1024000001C000E0CE0101960E94DB3C01C001E06A
:10241000CE0182960E94DB3C002309F4D6C0809155
:102420002314909124140797D8F066E070E0CE0151
:1024300001960E94CC35BE016F5F7F4F87E094E12B
:102440000E94A23CCE0101960E94DB3C0E94FC50FF
:1024500060933B0370933C0380933D0390933E0352
:10246000809121030E940F40BC01990F880B990BAA
:102470000E94CA612DE038E643E55BE30E942962D1
:102480006B017C01209163033091640340916503EB
:10249000509166030E94C46118164CF060914B0382
:1024A00070914C0380914D0390914E031BC020917D
:1024B0007703309178034091790350917A03C701F3
:1024C000B6010E94096587FF05C0C701B6010E94D9
:1024D000F53408C060915F037091600380916103DF
:1024E0009091620320E030E048EC52E40E942962BF
:1024F0006B017C0120E030E0A9010E94C461181644
:1025000034F0C12CD12C38EAE32E31E4F32EC09202
:102510003B03D0923C03E0923D03F0923E03C09215
:10252000E610D092E710E092E810F092E91069EE20
:1025300076E086E892E10E94803E60913B037091D4
:102540003C0380913D0390913E030E94E947109225
:1025500039101092381080E090E00E943E36409191
:102560003B0350913C0360913D0370913E0322E098
:10257000CE0182960E94E03C6AEF76E0CE010196A1
:102580000E949A3DBE016E5D7F4FCE0101960E9472
:10259000533CBC018DE094E10E948D3CCE0101963C
:1025A0000E94DB3CCE0182960E94DB3C6DE074E130
:1025B000CE0101960E94923DCE0101960E94022F0B
:1025C000CE0101960E94DB3C10E064E077E0CE0192
:1025D00082960E949A3DCE0182960E946B4A81119A
:1025E00013C069E077E0CE0101960E949A3DCE01CA
:1025F00001960E946B4A01E0811101C000E0CE010A
:1026000001960E94DB3C01C001E0CE0182960E944F
:10261000DB3C002309F4B8C080912314909124146A
:102620000697E8F065E070E0CE0101960E94CC3597
:10263000BE016F5F7F4F87E094E10E94A23CCE0114
:1026400001960E94DB3C0E94FC500E944A65609308
:102650007F03709380038093810390938203809122
:102660008B0390918C030E94F62B20E030E048E031
:1026700051E40E941A6460938703709388038093E7
:10268000890390938A036093D6107093D710809338
:10269000D8109093D91080917F0390918003A091DE
:1026A0008103B09182038093DE109093DF10A0939A
:1026B000E010B093E1106EE077E086E892E10E94CE
:1026C000803E20917F03309180034091810350919F
:1026D000820360E070E080E291E40E94C86541E01E
:1026E0000E94BA376EE177E086E892E10E94803E70
:1026F00060918703709188038091890390918A0388
:102700000E94E947109239101092381080E090E052
:102710000E943E364091870350918803609189035F
:1027200070918A0323E0CE0182960E94E03C65E22C
:1027300077E0CE0101960E949A3DBE016E5D7F4F0B
:10274000CE0101960E94533C6EE277E00E943C3C31
:10275000BC018DE094E10E948D3CCE0101960E9467
:10276000DB3CCE0182960E94DB3C6DE074E1CE0141
:1027700001960E94923DCE0101960E94022FCE0149
:1027800001960E94DB3C10E060E377E0CE01829688
:102790000E949A3DCE0182960E946B4A811113C01D
:1027A00065E377E0CE0101960E949A3DCE01019645
:1027B0000E946B4A01E0811101C000E0CE01019648
:1027C0000E94DB3C01C001E0CE0182960E94DB3C0E
:1027D000002309F4B8C08091231490912414069723
:1027E000E8F065E070E0CE0101960E94CC35BE01B4
:1027F0006F5F7F4F87E094E10E94A23CCE0101967B
:102800000E94DB3C0E94FC500E944A6560937B035F
:1028100070937C0380937D0390937E0380918B0360
:1028200090918C030E94F62B20E030E048E051E4C8
:102830000E941A64609383037093840380938503DA
:10284000909386036093DA107093DB108093DC1012
:102850009093DD1080917B0390917C03A0917D0388
:10286000B0917E038093E2109093E310A093E41064
:10287000B093E5106AE377E086E892E10E94803E3B
:1028800020917B0330917C0340917D0350917E0326
:1028900060E070E080E291E40E94C86541E00E943F
:1028A000BA376EE177E086E892E10E94803E60915F
:1028B00083037091840380918503909186030E9425
:1028C000E947109239101092381080E090E00E9491
:1028D0003E3640918303509184036091850370914B
:1028E000860323E0CE0182960E94E03C69E477E013
:1028F000CE0101960E949A3DBE016E5D7F4FCE01D2
:1029000001960E94533C6EE277E00E943C3CBC0181
:102910008DE094E10E948D3CCE0101960E94DB3C4B
:10292000CE0182960E94DB3C6DE074E1CE010196FF
:102930000E94923DCE0101960E94022FCE01019687
:102940000E94DB3C10E062E577E0CE0182960E94B7
:102950009A3DCE0182960E946B4A811113C066E5B2
:1029600077E0CE0101960E949A3DCE0101960E9429
:102970006B4A01E0811101C000E0CE0101960E9486
:10298000DB3C01C001E0CE0182960E94DB3C0023CB
:1029900009F478C080912703909128030E94382C75
:1029A0006093B2037093B3038093B4039093B50321
:1029B0006093CA107093CB108093CC109093CD107D
:1029C00080E090E5A3ECB7E48093A6039093A7037F
:1029D000A093A803B093A9038093C2109093C3104F
:1029E000A093C410B093C5106AE577E086E892E141
:1029F0000E94803E6091B2037091B3038091B40352
:102A00009091B5030E94E947109239101092381046
:102A100080E090E00E943E364091B2035091B303B3
:102A20006091B4037091B50322E0CE0182960E94BA
:102A3000E03C67E777E0CE0101960E949A3DBE0137
:102A40006E5D7F4FCE0101960E94533CBC018DE02C
:102A500094E10E948D3CCE0101960E94DB3CCE01A8
:102A600082960E94DB3C6DE074E1CE0101960E94EB
:102A7000923DCE0101960E94022FCE0101960E9446
:102A8000DB3C10E062E877E0CE0182960E949A3D3E
:102A9000CE0182960E946B4A811113C066E877E0EE
:102AA000CE0101960E949A3DCE0101960E946B4A8A
:102AB00001E0811101C000E0CE0101960E94DB3CE3
:102AC00001C001E0CE0182960E94DB3C002309F4A4
:102AD000A6C080912314909124140497D8F064E048
:102AE00070E0CE0101960E94CC35BE016F5F7F4F32
:102AF00087E094E10E94A23CCE0101960E94DB3C5B
:102B00000E94FC506093AA037093AB038093AC03C4
:102B10009093AD038091AA039091AB03A091AC0375
:102B2000B091AD038093BE109093BF10A093C010DE
:102B3000B093C1106AE877E086E892E10E94803E97
:102B40006091AA037091AB038091AC039091AD03A7
:102B500042E00E94BA3780912703909128030E9497
:102B6000382C6093AE037093AF038093B0039093BF
:102B7000B1036093C6107093C7108093C8109093F0
:102B8000C91062EA77E086E892E10E94803E609197
:102B9000AE037091AF038091B0039091B1030E9496
:102BA000E947109239101092381080E090E00E94AE
:102BB0003E364091AE035091AF036091B0037091E7
:102BC000B10322E0CE0182960E94E03C6CEA77E0FD
:102BD000CE0101960E949A3DBE016E5D7F4FCE01EF
:102BE00001960E94533CBC018DE094E10E948D3C13
:102BF000CE0101960E94DB3CCE0182960E94DB3C16
:102C00006DE074E1CE0101960E94923DCE010196E5
:102C10000E94022FCE0101960E94DB3C10E064EB83
:102C200077E0CE0182960E949A3DCE0182960E9464
:102C30006B4A811113C068EB77E0CE0101960E94C8
:102C40009A3DCE0101960E946B4A01E0811101C0BC
:102C500000E0CE0101960E94DB3C01C001E0CE0104
:102C600082960E94DB3C002309F4A2C080912314C9
:102C7000909124140497D8F064E070E0CE0101969E
:102C80000E94CC35BE016F5F7F4F87E094E10E94C8
:102C9000A23CCE0101960E94DB3C0E94FC50609356
:102CA000A6037093A7038093A8039093A903809130
:102CB000A6039091A703A091A803B091A9038093C4
:102CC000C2109093C310A093C410B093C5106CEBC6
:102CD00077E086E892E10E94803E6091A6037091C1
:102CE000A7038091A8039091A90342E00E94BA37FC
:102CF00080912703909128030E94382C6093B2039F
:102D00007093B3038093B4039093B5036093CA1098
:102D10007093CB108093CC109093CD1062EA77E043
:102D200086E892E10E94803E6091B2037091B30305
:102D30008091B4039091B5030E94E9471092391035
:102D40001092381080E090E00E943E364091B2032D
:102D50005091B3036091B4037091B50322E0CE01AA
:102D600082960E94E03C6CEA77E0CE0101960E94D8
:102D70009A3DBE016E5D7F4FCE0101960E94533C8D
:102D8000BC018DE094E10E948D3CCE0101960E9431
:102D9000DB3CCE0182960E94DB3C6DE074E1CE010B
:102DA00001960E94923DCE0101960E94022F15C00D
:102DB000112311F40C94AC0564E175E0CE01019689
:102DC0000E949A3D6FE174E1CE0101960E94533C4E
:102DD000BC0186E892E10E94703ECE0101960E94FD
:102DE000DB3C0C94AC050E943F4F182F882311F454
:102DF0000C94B7058EED94E10E94B7416CE57FE03D
:102E000089E194E10E94783C64ED77E086E892E104
:102E10000E94803E612F86E892E10E94AE3D86E8E6
:102E200092E10E946D3E812F0E9493320C94AC057A
:102E30000E94914028EEC22E23E0D22EE12CF12CEC
:102E4000A70196010E942263CA01B9010E94C861CC
:102E50002091CE0F3091CF0F4091D00F5091D10FD4
:102E60000E945363209100023091010240910202BE
:102E7000509103020E940965181614F00C94BC05C9
:102E80000E949140A70196010E942263CA01B901E4
:102E90000E94C8616093CE0F7093CF0F8093D00FC4
:102EA0009093D10F8091361090913710F4D664E151
:102EB00070E080E090E00E9459400C94DB0589E1CD
:102EC00094E10E94043C613071058105910511F087
:102ED0000C9439070E945E2C0C943907F12C0C9449
:102EE000A70501E02CC801E08EC8CE0188960E949B
:102EF000DB3C0C948507EF960FB6F894DEBF0FBE4F
:102F0000CDBFDF91CF911F910F91FF90EF90DF9098
:102F1000CF90BF90AF909F908F907F906F905F9079
:102F20004F903F9008952F923F924F925F926F92F1
:102F30007F928F929F92AF92BF92CF92DF92EF9249
:102F4000FF920F931F93CF93DF93CDB7DEB72897F0
:102F50000FB6F894DEBF0FBECDBFFC0185E393E151
:102F6000938782878091321390E095878487809140
:102F7000FF1390E09787868780912F13853009F0A3
:102F8000B7C38091371390913813885891098D35C4
:102F9000910588F480913213843041F48091391383
:102FA00090913A138097479708F407C280913213A3
:102FB000843408F0E8C1809132138A3108F448C0A3
:102FC0008091351390913613843F914050F41186CF
:102FD00010868FEF9FEFDC0184839583A683B783F0
:102FE00051C0809137139091381385974B9780F596
:102FF0001BE3E12E13E1F12E82E090E040E050E08F
:10300000BA018C010F5F1F4F2091321330E002177D
:1030100013076CF4970122503109D9012D913C918D
:10302000275031092730310508F40AC2C801019739
:1030300095958795918780870C971CF4118610864B
:1030400007C0448355836683778384E090E01CC186
:10305000809132138A3108F448C0809135139091E1
:1030600036138032934008F4B2CF80913713909199
:103070003813C697869708F403C237C04483558334
:10308000668377838BE090E0FFC0D7012D913C9160
:10309000255231092B31310508F004C2440F551F68
:1030A000661F771F41600296B4E0EB0EF11C8C01A5
:1030B0000F5F1F4F2091321330E00217130764F4A3
:1030C000970122503109D9012D913C912C503109A1
:1030D0002B303105D0F2C8010197959587959187DE
:1030E00080870C975CF611861086809132138232AD
:1030F00008F44CC0809137139091381306970797C6
:1031000008F044C04BE3C42E43E1D42E82E090E0AB
:1031100040E050E0BA018C010F5F1F4F2091321345
:1031200030E0021713070CF5D6011297ED90FC90D2
:1031300011979D01BEE1EB1AF108A7E1EA16F1042F
:1031400008F0BEC1440F551F661F771F4160D601AE
:103150002D913C91B4E0CB0ED11C23503109253088
:10316000310510F40296D7CFC80101979595879540
:103170009187808740971CF41186108607C044838E
:103180005583668377838CE090E07EC07F011C824C
:103190001B8281E090E09A838983809132138D3085
:1031A00008F475C029E733E0AE014D5F5F4FBE0103
:1031B0006F5F7F4FCF010E948850892B09F067C055
:1031C00029E733E0AE014D5F5F4FBE016F5F7F4F78
:1031D000C7010E948850019709F059C029E733E0E0
:1031E000AE014D5F5F4FBE016F5F7F4FC7010E9411
:1031F0008850892B09F04BC0812C912C540100E0A0
:1032000010E08091321390E029813A812817390724
:103210007CF529E733E0AE014D5F5F4FBE016F5F84
:103220007F4FC7010E9488506C0129E733E0AE014F
:103230004D5F5F4FBE016F5F7F4FC7010E94885097
:10324000E1E0CE16D10449F4892B09F5880C991CCC
:10325000AA1CBB1C689480F808C0CD28C1F4019753
:10326000B1F4880C991CAA1CBB1C0F5F1F4FC9CF5F
:10327000D70119961C930E931897F70184829582B3
:10328000A682B78281E090E09183808329C21C826C
:103290001B8281E090E09A838983D7011C968D91EF
:1032A0009C911D97181619060CF061C01A96ED91A5
:1032B000FC911B9782E090E09A83898382819381BD
:1032C00089974E9708F053C083E090E09A838983F2
:1032D000848195810B970A9708F049C02CEB31E067
:1032E000AE014D5F5F4FBE016F5F7F4FC7010E9410
:1032F0008850892BE1F52CEB31E0AE014D5F5F4F3B
:10330000BE016F5F7F4FC7010E948850019779F51A
:10331000412C512C320100E010E029813A81D70183
:103320001C968D919C911D97281739070CF010C1A0
:103330002CEB31E0AE014D5F5F4FBE016F5F7F4F01
:10334000C7010E9488505C010330110509F0C6C016
:103350002CEB31E0AE014D5F5F4FBE016F5F7F4FE1
:10336000C7010E948850A816B90609F4B7C0D70152
:103370001A96ED91FC911B9782819381C69786974F
:1033800008F4F2C03EC18091391390913A138254EF
:1033900091098E9708F00FCE20E030E0C12CD12C9F
:1033A0007601A901455C5C4EDA014D915C91495072
:1033B00051094930510598F0FECD80913B13909111
:1033C0003C130997099708F0F1CD118610868FEF0D
:1033D0009FEFDC0184839583A683B7838CC1B901F9
:1033E000635C7C4EDB014D915C9147515109423148
:1033F0005105C0F4D701C601880F991FAA1FBB1F32
:103400006C017D016894C0F82C5F3F4F2038310576
:1034100041F620E230E031872087C482D582E682FF
:10342000F78269C1DB014D915C91465051094730EB
:10343000510508F0C0CDCC0CDD1CEE1CFF1CE4CF08
:10344000D7012D913C91235131092F30310550F492
:10345000440F551F661F771F41600296B4E0EB0EC4
:10346000F11CCFCDD7012D913C912A503109293043
:10347000310508F0EDCD440F551F661F771FEDCFC6
:103480008091391390913A13C697869708F02DCE04
:103490008DE3E82E83E1F82E83E090E040E050E0F9
:1034A000BA0105CED7012D913C912C5031092A301B
:1034B000310508F01ACE440F551F661F771FF3CD54
:1034C000D9012D913C912C5031092B30310508F058
:1034D0005DCE440F551F661F771F39CE2CEB31E0B0
:1034E000AE014D5F5F4FBE016F5F7F4FC7010E940E
:1034F00088506C010330110579F42CEB31E0AE01FA
:103500004D5F5F4FBE016F5F7F4FC7010E948850C4
:10351000C816D90609F02BCFA114B10459F4CA94E6
:10352000CD2809F024CF440C551C661C771C6894E8
:1035300040F80BC0AA94AB2809F019CFCD2809F0A8
:1035400016CF440C551C661C771C0F5F1F4FE5CE31
:1035500019961C930E931897F70144825582668240
:10356000778282E090E090CE848195814B97459759
:1035700008F047C0DF0116966F0126ECC20ED11C81
:1035800020E030E040E050E060E070E080E090E07B
:103590000D911C911197095011090830110588F5FA
:1035A00012960D911C911397015111090D301105BF
:1035B000D8F401E00E949C6621601496AC15BD050C
:1035C00039F7F701248335834683578300E20E944D
:1035D000B7662283338385E090E09183808380E324
:1035E00090E0918780877CC012960D911C91139773
:1035F000045011090530110520F401E00E949C6679
:10360000DCCF80913213893340F0828193818957D6
:1036100091098335910508F47CC18091321382327F
:1036200009F46CC082819381895791098335910592
:1036300008F4E6C1828193818C549109C59708F002
:1036400064C080913213843031F4848195818097F5
:10365000479708F434C280913213843408F455C07B
:103660008481958189549109C39708F04EC09F01C8
:103670002A5F3F4FAF014A575F4F812C912C540175
:10368000D9016D917C916950710969307105E8F536
:10369000D90112966D917C91139766517109613130
:1036A000710508F022C2D501C401880F991FAA1F15
:1036B000BB1F4C015D01689480F82C5F3F4F2417BD
:1036C0003507F1F620E230E0F70131872087D70196
:1036D00084829582A682B78287E090E08D939C9346
:1036E00081E090E0BFC282E080932F1310923213EA
:1036F00080E090E0B7C283E090E0C6CD8281938104
:103700000A97099708F460C18DCF809132138634EF
:1037100060F1828193810C970B9708F4F6C125C064
:10372000D90112966D917C9113976E517109673191
:10373000710508F01EC2D501C401880F991FAA1F88
:10374000BB1F4C015D01689480F84E5F5F4F2C5F9A
:103750003F4F4534510509F4F3C1D9016D917C9176
:103760006C5071096B307105D8F280913213883535
:1037700078F182819381855891098B35910508F400
:1037800008C226C0BC016F5F7F4FD8012D913C91CC
:10379000275031092730310508F00AC2440F551F60
:1037A000416002960C5F1F4F2091321330E024508D
:1037B0003109821793070CF004C298012250310995
:1037C000D9012D913C912950310928303105D0F291
:1037D000809132138032E1F48281938106970697BB
:1037E000B8F4848195810997099790F49F012A5F25
:1037F0003F4FAF01425C5F4F812C912C5401D901A6
:103800006D917C91665071096630710508F4F3C1C1
:10381000D7011C962D903C901D97B6E02B163104D5
:103820000CF461CF8F010A5F1F4F73E0C72ED12CBC
:10383000E5EC8E2EEDE99E2EECE1AE2EE1E8BE2EFB
:10384000F8016081718134976080718080E090E040
:103850000E94C8616D837E838F839887B30180E067
:1038600090E00E94C8612B013C012DEC3CEC4CE443
:103870005FE30E9429629B01AC016D817E818F8193
:1038800098850E94C46187FD19C02DEC3CEC4CE486
:103890005FE36D817E818F8198850E9429629B0103
:1038A000AC01C301B2010E94C461E82F880FFF0B75
:1038B000EE27FF0FEE1FFF27319602C0E0E0F0E099
:1038C000A501940163E971E080E091E00E947266D5
:1038D0004F01FF0FAA08BB0886269726A826B926FF
:1038E000FFEFCF1ADF0A0E5F1F4FC214D30409F097
:1038F000A7CFD70114968D929D92AD92BC92179747
:1039000080E290E019969C938E9318978FEF9FEF2B
:10391000E5CE84819581CA97899708F07ECE9F0174
:103920002A5F3F4F812C912C540143E050E0D90194
:103930006D917C916A5071096930710508F06DCE06
:10394000D90112966D917C9113976651710961317D
:10395000710550F5D501C401880F991FAA1FBB1F1F
:103960004C015D01689480F84E5F5F4F2C5F3F4FC4
:103970004B335105E1F69F012A583F4FD9012D9154
:103980003C912A5031092930310508F046CE2CE10E
:1039900030E0F70131872087D70184829582A682A3
:1039A000B7828AE090E09ACED90112966D917C910F
:1039B0001397665071096730710508F02ECE880C98
:1039C000991CAA1CBB1CD0CF20913213CF01820FAF
:1039D000911D820F911DDC0112978D919C910A9788
:1039E000099708F01FCEF701118610868FEF9FEF21
:1039F000DC0184839583A683B78386E090E044CC82
:103A000080913213813208F415CE84819581CA9752
:103A1000899708F00FCE9F012A5F3F4F812C912C90
:103A2000540143E050E0D9016D917C916A507109D5
:103A30006930710508F0FECDD90112966D917C9127
:103A40001397665171096131710570F112966D918C
:103A50007C911397665071096730710508F0EACDC3
:103A6000880C991CAA1CBB1C4E5F5F4F2C5F3F4FFC
:103A700043325105C1F69F012A5B3F4FD9012D9179
:103A80003C912A5031092930310508F0D3CD20E18D
:103A900030E0F70131872087D70184829582A682A2
:103AA000B78286E090E01ACED501C401880F991F35
:103AB000AA1FBB1F4C015D01689480F8D5CF868199
:103AC00097810997099708F0C6CDD70119961C92DE
:103AD0001E9218978FEF9FEFDC01F7018483958387
:103AE000A683B78387E090E0CFCBD90112966D9182
:103AF0007C911397665071096730710508F005CE07
:103B0000880C991CAA1CBB1CD8CD8481958109976F
:103B1000099708F02ACE868197818C974F9708F0F5
:103B200024CE8085918589974D9708F01ECE9F0100
:103B3000265F3F4F812C912C540145E050E00DCE83
:103B40009F0126573F4FD9012D913C912C503109AF
:103B50002B30310508F009CE20E230E0F701318743
:103B60002087D70184829582A682B78288E090E080
:103B7000B5CDD90112966D917C9113976950710959
:103B80006930710508F0F1CD880C991CAA1CBB1C8A
:103B9000DCCD84819581825491098E9708F018CEEE
:103BA0008F01045C1F4F8DE190E040E050E0FCCDC0
:103BB000D8012D913C912851310922313105C0F0B5
:103BC000CB01019795958795D70119969C938E9374
:103BD00018978A970CF4FCCD052E000C660B770B1A
:103BE000F701448355836683778389E090E04CCB6B
:103BF000440F551FD6CDD90112966D917C91139724
:103C00006951710963317105E8F4D501C401880F68
:103C1000991FAA1FBB1F4C015D01689480F82C5F9F
:103C20003F4F2417350709F0EACD2EE030E0F701C9
:103C300031872087D70184829582A682B7828FE060
:103C400090E04CCDD90112966D917C9113976950FB
:103C500071096930710508F0DBCD880C991CAA1C2C
:103C6000BB1CDDCF28960FB6F894DEBF0FBECDBFCC
:103C7000DF91CF911F910F91FF90EF90DF90CF9048
:103C8000BF90AF909F908F907F906F905F904F907C
:103C90003F902F9008952F923F924F925F926F9294
:103CA0007F928F929F92AF92BF92CF92DF92EF92CC
:103CB000FF920F931F93CF93DF93CDB7DEB7A497F7
:103CC0000FB6F894DEBF0FBECDBF8C016BEE77E070
:103CD00086E892E10E94803EC8010E947447C801B4
:103CE00006960697F8F0809136109091371080175D
:103CF0009107F1F00E94E44A1093371000933610B8
:103D00004AE0B801CE0101960E94673DBE016F5F97
:103D10007F4F89E194E10E94A23CCE0101960E946E
:103D2000DB3C06C00E3F2FEF120711F40C945E2B04
:103D3000F8013A96E431F10510F00C94342B882701
:103D4000EE58FF4F8F4F0C9494666CE57FE0CE01E8
:103D500001960E949A3D4AE050E061E070E0CE0199
:103D600001960E94EE4ACE0101960E94DB3C8091B2
:103D700021030E940F40BC01990F880B990B0E94F0
:103D8000CA612DE038E643E55BE30E9429626B01DE
:103D90007C0120916303309164034091650350914D
:103DA00066030E94C46118164CF060914B03709139
:103DB0004C0380914D0390914E031BC020917703DB
:103DC000309178034091790350917A03C701B6018D
:103DD0000E94096587FF05C0C701B6010E94F5343E
:103DE00008C060915F0370916003809161039091BE
:103DF000620320E030E048EC52E40E94296220E0B7
:103E000030E048EA51E40E94296220913B0330915E
:103E10003C0340913D0350913E030E941A646B01A4
:103E20007C010E94E44A60E080E00E94B7380E9472
:103E3000914028EE33E040E050E00E942263BA0156
:103E4000A9012AE0CE0101960E940F3DBE016F5FDD
:103E50007F4F87E094E10E94A23CCE0101960E9430
:103E6000DB3C64EF77E087E094E10E94643C67E02C
:103E700074E18EED94E10E94B53D62E370E080E074
:103E800090E00E94594061E080E00E94B73822E053
:103E9000B701A601CE0101960E94E03C6FE078E0F8
:103EA000CE0107960E949A3DBE016F5F7F4FCE0103
:103EB00007960E94533C6EEF77E0F1C06CE57FE01F
:103EC000CE0101960E949A3D4AE050E061E070E028
:103ED000CE0101960E94EE4ACE0101960E94DB3C83
:103EE00080918B0390918C030E94F62B4B015C0117
:103EF000C0908703D0908803E0908903F0908A03F4
:103F00008091830390918403A0918503B0918603EF
:103F1000898F9A8FAB8FBC8F20917F033091800364
:103F200040918103509182032D8F3E8F4F8F58A374
:103F30009C01AD01C701B6010E9453632B013C01F6
:103F400020917B0330917C0340917D0350917E034F
:103F50006D8D7E8D8F8D98A10E9453639B01AC0166
:103F6000C301B2010E941A642B013C0120E030E041
:103F700048E051E4C501B4010E941A644B015C01A0
:103F800020E030E040EC5FE3C701B6010E94296207
:103F90009B01AC01C501B4010E94096518167CF1B2
:103FA00020E030E040E05FE3698D7A8D8B8D9C8D61
:103FB0000E9429629B01AC01C501B4010E94C46149
:103FC00087FD1DC0A7019601C501B4010E9453637E
:103FD000A30192010E941A642D8D3E8D4F8D58A130
:103FE0000E9454639B01AC0160E070E080E291E4C8
:103FF0000E94C8650E94B3646B017C0104C0CC249C
:10400000CA94DC2C76010E94E44A60E080E00E94C1
:10401000B7380E94914028EE33E040E050E00E9423
:104020002263BA01A9012AE0CE0101960E940F3D48
:10403000BE016F5F7F4F87E094E10E94A23CCE01FA
:1040400001960E94DB3C63E078E087E094E10E9407
:10405000643C67E074E18EED94E10E94B53D62E35B
:1040600070E080E090E00E94594061E080E00E94B2
:10407000B7382AE0B701A601CE0101960E943B3D68
:104080006EE078E0CE0107960E949A3DBE016F5F18
:104090007F4FCE0107960E94533C63E178E00E9477
:1040A0003C3CBC018DE094E10E948D3CCE01079622
:1040B0000E94DB3CCE0101960E94DB3C6DE074E186
:1040C0008EED94E10E94B53D62E370E080E090E007
:1040D0000E94594080914A15882311F40C94342B86
:1040E00060E273E080E090E0E3C16CE57FE0CE0148
:1040F00001960E949A3D4AE050E061E070E0CE01F6
:1041000001960E94EE4ACE0101960E94DB3C0E947D
:1041100091406B017C0180913703909138030A979D
:1041200031F48091390390913A030A97B1F089EE06
:1041300091E10E9412368CED95E0A0E0B0E0809312
:10414000ED119093EE11A093EF11B093F01164E68E
:1041500070E080E090E00E9459400E94E44A60E0F4
:1041600080E00E94B73867E178E08EED94E10E942C
:10417000803E62E370E080E090E00E9459400E943F
:104180009140DC01CB018C199D09AE09BF09883B28
:104190009B40A105B10508F069C00E94D83597FD84
:1041A00006C082349105C9F780E090E002C08FEF2D
:1041B0009FEF892B21F7A0EFAA2EAFE0BA2E450181
:1041C0000E94D83597FF07C08091F00F8D34B9F663
:1041D00080E090E009C0D4018D934D01BFE08B16C3
:1041E000B0E19B0669F7F0CFF50121915F01820FE5
:1041F000911DFDE0AF16F0E1BF06B1F79C012E5B0B
:104200003F4F80910D1090E0982F882740910E101D
:10421000840F911D2817390709F0B1CF8091F30F52
:1042200090E0982F88272091F40F820F911D909392
:10423000EF0F8093EE0F8091F50F90E0982F882775
:104240002091F60F820F911D9093ED0F8093EC0F4C
:104250008091F70F90E0982F88272091F80F820F18
:10426000911D9093EB0F8093EA0F89CF0E949140AC
:10427000DC01CB018C199D09AE09BF09883B9B402D
:10428000A105B10508F400C10E94E44A60E080E0A5
:104290000E94B7380E94914028EE33E040E050E0A1
:1042A0000E942263BA01A9012AE0CE0101960E9470
:1042B0000F3DBE016F5F7F4F87E094E10E94A23CFB
:1042C000CE0101960E94DB3C6AE474E087E094E151
:1042D0000E94643C67E074E18EED94E10E94B53D7C
:1042E0006CE271E080E090E00E94594067E278E083
:1042F00087E094E10E94643C60E086E00E94B73869
:1043000068E278E08EED94E10E94803E62E370E026
:1043100080E090E00E94594061E080E00E94B73860
:104320006091EA0F7091EB0F4AE0CE0101960E9476
:10433000673D6091EC0F7091ED0F4AE0CE0107965A
:104340000E94673D6091EE0F7091EF0F4AE0CE0141
:1043500043960E94673DBE016D5E7F4FCE010D9674
:104360000E94923D61EA76E0CE010D960E943C3CAF
:10437000BE01695F7F4F0E94533C61EA76E00E9474
:104380003C3CBE016F5F7F4F0E94533CBC018DE0FF
:1043900094E10E948D3CCE010D960E94DB3CCE0143
:1043A00043960E94DB3CCE0107960E94DB3CCE0187
:1043B00001960E94DB3C6DE074E18EED94E10E9479
:1043C000B53D61E08CE00E94B73864E478E08EEDA2
:1043D00094E10E94803E6091EA0F7091EB0F4AE0F9
:1043E000CE0101960E94673D6091EC0F7091ED0F38
:1043F0004AE0CE0107960E94673D6091EE0F7091F2
:10440000EF0F4AE0CE010D960E94673D63E378E02E
:10441000CE0143960E949A3DBE01635F7F4FCE015D
:1044200043960E94533C60E87FE00E943C3CBE0102
:10443000695F7F4F0E94533C60E87FE00E943C3CF4
:10444000BE016F5F7F4F0E94533C63E478E00E949F
:104450003C3CBC018DE094E10E948D3CCE01439632
:104460000E94DB3CCE010D960E94DB3CCE010796FC
:104470000E94DB3CCE0101960E94DB3C62E370E0CF
:1044800080E090E00E94594080913703909138037A
:104490000A9741F48091390390913A030A9711F4F5
:1044A0000C94342B0E942E4962E370E080E090E08F
:1044B0000E9459400C94342B9091331081E089274D
:1044C0008093331080914A15882331F06DE074E1B8
:1044D0008CE491E10E94703E68EC70E080E090E036
:1044E000E7CF10924A150C94342B81E080934A1543
:1044F0000C94342B69E478E0CE0107960E949A3D33
:1045000068ED74E1CE0107960E94533CBC01CE01D8
:1045100001960E94923D48EE53E060E070E0CE01CB
:1045200001960E94EE4ACE0101960E94DB3CCE012C
:1045300007960E94DB3C6DE478E0CE0101960E9474
:104540009A3D40ED57E061E070E0CE0101960E9497
:10455000EE4ACE0101960E94DB3C6DE578E0CE018B
:1045600001960E949A3D48EC50E060E070E0CE0178
:1045700001960E94EE4ACE0101960E94DB3C6DE658
:1045800078E0CE0101960E949A3D40ED57E061E04F
:1045900070E0CE0101960E94EE4ACE0101960E9483
:1045A000DB3C6AE778E0CE0101960E949A3D48EC38
:1045B00050E060E070E0CE0101960E94EE4ACE012C
:1045C00001960E94DB3C67E878E0CE0101960E94EC
:1045D0009A3D40ED57E061E070E0CE0101960E9407
:1045E000EE4ACE0101960E94DB3C62E978E0CE0102
:1045F00001960E949A3D48EC50E060E070E0CE01E8
:1046000001960E94EE4ACE0101960E94DB3C6EE9C3
:1046100078E0CE0101960E949A3D40ED57E061E0BE
:1046200070E0CE0101960E94EE4ACE0101960E94F2
:10463000DB3C6FEA78E0CE0101960E949A3D48EC9F
:1046400050E060E070E0CE0101960E94EE4ACE019B
:1046500001960E94DB3C69EB78E0CE0101960E9456
:104660009A3D40ED57E061E070E0CE0101960E9476
:10467000EE4ACE0101960E94DB3C64EC78E0CE016C
:1046800001960E949A3D48EC50E060E070E0CE0157
:1046900001960E94EE4ACE0101960E94DB3C61ED3C
:1046A00078E0CE0101960E949A3D40ED57E061E02E
:1046B00070E0CE0101960E94EE4ACE0101960E9462
:1046C000DB3C60EE78E0CE0101960E949A3D48EC1A
:1046D00050E060E070E0CE0101960E94EE4ACE010B
:1046E00001960E94DB3C6DEE78E0CE0101960E94BF
:1046F0009A3D40ED57E061E070E0CE0101960E94E6
:10470000EE4ACE0101960E94DB3C6DEF78E0CE01CF
:1047100001960E949A3D48EC50E060E070E0CE01C6
:1047200001960E94EE4ACE0101960E94DB3C6AE0AF
:1047300079E0CE0101960E949A3D40ED57E061E09C
:1047400070E0CE0101960E94EE4ACE0101960E94D1
:10475000DB3C66E179E0CE0101960E949A3D48EC8F
:1047600050E060E070E0CE0101960E94EE4ACE017A
:1047700001960E94DB3C62E279E0CE0101960E9444
:104780009A3D40ED57E061E070E0CE0101960E9455
:10479000EE4ACE0101960E94DB3C66C76CE57FE0E5
:1047A000CE0101960E949A3D4AE050E061E070E03F
:1047B000CE0101960E94EE4ACE0101960E94DB3C9A
:1047C00080912703909128030E944B494DC76CE5C7
:1047D0007FE0CE0101960E949A3D4AE050E061E000
:1047E00070E0CE0101960E94EE4ACE0101960E9431
:1047F000DB3C0E945E2C38C780911E03882309F49D
:1048000033C76CE57FE0CE0101960E949A3D4AE0F5
:1048100050E061E070E0CE0101960E94EE4ACE01C8
:1048200001960E94DB3C0E94E44A6EE170E080E069
:1048300090E00E9459400E9406452B013C0164E62D
:1048400070E080E090E00E9459400E947F394B0167
:104850005C0164E670E080E090E00E945940609165
:104860004703709148038091490390914A030E9445
:10487000CA619B01AC0169A33AA34BA35CA30E944C
:1048800006450E94CA6129A13AA14BA15CA10E94E0
:104890001A6421E03EED42E45EE30E94C8659B019C
:1048A000AC0160E070E080E89FE30E94536320E089
:1048B0003AE24DE257E40E9429626B017C0164E612
:1048C00070E080E090E00E94594060E080E00E944B
:1048D000B7380E94914028EE33E040E050E00E945B
:1048E0002263BA01A9012AE0CE0107960E940F3D7A
:1048F000BE01695F7F4FCE0101960E94923D69E142
:1049000075E0CE0101960E943C3CBC0187E094E139
:104910000E948D3CCE0101960E94DB3CCE010796A1
:104920000E94DB3CC301B2010E94CA6120E030E07A
:1049300048EC52E40E941A64AB01BC0122E030E072
:10494000CE0101960E94134BBE016F5F7F4F81E045
:1049500094E10E94A23CCE0101960E94DB3C6DE6F0
:1049600075E081E094E10E94643C61E074E187E0DD
:1049700094E10E94723C69E675E0CE0101960E94C6
:104980009A3D61E074E1CE0101960E94533CBC0166
:1049900081E094E10E948D3CCE0101960E94DB3CB7
:1049A00064E670E080E090E00E9459406EE775E0B8
:1049B0008DE094E10E94783C21E030E0B501A40153
:1049C000CE0101960E94134BBE016F5F7F4F8DE0B9
:1049D00094E10E94723CCE0101960E94DB3C6DE2A4
:1049E00079E08DE094E10E94643C21E030E0B70181
:1049F000A601CE0107960E94134BBE01695F7F4F4F
:104A0000CE0101960E94923D68E377E0CE010196C7
:104A10000E943C3CBC018DE094E10E94723CCE01BE
:104A200001960E94DB3CCE0107960E94DB3C61E0D0
:104A300074E1CE0101960E94923D60E87FE0CE01D4
:104A400001960E943C3C6DE074E10E94533CBC0125
:104A50008DE094E10E948D3CCE0101960E94DB3CEA
:104A600067E074E18EED94E10E94B53D21E030E015
:104A7000B501A401CE0107960E94134BBE01695FE8
:104A80007F4FCE0101960E94923D63E379E0CE0113
:104A900001960E943C3CBC0183E194E10E948D3C64
:104AA000CE0101960E94DB3CCE0107960E94DB3CC2
:104AB00021E030E0B701A601CE0107960E94134B1A
:104AC000BE01695F7F4FCE0101960E94923D68E36F
:104AD00077E0CE0101960E943C3CBC0183E194E169
:104AE0000E94723CCE0101960E94DB3CCE010796EB
:104AF0000E94DB3C61E080E00E94B73863E174E132
:104B00008EED94E10E94B53D64E670E080E090E0B7
:104B10000E94594080914A15882309F4A5C568E58B
:104B200072E080E090E0C4CC6CE57FE0CE010196BD
:104B30000E949A3D4AE050E061E070E0CE010196AB
:104B40000E94EE4ACE0101960E94DB3C80914A15FC
:104B5000882349F082E090E0A0E0B0E0898F9A8F4E
:104B6000AB8FBC8F08C02EE130E040E050E0298FD1
:104B70003A8F4B8F5C8F68E379E08DE094E10E947F
:104B8000783C61E080E00E94B7386DE074E18EED22
:104B900094E10E94B53D812C912C5401C12CD12C63
:104BA000760183E20E94CC3687E090E00E9439369D
:104BB0000E946F3666E970E080E090E00E94594004
:104BC00083E20E94CC3680E290E00E9439360E9457
:104BD0006F3666E970E080E090E00E94594062E044
:104BE00070E083E290E00E943539412C512C320173
:104BF0008091661090E020916710821B9109181631
:104C0000190664F483E293E172D5762C652C542C5A
:104C10004424480E511C611C711CEACFC301B2012F
:104C20000E94CA612AE939E949E95FE30E941A64EE
:104C30000E94B3642B013C01C616D706E806F906AC
:104C40000CF04BC00E94914028EE33E040E050E071
:104C50000E942263BA01A9012AE0CE0101960E94B6
:104C60000F3DBE016F5F7F4F87E094E10E94A23C41
:104C7000CE0101960E94DB3C2AE0B301A201CE01E5
:104C800001960E943B3D68E479E0CE0107960E94C0
:104C90009A3DBE016F5F7F4FCE0107960E94533C45
:104CA0006DE479E00E943C3CBC0187E094E10E9405
:104CB000723CCE0107960E94DB3CCE0101960E9419
:104CC000DB3C60E080E00E94B73867E074E18EED85
:104CD00094E10E94B53D7301620162E370E080E0FF
:104CE00090E00E9459403FEF831A930AA30AB30A47
:104CF000898D9A8DAB8DBC8D88159905AA05BB054C
:104D00000CF04FCF2AE0B701A601CE0101960E9418
:104D10003B3D61E579E0CE0107960E949A3DBE01D8
:104D20006F5F7F4FCE0107960E94533C64E579E0A8
:104D30000E943C3C6DE074E10E94533CBC018DE05C
:104D400094E10E948D3CCE0107960E94DB3CCE018F
:104D500001960E94DB3CA8CB6CE57FE0CE0101967A
:104D60000E949A3D4AE050E061E070E0CE01019679
:104D70000E94EE4ACE0101960E94DB3C81E08093C6
:104D8000A50364E670E080E090E00E9459400E9434
:104D9000E44A60E080E00E94B7380E94914028EE2B
:104DA00033E040E050E00E942263BA01A9012AE00A
:104DB0008EED94E10E94D83D6AE474E08EED94E1BA
:104DC0000E94803E88E30E940F4060E074E0681B10
:104DD000790B4AE0CE0101960E94673D69E579E0D2
:104DE000CE0107960E949A3DBE016F5F7F4FCE01B4
:104DF00007960E94533CBC018DE094E10E948D3CDB
:104E0000CE0107960E94DB3CCE0101960E94DB3C5E
:104E100060E086E00E94B73869E878E08EED94E1C2
:104E20000E94803E61E080E00E94B7386DE074E14E
:104E30008EED94E10E94B53D60E679E0CE010196E9
:104E40000E949A3D6DE074E1CE0101960E94533CB0
:104E5000BC018DE094E10E948D3CCE0101960E9440
:104E6000DB3C64E670E080E090E032C96CE57FE016
:104E7000CE0101960E949A3D4AE050E061E070E068
:104E8000CE0101960E94EE4ACE0101960E94DB3CC3
:104E9000F0901F030E94E44A60E080E00E94B7386F
:104EA0000E94914028EE33E040E050E00E942263EF
:104EB000BA01A9012AE0CE0101960E940F3DBE0170
:104EC0006F5F7F4F87E094E10E94A23CCE01019684
:104ED0000E94DB3C69E175E087E094E10E94643C5C
:104EE00067E074E18EED94E10E94B53D8F2D0E9444
:104EF0000F409093101080930F1062E370E080E0F9
:104F000090E00E94594060E088E00E94B7386091CC
:104F10000F10709110104AE0CE0101960E94673D7B
:104F2000BE016F5F7F4F8DE094E10E94A23CCE01F5
:104F300001960E94DB3C62E370E080E090E00E941A
:104F4000594080914A15882331F060E273E080E097
:104F500090E00E94594080912F03909130038B3054
:104F600091053CF12FE0289FB001299F700D11247D
:104F7000605F7D4FCE0101960E949A3DBE016F5F3A
:104F80007F4FCE0107960E94923D65E075E0CE010D
:104F900007960E943C3C6DE074E10E94533CBC01CA
:104FA0008DE094E10E948D3CCE0107960E94DB3C8F
:104FB00011C06AE679E0CE0101960E949A3D6DE04B
:104FC00074E1CE0101960E94533CBC018DE094E156
:104FD0000E948D3CCE0101960E94DB3C61E080E0A6
:104FE0000E94B73800C380911E03882309F43CC394
:104FF00080914A15882329F082E090E00E94804B3E
:1050000033C3C0900C02D0900D02E0900E02F090DD
:105010000F0220E030E040E450E4C701B6010E94F6
:10502000096518166CF420E030E04AE754E4C70143
:10503000B6010E9429620E94B3646B017C0106C024
:1050400070E3C72E75E7D72EE12CF12C0E94E44ABD
:1050500060E080E00E94B73865E779E08EED94E18A
:105060000E94803E61E080E00E94B73866E879E007
:105070008EED94E10E94803E68EC70E080E090E06C
:105080000E9459400E9491406093E60F7093E70F91
:105090008093E80F9093E90F0E9491402B013C010F
:1050A00062E3862E912CA12CB12C8091E60F909179
:1050B000E70FA091E80FB091E90FA3019201281B1F
:1050C000390B4A0B5B0B2C153D054E055F050CF0AB
:1050D000CBC283E090E00E94804B0E949140DC01B3
:1050E000CB0184199509A609B70988329105A10554
:1050F000B10554F4A5019401281B390B4A0B5B0B35
:10510000CA01B9010E9459400E9491402B013C0103
:10511000CCCF6CE57FE0CE0101960E949A3D4AE03B
:1051200050E061E070E0CE0101960E94EE4ACE01AF
:1051300001960E94DB3C0E94914028EE33E040E063
:1051400050E00E942263BA01A9012AE0CE01019633
:105150000E940F3DBE016F5F7F4F87E094E10E9488
:10516000A23CCE0101960E94DB3C67E074E1CE01D7
:1051700001960E94923D6EE879E0CE0101960E9470
:105180003C3CBC0187E094E10E948D3CCE0101963D
:105190000E94DB3C80914A15811102C00E94E44AC2
:1051A00080913703909138030A9771F48091390305
:1051B00090913A030A9741F40E942E4964E670E008
:1051C00080E090E00E9459408CE40E946F486B019F
:1051D0007C019B01AC010E945966882339F062E989
:1051E00079E08DE094E10E94783C97C021E030E0C6
:1051F000B701A601CE0101960E94134B6CE979E03C
:10520000CE0107960E949A3DBE016F5F7F4FCE018F
:1052100007960E94533C65EA79E00E943C3CBC0141
:105220008DE094E10E948D3CCE0107960E94DB3C0C
:10523000CE0101960E94DB3C61E080E00E94B7381D
:105240006DE074E18EED94E10E94B53D62E370E0A3
:1052500080E090E00E94594086E60E946F48AB01D2
:10526000BC0121E030E0CE0101960E94134B6EE7B5
:1052700075E0CE0107960E949A3DBE016F5F7F4F99
:10528000CE0107960E94533C65EA79E00E943C3CBF
:10529000BC0183E194E10E948D3CCE0107960E94FF
:1052A000DB3CCE0101960E94DB3C60E87FE0CE0152
:1052B00001960E949A3D63E174E1CE0101960E943D
:1052C000533CBC0187E094E10E94723CCE01019600
:1052D0000E94DB3C60E080E00E94B73867E074E148
:1052E0008EED94E10E94B53D63E174E1CE0101963B
:1052F0000E94923D60E87FE0CE0101960E943C3C16
:105300006DE074E10E94533CBC018DE094E10E9489
:105310008D3CCE0101960E94DB3C80913703909139
:1053200038030A97B1F48091390390913A030A97B0
:1053300081F489EE91E10E9412368CED95E0A0E0B7
:10534000B0E08093ED119093EE11A093EF11B09324
:10535000F01164E670E080E090E00E945940809196
:105360004A15882331F060E273E080E090E00E940B
:1053700059408CE491E10E94053B76C16CE57FE0E9
:10538000CE0101960E949A3D4AE050E061E070E053
:10539000CE0101960E94EE4ACE0101960E94DB3CAE
:1053A0000E94E44A60E080E00E94B73860E080E05C
:1053B0000E94B7380E94914028EE33E040E050E070
:1053C0000E942263BA01A9012AE0CE0101960E943F
:1053D0000F3DBE016F5F7F4F87E094E10E94A23CCA
:1053E000CE0101960E94DB3C69E175E087E094E123
:1053F0000E94643C67E074E18EED94E10E94B53D4B
:1054000061E080E00E94B73830912303398F8091AA
:105410002B1081110DC00E94914060932710709352
:1054200028108093291090932A1081E080932B10EC
:1054300080911F1081110DC00E94914060931B103C
:1054400070931C1080931D1090931E1081E0809328
:105450001F1010921A1010921910209019103090ED
:105460001A1058E2251631040CF084C0898D0E9470
:105470000F40F101EE0FFF1FE450FF4E9183808338
:105480000E94D63320E030E040EA50E40E942962D6
:1054900020E030E040E85AE30E9429626B017C0181
:1054A0006093151070931610809317109093181036
:1054B000409004025090050260900602709007022E
:1054C000A3019201609108027091090280910A0281
:1054D00090910B020E9453639B01AC0160E070E06D
:1054E00080EC90E40E9453634B015C0120E030E0CB
:1054F000A9010E94C46120E030E040E650E481113F
:1055000005C0C701B6010E9429621EC0C701B601CD
:105510000E942962A30192010E94546320E030E0BE
:1055200040E850E40E945363A50194010E941A646C
:1055300020E030E040EC50E40E94296220E030E0BE
:1055400040E850E40E94546360931110709312106D
:10555000809313109093141064E170E080E090E069
:105560000E9459404FEF241A340A30921A102092A8
:10557000191073CFC0901110D0901210E09013103A
:10558000F090141020E030E0A901C701B6010E949C
:10559000096587FD22C022E0B701A601CE01019670
:1055A0000E94E03C68EA79E0CE0107960E949A3DAD
:1055B000BE016F5F7F4FCE0107960E94533CBC0136
:1055C0008DE094E10E948D3CCE0107960E94DB3C69
:1055D000CE0101960E94DB3C06C06CEA79E08DE0CA
:1055E00094E10E94783C6DE074E18EED94E10E94BC
:1055F000B53D3AC080911E038823B1F16CE57FE090
:10560000CE0101960E949A3D4AE050E061E070E0D0
:10561000CE0101960E94EE4ACE0101960E94DB3C2B
:1056200080914A15811117C020E030E040EA51E432
:1056300060910C0270910D0280910E0290910F0208
:105640000E9429620E94B3649B01AC016AE070E091
:1056500080E090E008C021E030E040E050E064EFFE
:1056600071E080E090E0DDD361E080E00E94B73837
:105670008091111490911214009791F0419718F4B1
:1056800002301105A4F46DE074E1CE0101960E9490
:10569000923DCE010196B6D3CE0101960E94DB3C2D
:1056A00064E670E080E090E00E94594007C06DE041
:1056B00074E18EED94E10E94B53DE5CFA4960FB65E
:1056C000F894DEBF0FBECDBFDF91CF911F910F9138
:1056D000FF90EF90DF90CF90BF90AF909F908F9012
:1056E0007F906F905F904F903F902F900895909192
:1056F000671080916610981750F4E92FF0E0EA5B8C
:10570000FF4E208130E09F5F9093671002C02FEF23
:105710003FEFC90108958091661090E020916710D5
:10572000821B91090895089580E090E00895CF923A
:10573000DF92EF92FF920F931F93CF93DF937C0141
:10574000262F972F8A0180918F10882391F0C62FE2
:10575000D72F6E01C40ED51ECC15DD0571F06991F1
:10576000D701ED91FC910190F081E02DC7011995D1
:10577000F3CF642F822F0E94BB44C801DF91CF91E9
:105780001F910F91FF90EF90DF90CF900895CF93EE
:10579000DF931F92CDB7DEB7698320918F1022234C
:1057A000D1F02091B110203240F021E030E0FC0136
:1057B0003383228380E090E015C080919010E82F21
:1057C000F0E0EF56FF4E998190838F5F80939010A9
:1057D0008093B11005C061E0CE0101960E94BB44E8
:1057E00081E090E00F90DF91CF910895CF92DF920A
:1057F000EF92FF921F93CF93DF93182FCAE0D0E070
:10580000C12CD12C7601812F0E940F40BC01990F31
:10581000880B990B0E94CA619B01AC01C701B601BC
:105820000E9454636B017C0162E370E080E090E0D1
:105830000E945940219739F720E030E040E251E4DE
:10584000C701B6010E941A6420E030E040EA50E44B
:105850000E94296220E030E040E85AE30E94296279
:10586000DF91CF911F91FF90EF90DF90CF9008953F
:105870001F93CF93DF93182FCCEFD0E1812F0E949D
:105880000F40899399936CE370E080E090E00E9470
:10589000594081E1CC34D80789F788D720E030E03F
:1058A00040EA50E40E94296220E030E040E85AE3F8
:1058B0000E942962DF91CF911F9108954F925F92CC
:1058C0006F927F928F929F92AF92BF92CF92DF9210
:1058D000EF92FF920F931F93CF93DF93CDB7DEB775
:1058E0002C970FB6F894DEBF0FBECDBF61E080E00D
:1058F0000E94B7386BE77EE08EED94E10E94803E17
:1059000064EF71E080E090E00E94594060E080E048
:105910000E94B7380E94914028EE33E040E050E00A
:105920000E942263BA01A9012AE08EED94E10E944F
:10593000D83D6CE87EE08EED94E10E94803E1982B5
:105940001A821B821C821D8261E087E30E94D33F82
:1059500060E087E30E94A13F62E170E080E090E0B8
:105960000E94594061E087E30E94A13F8BE990E0EB
:105970000197F1F760E087E30E94D33F01E117E26E
:1059800087E30E94773F892B31F401501109C1F759
:105990008EEF9FEF72C001E117E287E30E94773F2D
:1059A000019721F401501109C1F7F2CF28E2E22E4C
:1059B000F12C17E0D12CAA24A394B12C91E1892ECB
:1059C00097E2992E87E30E94773F892B29F481E0A3
:1059D000881A9108B9F7DCCF0E9434402B013C01B2
:1059E00081E1882E87E2982E87E30E94773F019716
:1059F00029F481E0881A9108B9F7CACF0E9434408F
:105A0000DC01CB0184199509A609B7098997A1057D
:105A1000B10578F0E1E0F0E0EC0FFD1FED0DF11DB8
:105A20002081C501012E01C0880F0A94EAF7822B5C
:105A30008083111103C0D39417E001C0115081E09D
:105A4000E81AF10809F0BACF8981282F30E03093A5
:105A50004310209342102B81422F50E05093451069
:105A600040934410280F81E090E03D81321302C042
:105A700080E090E0919581959109892B09F025C1ED
:105A80006091441070914510072E000C880B990B03
:105A90000E94CA616B017C0160933E1070933F10BD
:105AA0008093401090934110809142109091431048
:105AB000BC01990F880B990B0E94CA6160933A1040
:105AC00070933B1080933C1090933D1021E030E0A8
:105AD000B701A601CE0107960E94134B6EE775E051
:105AE000CE0101960E949A3DBE01695F7F4FCE01B3
:105AF00001960E94533CBC018DE094E10E948D3CD4
:105B0000CE0101960E94DB3CCE0107960E94DB3C51
:105B100040913A1050913B1060913C1070913D10B3
:105B200021E030E0CE0107960E94134B62E97EE04F
:105B3000CE0101960E949A3DBE01695F7F4FCE0162
:105B400001960E94533CBC018DE094E10E94723C9E
:105B5000CE0101960E94DB3CCE0107960E94DB3C01
:105B600061E078E08DE094E10E94643C60E086E0D2
:105B70000E94B73860913E1070913F1080914010A4
:105B8000909141100E94B3644AE050E08EED94E1A0
:105B90000E94673E6FED8EED94E10E94AE3D68E994
:105BA0007EE08EED94E10E94803E60913A1070910B
:105BB0003B1080913C1090913D100E94B3644AE0EC
:105BC00050E08EED94E10E94673E6BE97EE08EED41
:105BD00094E10E94803E64E670E080E090E00E94E4
:105BE000594089E194E10E94043C613071058105CE
:105BF000910509F0F0C061E080E00E94B73862E7EB
:105C00007FE08EED94E10E94803E61E080E00E94A2
:105C1000B738C0903E10D0903F10E0904010F09008
:105C2000411020E030E040EF51E4C701B6010E948E
:105C3000096587FD03C06FE97EE03CC020E030E0ED
:105C400040ED51E4C701B6010E94096587FD13C00C
:105C50006FEA7EE08EED94E10E94803E6CED75E08F
:105C600080E090E00E94594061E080E00E94B738F7
:105C70006FEB7EE01FC020E030E040EB51E4C70155
:105C8000B6010E94096587FD03C06FEC7EE012C07B
:105C90006FED7EE08EED94E10E94803E6CED75E04C
:105CA00080E090E00E94594061E080E00E94B738B7
:105CB0006FEE7EE08EED94E10E94803E6CED75E02B
:105CC00080E090E00E94594086C00E94E44A6EE164
:105CD00070E080E090E00E9459400E947F396B01A3
:105CE0007C0164E670E080E090E00E94594060E052
:105CF00080E00E94B7380E94914028EE33E040E0F7
:105D000050E00E942263BA01A9012AE0CE01079661
:105D10000E940F3DBE01695F7F4FCE0101960E9438
:105D2000923D69E175E0CE0101960E943C3CBC01C8
:105D300087E094E10E948D3CCE0101960E94DB3CFD
:105D4000CE0107960E94DB3C6EE775E08DE094E1A2
:105D50000E94783C21E030E0B701A601CE01019617
:105D60000E94134BBE016F5F7F4F8DE094E10E9454
:105D7000723CCE0101960E94DB3C65EA79E08DE041
:105D800094E10E94643C67E074E1CE0101960E94B8
:105D9000923D6DE074E1CE0101960E94533CBC013E
:105DA0008DE094E10E948D3CCE0101960E94DB3C87
:105DB0006DE074E18EED94E10E94B53D61E080E01C
:105DC0000E94B738C0923E10D0923F10E09240102F
:105DD000F092411026CF2C960FB6F894DEBF0FBE7E
:105DE000CDBFDF91CF911F910F91FF90EF90DF908A
:105DF000CF90BF90AF909F908F907F906F905F906B
:105E00004F900895CF93DF93EC01BC0186E892E1B7
:105E10000E94703EBE018CE491E1DF91CF910C9421
:105E2000703E2F923F924F925F926F927F928F922D
:105E30009F92AF92BF92CF92DF92EF92FF920F9319
:105E40001F93CF93DF93CDB7DEB7C354D1090FB6FD
:105E5000F894DEBF0FBECDBF6EAF7FAF1C0129AB84
:105E60003AAB4BAB5CAB0E94914024966CAF7DAFDC
:105E70008EAF9FAF249729A93AA94BA95CA92A30D4
:105E80003105410551052CF42DA73EA74FA758AB6E
:105E900008C08AE090E0A0E0B0E08DA79EA7AFA781
:105EA000B8AB80914A15882341F029A93AA94BA99A
:105EB0005CA92DA73EA74FA758AB31E03DAF94EFAB
:105EC000492E55245394612C712C19A61AA61BA691
:105ED0001CA68E01035F1F4F89A59AA5ABA5BCA583
:105EE0002DA53EA54FA558A982179307A407B5076E
:105EF0000CF0DCC20E94914024962CAD3DAD4EAD1D
:105F00005FAD2497621B730B840B950B0E94C861D5
:105F100020E030E04AE754E40E941A64AB01BC017F
:105F200022E030E0C8010E94134BB80187E094E101
:105F30000E94A23CC8010E94DB3CCE0101960E9457
:105F4000F8476FEF7EE08DE094E10E94783CAE016F
:105F50004F5F5F4F5EA34DA3C12CD12C7601ADA145
:105F6000BEA18D909D90AD90BD90BEA3ADA3A501A7
:105F70009401C501B4010E9429629B01AC01C701D3
:105F8000B6010E9454636B017C0123E030E0B5014F
:105F9000A401C8010E94134BB801CE0143960E9490
:105FA000923D60E87FE0CE0143960E943C3CBC01FC
:105FB0008DE094E10E94723CCE0143960E94DB3C4E
:105FC000C8010E94DB3CEDA1FEA1E017F10739F604
:105FD000C701B6010E9418666B017C01FDE24F16F5
:105FE000F1E05F066104710434F00E94E44A60E06D
:105FF00080E00E94B73823E030E0B701A601CE016F
:1060000043960E94134B6BE57FE0C8010E949A3DC6
:1060100067E074E1C8010E94533C6CE07FE00E949D
:106020003C3CBE016D5E7F4F0E94533C61E17FE0CE
:106030000E943C3CBC018DE094E10E94723CC8018E
:106040000E94DB3CCE0143960E94DB3C26E636E60E
:1060500046E65FE3C701B6010E94096589849A8418
:10606000AB84BC8418160CF081C12DEC3CEC4CE8E0
:106070005FE3C701B6010E94C46187FF83C12DADF4
:10608000222309F48AC120E030E0A901C501B4014E
:106090000E94C461C980DA80EB80FC802D813E8142
:1060A0004F8158852DA33EA34FA358A7882309F1FC
:1060B000A7019601C701B6010E9429626DAB7EABB4
:1060C0008FAB98AF2DA13EA14FA158A5CA01B90130
:1060D0000E9429629B01AC016DA97EA98FA998AD90
:1060E0000E9454630E941866A50194010E94C76330
:1060F00004C06BED7FE089EC9FE320EE3EE245E6D5
:1061000052E40E9429626DAB7EAB8FAB98AF20E06A
:1061100030E0A9016DA17EA18FA198A50E94C46164
:10612000882309F1A7019601C701B6010E942962DF
:1061300069AF7AAF8BAF9CAFA5019401C501B401E3
:106140000E9429629B01AC0169AD7AAD8BAD9CAD1B
:106150000E9454630E9418662DA13EA14FA158A52C
:106160000E94C76304C06BED7FE089EC9FE320EEE3
:106170003EE245E652E40E94296269AF7AAF8BAFF6
:106180009CAF20E030E0A901C701B6010E94C461C4
:106190008823F9F0A5019401C501B4010E94296288
:1061A0004B015C012DA13EA14FA158A5CA01B90127
:1061B0000E9429629B01AC01C501B4010E94546395
:1061C0000E941866A70196010E94C7636B017C01BB
:1061D00008C08BEDC82E8FE0D82E89ECE82E8FE317
:1061E000F82E64E17FE08DE094E10E94783C0E940B
:1061F000914028EE33E040E050E00E942263BA0173
:10620000A9012AE0C8010E940F3DB801CE014396C2
:106210000E94923D6CE27FE0CE0143960E943C3C9E
:10622000BC0187E094E10E948D3CCE0143960E9420
:10623000DB3CC8010E94DB3C21E04DA95EA96FA9AF
:1062400078ADCE014F960E94E03C21E049AD5AADB9
:106250006BAD7CADCE0149960E94E03C20EE3EE263
:1062600045E652E4C701B6010E942962AB01BC01B8
:1062700021E0C8010E94E03CB801CE0143960E9493
:10628000923D60E87FE0CE0143960E943C3CBE0117
:10629000675E7F4F0E94533C60E87FE00E943C3C79
:1062A000BE01615E7F4F0E94533CBC0181E094E1DE
:1062B0000E948D3CCE0143960E94DB3CC8010E94A7
:1062C000DB3CCE0149960E94DB3CCE014F960E94FA
:1062D000DB3C3DE2431631E053066104710444F4B3
:1062E00089A59AA5ABA5BCA5892B8A2B8B2B79F404
:1062F00067E074E18EED94E10E94B53D61E080E0DD
:1063000036D761E074E18EED94E10E94B53D61E025
:1063100074E18DE094E10E94723C9DE2491691E0A7
:1063200059066104710444F429A53AA54BA55CA55E
:10633000232B242B252B51F46DE074E1C8010E941E
:10634000923DC8015FDDC8010E94DB3CC301B20180
:106350000E94594089A59AA5ABA5BCA50196A11D8F
:10636000B11D89A79AA7ABA7BCA793C04EAC5FACE1
:10637000310129A93AA94BA95CA92DA73EA74FA78E
:1063800058AB0BC04EAC5FAC310189A99AA9ABA93F
:10639000BCA98DA79EA7AFA7B8AB23E030E0B5019D
:1063A000A401CE0143960E94134B69E37FE0C8012C
:1063B0000E949A3DBE016D5E7F4FC8010E94533C12
:1063C00062E17FE00E943C3CBC0187E094E10E94D6
:1063D000723CC8010E94DB3CCE0143960E94DB3C2C
:1063E0009DE2491691E05906610471044CF067E0A2
:1063F00074E18EED94E10E94B53D61E080E0B7D696
:106400004D815E816F81788523E030E0CE01499631
:106410000E94134B49815A816B817C8123E030E0DB
:10642000C8010E94134BB801CE0143960E94923DD1
:106430006FE37FE0CE0143960E943C3CBE01675E65
:106440007F4F0E94533C62E17FE00E943C3CBC01D4
:1064500081E094E10E948D3CCE0143960E94DB3C9A
:10646000C8010E94DB3CCE0149960E94DB3CADE2B4
:106470004A16A1E05A066104710434F061E074E147
:106480008EED94E10E94B53DC301B2010E945940D6
:106490001DAE29A53AA54BA55CA52F5F3F4F4F4FD9
:1064A0005F4F29A73AA74BA75CA716CD0E94E44AE5
:1064B00061E080E05CD661E074E18EED94E10E94E1
:1064C000B53D60E080E053D667E074E18EED94E185
:1064D0000E94B53DCD5BDF4F0FB6F894DEBF0FBE17
:1064E000CDBFDF91CF911F910F91FF90EF90DF9083
:1064F000CF90BF90AF909F908F907F906F905F9064
:106500004F903F902F900895CF93DF93EC01BC0103
:1065100086E892E10E94B53DBE018CE491E1DF91F5
:10652000CF910C94B53DCF92DF92EF92FF920F93F3
:106530001F93CF93DF93CDB7DEB728970FB6F894AC
:10654000DEBF0FBECDBF823409F4BAC0D4F48033AD
:1065500009F4D6C07CF4833209F4C9C08A3209F048
:10656000EFC061E274E08FE194E10E94783C8FEF2C
:106570009FEFE3C0813309F4D2C0813409F495C0A0
:10658000DFC0813609F491C034F4833409F4A3C028
:10659000843449F0D5C0833609F49DC00CF490C012
:1065A000843609F0CDC089E194E10E94043C1616BE
:1065B0001706180619067CF562E47FE086E892E18A
:1065C0000E94803E69E174E186E892E10E94703E9B
:1065D00089E194E10E94043C0AEF1FEF2FEF3FEFA7
:1065E00068017901C61AD70AE80AF90AB701A601B3
:1065F0002AE0CE0101960E943B3DBE016F5F7F4FB6
:1066000089E194E10E94A23CCE0101960E94DB3C0C
:1066100089E194E146C00E943F4F182FE12CF12CF4
:10662000111112C08FEFE81AF80A89EEE81683E01C
:10663000F80651F06EE170E080E090E00E94594071
:106640000E943F4F182FECCF6AE270E0611B710986
:1066500017FD73954AE0CE0101960E94673DBE0189
:106660006F5F7F4F8FE194E10E94A23CCE010196C3
:106670000E94DB3C6FE174E189E194E10E948D3C72
:1066800062E47FE086E892E10E94803E612F86E826
:1066900092E10E94AE3D86E892E10E946D3E8FE15C
:1066A00094E10E94043CCB0148C068E174E08FE1B2
:1066B00094E10E94783C80913610909137103DC053
:1066C00065E174E08FE194E10E94783C10924A15F4
:1066D0008CEF9FEF32C06BE174E08FE194E10E9498
:1066E000783C81E080934A158DEF9FEF26C06EE1E4
:1066F00074E08FE194E10E94783C8EEF9FEF1DC023
:1067000061E378E089E194E10E94783C61E378E01C
:106710008FE194E10E94783C80E090E00EC062E25C
:1067200074E089E194E10E94783C62E274E08FE1D8
:1067300094E10E94783C81E090E00E944B1E27C0CB
:106740001A8219821C821B821E821D828F831886E8
:10675000BE01695F7F4FCE0101960E94783CBE0169
:106760006F5F7F4F89E194E10E94A23CCE010196C8
:106770000E94DB3C89E194E10E94043CCB010E9431
:106780004B1E64E670E080E090E00E94594028963D
:106790000FB6F894DEBF0FBECDBFDF91CF911F9132
:1067A0000F91FF90EF90DF90CF9008952F923F923E
:1067B0004F925F926F927F928F929F92AF92BF9211
:1067C000CF92DF92EF92FF920F931F93CF93DF93BD
:1067D00000D01F92CDB7DEB74091FC105091FD1054
:1067E000C090FE10D090FF104C155D052CF03C2D94
:1067F0002D2D6A01432F522FE0E0F1E160E070E0BF
:10680000CB01019111910417150754F44A01550F5A
:10681000AA08BB08680D791D8A1D9B1DA80115C01B
:10682000C016D10654F40D2C000CEE08FF086C0DB8
:106830007D1D8E1D9F1D680108C0012E000C220BBE
:10684000330B600F711F821F931F21E1EC34F2079D
:10685000C1F60E94CA6120E030E048E152E40E94A3
:106860001A646B017C010CEF10E1812C912C540116
:10687000D8016D917D918D01072E000C880B990B2D
:106880000E94CA61A70196010E9453639B01AC015B
:106890000E9429629B01AC01C501B4010E945463AE
:1068A0004B015C01B1E10C341B0711F720E030E033
:1068B0004CE152E40E941A640E9418664B015C018C
:1068C00020E030E040E85FE30E94096518160CF014
:1068D00062C00CEF10E1212C312C412C512C3201E3
:1068E000F801819191918F019C01990F440B550BF7
:1068F00029833A834B835C83CA01B9010E94CA6130
:10690000A70196010E9453630E94B3649B0177FF25
:1069100004C022273327261B370BB901330F880BFE
:10692000990B0E94CA61A50194010E94C46187FF6E
:106930000BC089819A81AB81BC81480E591E6A1EA9
:106940007B1E9FEF291A390AA1E10C341A0741F680
:1069500020E030E040EC5FE3C501B4010E94296211
:106960004B015C01B5E02B1631040CF4B2CFC3012E
:10697000B2010E94CA616B017C01B101330C880B2A
:10698000990B0E94CA619B01AC01C701B6010E942C
:106990001A646B017C01C701B6010F900F900F9034
:1069A0000F90DF91CF911F910F91FF90EF90DF90AB
:1069B000CF90BF90AF909F908F907F906F905F909F
:1069C0004F903F902F900895CF93DF93BC0186E8BE
:1069D00092E10E94C33DEC0186E892E10E946D3E87
:1069E0008C0F9D1FDF91CF9108954F925F926F9210
:1069F0007F928F929F92AF92BF92CF92DF92EF924F
:106A0000FF920F931F93CF93DF9300D01F92CDB7C8
:106A1000DEB76B017C0111E0A12EB12C4501880C81
:106A2000991C880C991CF401ED59FC4F4080518051
:106A300062807380A3019201C701B6010E940965BB
:106A4000181614F41F5FE8CFA3019201C701B60125
:106A50000E94C4618401055B1C4F811106C0D801EE
:106A60006D917D918D919C9142C0C5018150904C5A
:106A7000880F991F880F991FFC01ED59FC4F208149
:106A800031814281538129833A834B835C83FC01AA
:106A9000E55BFC4F80809180A280B380C701B60186
:106AA0000E9453636B017C01A5019401D8016D9193
:106AB0007D918D919C910E9453639B01AC01C70114
:106AC000B6010E9429626B017C0129813A814B81C8
:106AD0005C81C301B2010E9453639B01AC01C701F9
:106AE000B6010E941A64A50194010E9454630F909C
:106AF0000F900F900F90DF91CF911F910F91FF900A
:106B0000EF90DF90CF90BF90AF909F908F907F904D
:106B10006F905F904F900895DF92EF92FF920F93E6
:106B20001F93CF93DF937C018B01EA014617570730
:106B300020F4812F8A01C62FD82F6CE57FE0C70192
:106B4000F9D7809123149091241408171907D8F4C9
:106B50008C179D0708F4EC01E0911F14F0912014AC
:106B6000EC0FFD1FD080108260911F1470912014D3
:106B7000600F711FC701BCD6E0911F14F091201463
:106B8000EC0FFD1FD082C701DF91CF911F910F91B4
:106B9000FF90EF90DF900895CF93DF93EC01409149
:106BA000231450912414B8DFCE01DF91CF910895C2
:106BB0000F931F930E9491406093F1117093F21113
:106BC0008093F3119093F411E091E911F091EA119F
:106BD0000284F385E02D89EE91E1199597FF1FC09E
:106BE0000E9491400091F1111091F2112091F31146
:106BF0003091F411DC01CB01801B910BA20BB30B84
:106C00000091ED111091EE112091EF113091F011E2
:106C100080179107A207B307B8F28FEF9FEF1F917C
:106C20000F910895FC01A089B18982E08C93A4851D
:106C3000B5851C92A685B7858FEC8C93108EA489A0
:106C4000B58986E08C93A289B3898C9180618C93FD
:106C5000A289B3898C9188608C93A289B3898C9125
:106C600080688C930288F389E02D80818F7D8083FA
:106C70000895682F83E293E10C94C72BCF92DF92A3
:106C8000EF92FF920F931F93CF93DF931F92CDB795
:106C9000DEB76C0102EB10E17C018AE4E80EF11C26
:106CA000F80161918F01C60169830E94E0626981E8
:106CB000681719F0C6010E94E862FFEFCF1ADF0AD9
:106CC000CE14DF0469F782EB90E10F90DF91CF9152
:106CD0001F910F91FF90EF90DF90CF90089520913A
:106CE000B1109091F714213208F04AC080918E10B3
:106CF0008111FCCF32E030938E1031E030938D1053
:106D00003FEF30938C1010928B1020938A10A1E9E2
:106D1000B0E14AE650E1FA013E2F341B321718F475
:106D20003D913193F9CF1092691020916910990F1C
:106D3000922B9093691090916810913061F41092A9
:106D40006810909169109093BB009091BC0093FDE6
:106D5000F8CF95EC01C095EE9093BC0090918E1009
:106D60009230E1F390918C109F3F79F080918C10DC
:106D7000803241F080918C10803331F084E005C086
:106D800081E003C082E001C083E010929010109275
:106D9000B11010928F10089591E090938F1080930E
:106DA000F714109290101092B11008950F931F9342
:106DB000CF93DF938C01EB018EE1EEDFC80159DF49
:106DC000CE0157DFDF91CF911F910F9188CFCF92E6
:106DD000DF92EF92FF926B017C012EEA37E441E6ED
:106DE0005FE30E94C46181110EC088E491EEAAE3C2
:106DF000BFE380933C1490933D14A0933E14B09352
:106E00003F1460E0ABC026E636E646EA5FE3C70122
:106E1000B6010E94C46181110EC08FE195E8ABE616
:106E2000BFE380933C1490933D14A0933E14B09321
:106E30003F1461E093C023E333E343EF5FE3C70113
:106E4000B6010E94C46181110EC086EF98E2ACE9E0
:106E5000BFE380933C1490933D14A0933E14B093F1
:106E60003F1462E07BC020E030E040E250E4C70124
:106E7000B6010E94C46181110EC08CE59FE8A2ECAE
:106E8000BFE380933C1490933D14A0933E14B093C1
:106E90003F1463E063C020E030E040E850E4C70105
:106EA000B6010E94C46181110EC08EEA97E4A1E18F
:106EB000B0E480933C1490933D14A0933E14B0939F
:106EC0003F1464E04BC026E636E646E950E4C701CD
:106ED000B6010E94C46181110EC08AE097EDA3E261
:106EE000B0E480933C1490933D14A0933E14B0936F
:106EF0003F1465E033C023E333E343EB50E4C701C1
:106F0000B6010E94C46181110EC085E89BEEA1E428
:106F1000B0E480933C1490933D14A0933E14B0933E
:106F20003F1466E01BC02AE939E941E051E4C7019A
:106F3000B6010E94C46181110EC083E393E3ABE804
:106F4000B0E480933C1490933D14A0933E14B0930E
:106F50003F1467E003C081E090E007C06295660FD0
:106F6000607E70E081E090E021DFFF90EF90DF90A5
:106F7000CF9008954F925F926F927F928F929F92DF
:106F8000AF92BF92CF92DF92EF92FF926B017C01A2
:106F9000B42E9B01AC010E945966882319F06EE45F
:106FA0007FE027C026013701E89477F82FEF3FEF05
:106FB0004FE75FE7C301B2010E94596681110DC01E
:106FC0002FEF3FEF4FE75FE7C301B2010E94C461BB
:106FD00018161CF462E57FE00CC02FEF3FEF4FE77F
:106FE0005FE4C701B6010E94096518168CF466E5D6
:106FF0007FE086E892E1FF90EF90DF90CF90BF9026
:10700000AF909F908F907F906F905F904F90BBC597
:107010002FEF3FEF4FE75FECC701B6010E94C4615D
:1070200087FDE5CF20E030E0A901C701B6010E944D
:10703000C46187FF0AC06DE286E892E18FD54C01FA
:10704000F7FAF094F7F8F09402C0812C912CA12C5F
:1070500060E070E080E09FE3AB1441F020E030E0BE
:1070600040E251E40E941A64A394F6CF9B01AC0164
:10707000C701B6010E9454632B013C010E94B86411
:107080006B017C010E94C8619B01AC01C301B2018C
:107090000E9453632B013C012AE0B701A60186E858
:1070A00092E186D57C01E80CF91CBB2031F06EE240
:1070B00086E892E153D5E80EF91EDB2CDD2029F19C
:1070C00020E030E040E251E4C301B2010E942962B5
:1070D0002B013C010E94B8644B01A12CB12C2AE089
:1070E000B501A40186E892E163D5E80EF91EC50159
:1070F000B4010E94C8619B01AC01C301B2010E94AE
:1071000053632B013C01DA94D9CFC701FF90EF9074
:10711000DF90CF90BF90AF909F908F907F906F90B7
:107120005F904F9008951092671010926610109221
:1071300090101092B11010928E1081E080938D10FB
:107140001092681061E084E1FCD661E085E1F9D637
:10715000E9EBF0E080818E7F808380818D7F80836A
:1071600088E48093B80085E48093BC000895CF93B1
:10717000DF93CDB7DEB728970FB6F894DEBF0FBE0A
:10718000CDBF1D8290E49E8324E12F8324E52887D0
:1071900019829A8390E19B8390E59C839091E514FA
:1071A000691710F06FEF690F4091E614262F30E059
:1071B000FE01E20FF31F403121F4943011F491816C
:1071C00001C09581682F690F60688EED94E1289663
:1071D0000FB6F894DEBF0FBECDBFDF91CF910C94F8
:1071E000AF4190918E109111FCCF91E090938E1051
:1071F00090938D102FEF20938C1010928B10260FF0
:1072000020938A109093691090916910880F892BB0
:107210008093691080916810813061F41092681039
:10722000809169108093BB008091BC0083FDF8CFF2
:1072300085EC01C085EE8093BC0080918E1081307A
:10724000E1F380918B10861710F460918B10AAE601
:10725000B0E126E430E1F9018E2F821B861718F485
:107260008D918193F9CF862F0895613208F060E205
:10727000B8DF109267108093661008950F931F93E4
:10728000CF93DF931F92CDB7DEB7682F87E769836F
:1072900083DD698183E293E10E94C72B20DD87E7CC
:1072A0007BDD62E070E087E790E0DFDF83E293E17F
:1072B0000E94772B00E010E0182F83E293E10E94F8
:1072C000772B082B192B0BDDC8010F90DF91CF9185
:1072D0001F910F91089587E75FDD64EF83E293E1EB
:1072E0000E94C72B6EE283E293E10E94C72BF7DC7A
:1072F00065E070E080E090E0DCD686EFBFCFCF9213
:10730000DF92EF92FF920F931F93E5DFAC0160E0F5
:1073100070E0E5E2F4E1858996899A01AB01281BCA
:10732000390B41095109A389B4890E9412636B0189
:107330007C018FE0F594E794D794C7948A95D1F7B0
:1073400065857685CB01770FAA0BBB0BBC01CD0100
:107350002BE0660F771F881F991F2A95D1F7278585
:1073600030898901330F220B330BA90198012C0DB1
:107370003D1D4E1D5F1D0E94F662D701C601820FA2
:10738000931FA41FB51F0896A11DB11DBC01CD01FF
:1073900034E095958795779567953A95D1F70E9452
:1073A000CA6120E030E040E251E40E941A641F917B
:1073B0000F91FF90EF90DF90CF9008951F93CF93A0
:1073C000DF931F92CDB7DEB7682F87E76983E4DCD0
:1073D000698183E293E10E94C72B81DC87E7DCDCD3
:1073E00061E070E087E790E040DF83E293E10E9494
:1073F000772B182F74DC812F0F90DF91CF911F9185
:1074000008950895CF92DF92EF92FF920F931F930A
:10741000CF93DF936C017A018B01C0E0D0E0CE15F1
:10742000DF0589F0D8016D918D01D601ED91FC91B8
:107430000190F081E02DC6011995892B11F47E0190
:1074400002C02196ECCFC701DF91CF911F910F9120
:10745000FF90EF90DF90CF900895FC01A089B18953
:107460008C91A689B78982FD0FC09C91818D8F5F19
:107470008F73228D821749F0218DDF01A20FB11D7C
:107480005D969C93818F08958C910895FC01538D96
:10749000448D252F30E0842F90E0821B930B5417EE
:1074A00010F0CF96089501970895FC01918D828D7B
:1074B000981761F0828DDF01A80FB11D5D968C9148
:1074C000928D9F5F9F73928F90E008958FEF9FEF53
:1074D0000895FC01918D828D981731F0828DE80F0F
:1074E000F11D858D90E008958FEF9FEF0895FC01C9
:1074F000918D228D892F90E0805C9F4F821B910996
:107500008F73992708958CE491E1F1DF21E0892BB5
:1075100009F420E0822F089589EE91E1E8DF21E06F
:10752000892B09F420E0822F089586E892E1DFDFBD
:1075300021E0892B09F420E0822F0895FC01848D3D
:10754000DF01A80FB11DA35ABF4F2C91848D90E08D
:1075500001968F739927848FA689B7892C93A08968
:10756000B1898C9180648C93938D848D981306C01F
:107570000288F389E02D80818F7D80830895EF92CA
:10758000FF920F931F93CF93DF93EC0181E0888FDD
:107590009B8D8C8D981305C0E889F989808185FDC4
:1075A00023C0F62E0B8D10E00F5F1F4F0F731127B6
:1075B000E02E8C8DE8120BC00FB607FCFACFE889DD
:1075C000F989808185FFF5CFCE01B8DFF2CF8B8DB1
:1075D000FE01E80FF11DE35AFF4FF0820B8FEA899D
:1075E000FB898081806207C0EE89FF896083E8891A
:1075F000F98980818064808381E090E0DF91CF9180
:107600001F910F91FF90EF900895CF93DF93EC01BE
:10761000888D8823C1F0EA89FB89808185FD05C0BA
:10762000A889B9898C9186FD0EC00FB607FCF5CFED
:10763000808185FFF2CFA889B9898C9185FFEDCF34
:10764000CE017CDFE8CFDF91CF91089580E090E01C
:10765000892B19F06ADF81111BC080E090E0892B33
:1076600041F080E090E0892B21F00E940000811120
:1076700012C080E090E0892B19F04EDF81110EC01E
:1076800080E090E0892B79F03EDF81110AC00895F7
:107690000E940000E2CF0E940000EBCF0E94000099
:1076A000EFCF0C940000089590E0FC013197E23197
:1076B000F10508F04EC08827EA57FF4F8F4F0C9412
:1076C0009466809180008F7703C0809180008F7DC9
:1076D00080938000089580918000877FF9CF84B5E2
:1076E0008F7702C084B58F7D84BD08958091B000EE
:1076F0008F7703C08091B0008F7D8093B000089594
:10770000809190008F7707C0809190008F7D03C09B
:1077100080919000877F8093900008958091A000D1
:107720008F7707C08091A0008F7D03C08091A0005B
:10773000877F8093A0000895809120018F7707C0F4
:10774000809120018F7D03C080912001877F8093ED
:10775000200108950E94F868CF93DF93EC0188819F
:107760009981009711F00E947C67198218821D820E
:107770001C821B821A82DF91CF9108950F931F9371
:10778000CF93DF93EC0188819981009729F02A81BA
:107790003B812617370788F48B016F5F7F4F0E946C
:1077A0001468009761F0998388831B830A832C8176
:1077B0003D81232B11F4FC01108281E001C080E0A7
:1077C000DF91CF911F910F910895EF92FF920F9348
:1077D0001F93CF93DF93EC017B018A01BA01CEDFC7
:1077E000811103C0CE01B8DF07C01D830C83B70130
:1077F000888199810E940569CE01DF91CF911F9107
:107800000F91FF90EF900895FC0180819181009786
:1078100011F00C941E5D60E070E0CB010895EF92D2
:10782000FF920F931F93CF93DF93FC012481358147
:107830006115710511F480E018C041155105A1F0E2
:107840007B01EC018A01020F131FB80197DF882327
:1078500091F3288139818C819D81B701820F931F1B
:107860000E9405691D830C8381E0DF91CF911F91F8
:107870000F91FF90EF900895CF93DF93EC01611586
:10788000710559F0FB0101900020E9F73197AF0134
:10789000461B570BC4DF811102C0CE015DDFCE0154
:1078A000DF91CF910895CF93DF93EC01FB014481E9
:1078B000558160817181B3DF811102C0CE014CDF3F
:1078C000CE01DF91CF9108956115710549F0FB015B
:1078D00001900020E9F73197AF01461B570B9FCF6E
:1078E00080E00895FB01448155816081718197CFCB
:1078F000CF93DF93EC016115710551F0FB0101900D
:107900000020E9F73197AF01461B570B5EDF01C03E
:1079100023DFCE01DF91CF910895CF93DF93EC0168
:10792000FB018617970751F0608171816115710520
:1079300021F04481558149DF01C00EDFCE01DF9186
:10794000CF9108950F931F93CF93DF938C01EB0199
:10795000FC01808191810097B1F068817981611586
:10796000710579F0428153812C813D814217530783
:1079700040F00E9405698C819D81F8019583848384
:1079800013C00E947C6788819981F801918380836C
:107990008A819B81938382838C819D81958384835B
:1079A000198218821B821A821D821C82DF91CF915C
:1079B0001F910F910895FC01808191810C947C6747
:1079C000EF92FF920F931F93CF93DF93CDB7DEB764
:1079D000A1970FB6F894DEBF0FBECDBF7C01CB01DF
:1079E000BA01F70111821082138212821582148269
:1079F00042E0420F8E010F5F1F4F0E94FC5CBC01F2
:107A0000C70176DFA1960FB6F894DEBF0FBECDBFDB
:107A1000DF91CF911F910F91FF90EF9008950F93F9
:107A20001F93CF93DF93CDB7DEB7A1970FB6F8942E
:107A3000DEBF0FBECDBF8C01CB01BA01F8011182B0
:107A40001082138212821582148230E0AE014F5FE1
:107A50005F4F0E94855DBE016F5F7F4FC80148DFA9
:107A6000A1960FB6F894DEBF0FBECDBFDF91CF91C8
:107A70001F910F9108950F931F93CF93DF93CDB76D
:107A8000DEB7A2970FB6F894DEBF0FBECDBF8C0154
:107A9000CB01BA01F8011182108213821282158281
:107AA000148230E0AE014F5F5F4F0E94585DBE010F
:107AB0006F5F7F4FC8011CDFA2960FB6F894DEBF40
:107AC0000FBECDBFDF91CF911F910F9108950F93FE
:107AD0001F93CF93DF93CDB7DEB762970FB6F894BD
:107AE000DEBF0FBECDBF8C01CB01F8011182108229
:107AF000138212821582148250E0BE016F5F7F4FA5
:107B00000E94445DBE016F5F7F4FC801F1DE629647
:107B10000FB6F894DEBF0FBECDBFDF91CF911F919E
:107B20000F910895FC011182108213821282158236
:107B30001482F3CEFC01118210821382128215820C
:107B400014826115710549F0FB0101900020E9F7ED
:107B50003197AF01461B570B38CE0895DC01ED91EC
:107B6000FC910190F081E02D1994DC01ED91FC91E4
:107B7000DB0114964D915C9115976D917C9102807B
:107B8000F381E02D19946115710579F0FB010190E5
:107B90000020E9F73197AF01461B570BDC01ED914F
:107BA000FC910280F381E02D199480E090E008952B
:107BB0004F925F926F927F92EF92FF920F931F937B
:107BC000CF93DF93CDB7DEB7A1970FB6F894DEBFA2
:107BD0000FBECDBF7C01FA01CB0119A2223008F4FF
:107BE0002AE08E010F5D1F4F422E512C612C712C0B
:107BF000BF01A30192010E942263F901CA01015051
:107C000011096A3014F4605D01C0695CD8016C939D
:107C1000232B242B252B61F7B801C701B4DFA196D4
:107C20000FB6F894DEBF0FBECDBFDF91CF911F918D
:107C30000F91FF90EF907F906F905F904F9008951D
:107C4000CF92DF92EF92FF920F931F93CF93DF9328
:107C5000EC016A017B012115310579F4E881F98194
:107C60000190F081E02D642FDF91CF911F910F9152
:107C7000FF90EF90DF90CF9019942A303105D9F41E
:107C800077FF18C06DE26ADF8C0144275527BA01DF
:107C90004C195D096E097F092AE0CE0189DF800F4A
:107CA000911FDF91CF911F910F91FF90EF90DF9087
:107CB000CF9008952AE0B701A601CE01DF91CF91C0
:107CC0001F910F91FF90EF90DF90CF9071CF9A01AD
:107CD000AB01770F660B770BB3CF6AE57FE053CF2D
:107CE0000F931F93CF93DF93EC013FDF8C01CE0105
:107CF000F4DF800F911FDF91CF911F910F910895B5
:107D000042CF1F920F920FB60F9211240BB60F9213
:107D10002F933F934F935F936F937F938F939F9393
:107D2000AF93BF93EF93FF938CE491E107DCFF9156
:107D3000EF91BF91AF919F918F917F916F915F91E3
:107D40004F913F912F910F900BBE0F900FBE0F9050
:107D50001F9018951F920F920FB60F9211240BB619
:107D60000F922F933F934F935F936F937F938F93D4
:107D70009F93AF93BF93EF93FF938CE491E16DDBFF
:107D8000FF91EF91BF91AF919F918F917F916F91F3
:107D90005F914F913F912F910F900BBE0F900FBEAF
:107DA0000F901F9018951F920F920FB60F921124EB
:107DB0000BB60F922F933F934F935F936F937F93E5
:107DC0008F939F93AF93BF93EF93FF9389EE91E1CE
:107DD000B5DBFF91EF91BF91AF919F918F917F9113
:107DE0006F915F914F913F912F910F900BBE0F902C
:107DF0000FBE0F901F9018951F920F920FB60F9203
:107E000011240BB60F922F933F934F935F936F9371
:107E10007F938F939F93AF93BF93EF93FF9389EEDD
:107E200091E11BDBFF91EF91BF91AF919F918F91FA
:107E30007F916F915F914F913F912F910F900BBE6A
:107E40000F900FBE0F901F9018951F920F920FB6B4
:107E50000F9211240BB60F922F933F934F935F9382
:107E60006F937F938F939F93AF93BF93EF93FF9302
:107E700086E892E163DBFF91EF91BF91AF919F9113
:107E80008F917F916F915F914F913F912F910F90C3
:107E90000BBE0F900FBE0F901F9018951F920F9260
:107EA0000FB60F9211240BB60F922F933F934F935F
:107EB0005F936F937F938F939F93AF93BF93EF9352
:107EC000FF9386E892E1C9DAFF91EF91BF91AF91FC
:107ED0009F918F917F916F915F914F913F912F91E2
:107EE0000F900BBE0F900FBE0F901F901895CF9361
:107EF000DF93282F30E0F901E151FC4F8491F90123
:107F0000E755FC4FD491F901ED59FC4FC491CC23B6
:107F100089F08111C9DBEC2FF0E0EE0FFF1FE75B6A
:107F2000FC4FA591B491EC91ED2381E090E021F418
:107F300080E002C080E090E0DF91CF910895862F2D
:107F4000D6CF1F93CF93DF93282F30E0F901E15173
:107F5000FC4F8491F901E755FC4FD491F901ED599B
:107F6000FC4FC491CC23C1F0162F81119DDBEC2F67
:107F7000F0E0EE0FFF1FE15DFC4FA591B4918FB7CC
:107F8000F894111105C09C91ED2FE095E92302C0F2
:107F9000EC91ED2BEC938FBFDF91CF911F91089562
:107FA000862F642FCECFCF93DF9390E0FC01E7556F
:107FB000FC4F2491FC01ED59FC4F8491882361F121
:107FC00090E0880F991FFC01EB5EFC4FC591D491A6
:107FD000FC01E15DFC4FA591B491611109C09FB70F
:107FE000F8948881209582238883EC912E230BC0FE
:107FF000623061F49FB7F8943881822F8095832393
:108000008883EC912E2B2C939FBF06C08FB7F894DA
:10801000E8812E2B28838FBFDF91CF91089586337F
:1080200008F0865390917B00282F2870977F922B21
:1080300090937B0087702091A50390E4299F900185
:108040001124822B80937C0080917A00806480933D
:108050007A0080917A0086FDFCCF80917800209193
:10806000790090E0922B08953FB7F8948091FD1429
:108070009091FE14A091FF14B091001526B5A89B15
:1080800005C02F3F19F00196A11DB11D3FBFBA2FAA
:10809000A92F982F8827820F911DA11DB11DBC010A
:1080A000CD0142E0660F771F881F991F4A95D1F7CF
:1080B00008958F929F92AF92BF92CF92DF92EF92EC
:1080C000FF926B017C01D0DF4B015C01C114D10434
:1080D000E104F104E9F0C8DFDC01CB01881999095A
:1080E000AA09BB09883E9340A105B10578F321E0B8
:1080F000C21AD108E108F10888EE880E83E0981EC4
:10810000A11CB11CC114D104E104F10421F7DECF9C
:10811000FF90EF90DF90CF90BF90AF909F908F90A7
:1081200008952FB7F8946091F9147091FA14809122
:10813000FB149091FC142FBF08951F920F920FB65D
:108140000F9211242F933F938F939F93AF93BF93DD
:108150008091F9149091FA14A091FB14B091FC1441
:108160003091F81423E0230F2D3720F40196A11D40
:10817000B11D05C026E8230F0296A11DB11D209355
:10818000F8148093F9149093FA14A093FB14B0930D
:10819000FC148091FD149091FE14A091FF14B091F5
:1081A00000150196A11DB11D8093FD149093FE143E
:1081B000A093FF14B0930015BF91AF919F918F9141
:1081C0003F912F910F900FBE0F901F90189521E0B7
:1081D00001C0220F6A95EAF7DC011C962C931C97CC
:1081E0001A965C934E931997ED91FC910484F58552
:1081F000E02D60E01994DC01ED91FC910684F78597
:10820000E02D41E0199581E090E0089508950895EA
:1082100085ED8093BC008091BC0084FDFCCF109262
:108220008E1008950895E091671080916610E81708
:1082300030F4F0E0EA5BFF4E808190E008958FEF2C
:108240009FEF0895862F642FAECECF93DF93FC016E
:108250002381222391F0EC01818180956823608342
:1082600082810E94CC36688183E293E10E94C72B11
:108270000E946F36282F30E002C020E030E081E01D
:1082800090E0232B11F080E090E0DF91CF910895F2
:10829000EF92FF920F931F93CF938C01FC01759681
:1082A00084E0C0E060FF02C09081C92B66958150D8
:1082B00031968111F7CF413011F4F8014489F8016A
:1082C0008585C82BC42B7801FEE0EF0EF11CF80168
:1082D00062896C2BC701B9DFF801628960956C2354
:1082E000C701CF911F910F91FF90EF90AECF0F93E9
:1082F0001F93CF93DF93062F0F70423019F440E0A5
:10830000602F0FC0142F262FEC0130E0B90184E05C
:10831000759567958A95E1F7CE01BADF412F602FF9
:10832000CE01DF91CF911F910F91B2CFFC018485D7
:108330008823A1F0218532852115310519F46111B9
:1083400006C007C02130310521F4611102C08587C4
:1083500001C015866585CF010E9677CF0895DC01A3
:10836000ED91FC910684F785E02D40E01994FC0125
:108370006581262F246025836C60F1CF0F931F93B6
:10838000CF93DF93EC01423018F08C8188608C83AE
:108390004F836887222329F0413019F48C8184604F
:1083A0008C8364E670E080E090E083DE6C8164FDA5
:1083B00031C0E881F9810684F785E02D42E063E071
:1083C000CE0119950BE416E4C8010197F1F7E88195
:1083D000F9810684F785E02D42E063E0CE0119952E
:1083E000C8010197F1F7E881F9810684F785E02D4E
:1083F00042E063E0CE01199583E592E00197F1F741
:10840000E881F9810684F785E02D42E062E0CE0143
:10841000199513C06062CE01A2DF8BE496E4019748
:10842000F1F76C816062CE019ADF83E592E00197FB
:10843000F1F76C816062CE0192DF6C816062CE01E7
:108440008EDF84E08D83CE0192DF61E0CE0187DF95
:108450008BE39FE10197F1F782E08E8366E0CE0126
:108460007EDFE881F9810484F585E02D6FEFCE0190
:10847000DF91CF911F910F911994FF920F931F934A
:10848000CF93DF93EC01162F042FF22E8B85888B70
:108490000E94933861E088890E94F1381092671039
:1084A0008093661091E0811101C090E0998B83E286
:1084B00093E10E94772B8E878989882331F01F866C
:1084C0001C8260E0CE010E96C0DE2F2D402F612F62
:1084D000CE01DF91CF911F910F91FF904FCF1F924F
:1084E0000F920FB60F9211240F900FBE0F901F9096
:1084F00018951F920F920FB60F9211240BB60F9280
:108500002F933F934F935F936F937F938F939F939B
:10851000AF93BF93EF93FF9380913013E8DC2091EA
:108520003313309134132F5F3F4F30933413209324
:10853000331390913213953618F096E090932F13E1
:1085400090912F139430C9F128F4923069F0933050
:10855000D1F05EC0953009F451C0963009F058C092
:1085600091E09093FF1351C0811152C020913313B9
:10857000309134132436310508F442C01092FF13B1
:10858000109232131CC0813009F042C0E0913213C6
:1085900091E09E0F90933213F0E0209133133091CD
:1085A0003413EE0FFF1FEB5CFC4E318320831092DF
:1085B00034131092331394E029C0811117C0E09155
:1085C000321391E09E0F90933213F0E02091331319
:1085D00030913413EE0FFF1FEB5CFC4E3183208390
:1085E000109234131092331393E010C02091331380
:1085F000309134132536310558F007C0811108C079
:10860000109234131092331303C095E090932F13FC
:1086100090913113992329F0811102C02F9A01C042
:108620002F98FF91EF91BF91AF919F918F917F9183
:108630006F915F914F913F912F910F900BBE0F90D3
:108640000FBE0F901F901895CF92DF92EF92FF927E
:10865000CF93DF93EC01072E000C880B990B0E943F
:10866000CA616B017C0120E030E040E45FE30E94DE
:10867000296220E030E048E452E40E941A640E943B
:10868000B364C617D707D4F020E030E040EA5FE3D8
:10869000C701B6010E94296220E030E048E452E4BC
:1086A0000E941A6420E030E040E85FE30E945463D7
:1086B0000E94B36421E06C177D070CF420E0822F48
:1086C00090E0DF91CF91FF90EF90DF90CF900895F1
:1086D0000F931F93CF93DF93082F66E374E086E830
:1086E00092E10EDBC7E0D0E010E0B8010C2E02C032
:1086F000759567950A94E2F76170772742E050E03C
:1087000086E892E1E4DA219780F7DF91CF911F911B
:108710000F9108951F920F920FB60F9211240BB66E
:108720000F922F933F934F935F936F937F938F930A
:108730009F93AF93BF93EF93FF938091B900887F8E
:10874000803609F49CC068F5883209F45BC090F467
:10875000803109F454C038F4882309F4F6C0883015
:1087600009F44DC0F5C0883109F44CC0803209F4D9
:108770005DC0EEC0803409F468C048F4803309F469
:1087800055C0883309F0E4C080938C10D8C0803580
:1087900009F44FC0883509F45DC0883409F0D8C0A9
:1087A000D6C0883909F4C7C0A8F4883709F467C06F
:1087B00038F4883609F463C0803709F460C0C8C053
:1087C000883809F4B8C0803909F45FC0803809F0EE
:1087D000BFC05BC0803B09F486C038F4803A09F41E
:1087E00066C0883A09F47FC0B3C0803C09F4A7C0D2
:1087F000883C09F4A4C0883B09F48AC0A9C08091D0
:10880000691010C090918B1080918A10981770F5A4
:10881000E0918B1081E08E0F80938B10F0E0E65991
:10882000FF4E80818093BB0085EC86C080938C10C6
:108830008EC0E0918B1081E08E0F80938B10809121
:10884000BB00F0E0E659FF4E808390918B10809141
:108850008A106EC0E0918B1081E08E0F80938B1098
:108860008091BB00F0E0E659FF4E808380918D102F
:1088700081116DC081E08093681084EA61C083E05B
:1088800080938E1010924715CFCF8091471580327C
:1088900008F051C0E091471581E08E0F8093471595
:1088A0008091BB00F0E0E95DFA4E8083BDCF85EC9E
:1088B0008093BC0010928E1080914715803230F466
:1088C000E0914715F0E0E95DFA4E1082609147159E
:1088D00070E0E0912515F091261587E295E1199554
:1088E0001092471535C084E080938E1010922415A5
:1088F00010922315E0912115F09122151995809180
:108900002315811105C081E0809323151092011574
:10891000E091241581E08E0F80932415F0E0EF5F45
:10892000FA4E80818093BB0090912415809123158D
:10893000981708F479CF85E88093BC0009C085ECCE
:108940008093BC0010928E1003C010928C1060DCDB
:10895000FF91EF91BF91AF919F918F917F916F9117
:108960005F914F913F912F910F900BBE0F900FBED3
:108970000F901F90189540912315262F30E0240F5B
:10898000311D21323105DCF420918E102430C9F4E0
:10899000FC0180E090E0861758F430912315219176
:1089A000DC01AF5FBA4EA30FB11D2C930196F3CF3C
:1089B00080912315680F6093231580E0089581E06E
:1089C000089582E0089596E0899FD0011124AA5964
:1089D000BB4E90967C936E935F9791E091969C939B
:1089E00091979091D214E091D314F091D4149923DB
:1089F00039F0309751F0811108C08091821404C081
:108A0000309719F05C968C91199408953F924F928B
:108A10005F926F927F928F929F92AF92BF92CF920E
:108A2000DF92EF92FF920F931F93CF93DF93CDB717
:108A3000DEB728970FB6F894DEBF0FBECDBF0E94F9
:108A40006B396C01E12CF12C109125141295110F4A
:108A5000110F107C1C5C87E70E94CC3664EF83E228
:108A600093E10E94C72B612F83E293E10E94C72B01
:108A70000E946F3680912514811105C065E070E079
:108A800080E090E012C0813029F468E070E080E07E
:108A900090E00BC0823029F46EE070E080E090E05E
:108AA00004C06AE170E080E090E003DB86EF0E94A2
:108AB0003E394C01A12CB12CBA2CA92C982C88241D
:108AC00088EF0E94DE39882A3090251480913A146C
:108AD00090913B14A7019601281B390B41095109BC
:108AE000A0913814B09139140E9412636B017C017B
:108AF000AFE0F594E794D794C794AA95D1F7609125
:108B0000321470913314CB01770FAA0BBB0BBC014D
:108B1000CD01BBE0660F771F881F991FBA95D1F76B
:108B200020913414309135148901330F220B330B0B
:108B3000A90198012C0D3D1D4E1D5F1D0E94F6627E
:108B4000C20ED31EE41EF51E20EAC21A2FE0D20A7E
:108B5000E108F108A7019601C701B6010E947266FB
:108B60009B01AC011CE055954795379527951A95C3
:108B7000D1F729833A834B835C83009126141091AB
:108B80002714A0912A14B0912B14A70196010E94DA
:108B90001C632B013C018DE07594679457944794B6
:108BA0008A95D1F7A0912C14B0912D1429813A8186
:108BB0004B815C810E941C63BB2797FDB095AB2F56
:108BC000840D951DA61DB71D0296A11DB11D32E095
:108BD000B595A795979587953A95D1F79C01AD01E5
:108BE00030584F4F5F4FA0913614B09137140E9408
:108BF00012632B013C014FE076946794579447949D
:108C00004A95D1F788E090E083199109A501940174
:108C100004C056954795379527958A95D2F72D83A9
:108C20003E834F8358874801110FAA08BB0852E0C2
:108C3000880C991CAA1CBB1C5A95D1F7A0912E1424
:108C4000B0912F1429813A814B815C810E941C6371
:108C50009B01AC016BE055954795379527956A9533
:108C6000D1F729833A834B835C83A0912814B09178
:108C70002914A70196010E941C63DC01CB017BE053
:108C8000B595A795979587957A95D1F729813A81DA
:108C90004B815C81820F931FA41FB51F880D991D06
:108CA000AA1DBB1D032C04C0880F991FAA1FBB1F40
:108CB0000A94D2F7BC01CD016E5F7F4F8F4F9F4F5B
:108CC00024E030E040E050E00E94F6628D819E8119
:108CD000AF81B885821B930BA40BB50B9C01AD0132
:108CE00080E593ECA0E0B0E0BC01CD0104C0969516
:108CF0008795779567953A94D2F70E94726697FDAB
:108D00000BC0660F771F881F991FA30192010E9455
:108D1000226369017A010AC0A30192010E942263C1
:108D200069017A01CC0CDD1CEE1CFF1C9927F7FCB5
:108D30009A958F2D7E2D6D2D9B01AC010E94726640
:108D40009B01AC01AEEDBBE00E9412634C01BB2461
:108D500097FCB094AB2CA3E4B3EEA70196010E945C
:108D60001E63BB2797FDB095AB2F880D991DAA1DDB
:108D7000BB1D8153914FAF4FBF4F44E0B595A795B1
:108D8000979587954A95D1F7BC01CD016C0D7D1D56
:108D90008E1D9F1D28960FB6F894DEBF0FBECDBF67
:108DA000DF91CF911F910F91FF90EF90DF90CF90C7
:108DB000BF90AF909F908F907F906F905F904F90FB
:108DC0003F9008951F93CF93DF93CDB7DEB72C97D5
:108DD0000FB6F894DEBF0FBECDBF8EE10E94CC3639
:108DE00083E090E00E9439360E946F368EE10E9447
:108DF000CC3666E070E08EE190E00E9435398091DB
:108E0000661090E020916710821B9109069741F44B
:108E100010E083E293E10E94772B1F5F1630C9F7C1
:108E20000E946F366B8170E0762F66278C81682BED
:108E30004D8150E0542F44278E81482B298130E00A
:108E4000322F22278A81282B38872F835A874987F8
:108E50007C876B8738855A857C8580E090E02C96EE
:108E60000FB6F894DEBF0FBECDBFDF91CF911F913B
:108E70000895EF92FF920F931F93CF93DF93C82F24
:108E80008B017A0183E50E94CC366C2F83E293E15B
:108E90000E94C72B0E946F3683E50E94CC36B80132
:108EA00083E590E00E943539E701CE018E199F09D4
:108EB0003091661020916710321731F083E293E110
:108EC0000E94772B8993F1CF8017910729F0109298
:108ED000521481E080935314DF91CF911F910F9131
:108EE000FF90EF900C946F36CF93DF93AC01990F06
:108EF000660B770B2AE030E086E892E10E94203E84
:108F0000EC0186E892E10E946D3E8C0F9D1FDF917F
:108F1000CF9108951F93CF93DF931F92CDB7DEB704
:108F2000162FAE014F5F5F4F61E070E0A2DF8981D5
:108F300090E002C0959587951A95E2F781700F90A1
:108F4000DF91CF911F910895CF93DF93D82FC62F34
:108F500083E50E94CC366D2F83E293E10E94C72BFC
:108F60006C2F83E293E10E94C72BDF91CF910C9489
:108F70006F36FF920F931F93CF93DF931F92CDB75E
:108F8000DEB7182F062FF42EAE014F5F5F4F61E062
:108F900070E06FDF8981FF2049F041E050E001C0BF
:108FA000440F0A95EAF7482B498309C021E030E0D5
:108FB00001C0220F0A95EAF72095282329836981A9
:108FC000812FC2DF0F90DF91CF911F910F91FF9002
:108FD0000895CF93DF9342E00E94BA37EC0186E810
:108FE00092E10E946D3E8C0F9D1FDF91CF910895FD
:108FF000AF92BF92CF92DF92EF92FF921F93CF93E7
:10900000DF93CDB7DEB72A970FB6F894DEBF0FBE59
:10901000CDBF182F40E654E166E070E082E39F8305
:1090200028DF2091611430E0322F222780916014D4
:10903000282B3A8329832091631430E0322F222792
:1090400080916214282B3C832B832091651430E09F
:10905000322F222780916414282B3E832D839E017A
:109060002F5F3F4F590154E5C52E54E1D52EE12E17
:109070009F81F92EF501619171915F01F6012191B6
:109080003191419151916F01072E000C880B990B82
:109090002F83388749875A870E94CA612F81388574
:1090A00049855A850E942962F701619371938193E2
:1090B00091937F01F0E6CF16F4E1DF06D9F62A9608
:1090C0000FB6F894DEBF0FBECDBFDF91CF911F91D9
:1090D000FF90EF90DF90CF90BF90AF9008953F92B8
:1090E0004F925F926F927F928F929F92AF92BF92B8
:1090F000CF92DF92EF92FF920F931F93CF93DF9364
:1091000000D01F921F92CDB7DEB7982E0AD82B0140
:109110003C0120ED420E27E0521E611C711C60E0F4
:109120008091D5140E94A13F35E0832ECE01019697
:109130006C01AA24A394B12C55E0352E380EF6010B
:10914000282D11922A95E9F7860127E0E22EF12CCD
:109150008091D6140E94773F019739F40E94914084
:10916000641575058605970598F38091D6140E94BD
:10917000773F892B39F40E94914064157505860567
:10918000970598F38091D7140E94773F892B51F06F
:10919000F8012081C5010E2C01C0880F0A94EAF75E
:1091A000822B8083F1E0EF1AF10890F60F5F1F4FDA
:1091B0003012CBCF0E949140641575058605970546
:1091C00050F061E08091D5140E94A13F60E070E012
:1091D00080EC9FE72CC089818911B1CF9B818A8166
:1091E000980F990D8C818913AACF8D818D3009F04C
:1091F000A6CF61E08091D5140E94A13F6A818B8146
:1092000070E0762F6627680F711D072E000C880B03
:10921000990B0E94CA6120E030E040E85DE30E94C3
:10922000296223E333E948E853E40E9453630F9033
:109230000F900F900F900F90DF91CF911F910F9192
:10924000FF90EF90DF90CF90BF90AF909F908F9066
:109250007F906F905F904F903F90089589EE91E1DD
:109260000E94053BE9EEF1E1A289B3898C918F7EE2
:109270008C93A289B3898C91877F8C93A289B389BF
:109280008C918F778C93A289B3898C918F7D8C93ED
:10929000828D818F08954F925F926F927F928F920D
:1092A0009F92AF92BF92CF92DF92EF92FF92CF93B5
:1092B000DF93CDB7DEB764970FB6F894DEBF0FBE6D
:1092C000CDBF0E94382C698B7A8B8B8B9C8B8090C6
:1092D000AE039090AF03A090B003B090B103A5018E
:1092E00094016091B2037091B3038091B4039091A3
:1092F000B5030E9453632B013C0120E030E0A9013B
:109300000E94C461882309F451C0C090AA03D09080
:10931000AB03E090AC03F090AD0320E030E0A90196
:10932000C701B6010E94C46118160CF03FC08091BD
:10933000A6039091A703A091A803B091A9038D87DC
:109340009E87AF87B88B9C01AD01C701B6010E9413
:10935000C461882359F1A70196016D857E858F85AB
:1093600098890E941A640E9455656D877E878F8751
:10937000988BA501940169897A898B899C890E94BF
:109380005363A30192010E941A642D853E854F8587
:1093900058890E9429620E9487649B01AC01C70121
:1093A000B6010E9429626B017C0103C0C12CD12C43
:1093B000760160E080E00E94B7380E94914028EE7C
:1093C00033E040E050E00E942263BA01A9012AE0A4
:1093D000CE0101960E940F3DBE016F5F7F4F87E077
:1093E00094E10E94A23CCE0101960E94DB3C67E022
:1093F00074E1CE0101960E94923D6DE57FE0CE01C1
:1094000001960E943C3CBC0187E094E10E948D3CA7
:10941000CE0101960E94DB3CD7D060E080E00E9444
:10942000B73867E074E18EED94E10E94B53D21E02C
:10943000B701A601CE0101960E94E03C69E67FE0FB
:10944000CE0107960E949A3DBE016F5F7F4FCE010D
:1094500007960E94533C6DE67FE00E943C3CBC01B5
:109460008DE094E10E948D3CCE0107960E94DB3C8A
:10947000CE0101960E94DB3C61E080E00E94B7389B
:109480006DE074E18EED94E10E94B53D64E670E01C
:1094900080E090E00E94594080914A15882331F085
:1094A00060E273E080E090E00E94594064960FB65D
:1094B000F894DEBF0FBECDBFDF91CF91FF90EF904C
:1094C000DF90CF90BF90AF909F908F907F906F90E4
:1094D0005F904F900895FC01448155818091231441
:1094E000909124148417950780F080911F14909117
:1094F0002014009751F0608171816115710529F088
:109500000E940C6921E0892B09F020E0822F089548
:109510000F931F93CF93DF93C82FD62F86E0C89F5A
:10952000F0011124EA59FB4E11A2878D90A18130E0
:109530009105E9F01CF4892B49F041C08230910576
:10954000A1F10397E1F560E070E033C06623B9F163
:1095500061E070E08C2F37DA0E9491406093BE1476
:109560007093BF148093C0149093C11428C00E94BC
:1095700091400091BE141091BF142091C0143091FD
:10958000C114AB01BC01401B510B620B730B8091EA
:10959000D0149091D114A0E0B0E084179507A607ED
:1095A000B70718F462E070E004C0D11108C063E0AE
:1095B00070E08C2FDF91CF911F910F9104CADF9142
:1095C000CF911F910F91089561E08EED94E10E947B
:1095D000AF418BE39FE10197F1F70895EF92FF927E
:1095E0000F931F93CF938C01C62F7A0180E00E94C6
:1095F000B73861E77FE08EED94E10E94803E6C2FEA
:1096000080E00E94B738B8018EED94E10E94B53D2C
:10961000B701FF0C880B990BCF911F910F91FF9011
:10962000EF900C9459408F929F92AF92BF92CF923D
:10963000DF92EF92FF920F931F93CF93DF93CDB7FB
:10964000DEB728970FB6F894DEBF0FBECDBF7C0102
:109650004A015B01690119821A821B821C821D82E8
:109660001E821F821886CB01BA010E94B3649B013F
:1096700077FF04C022273327261B370BB901330F8E
:10968000880B990B0E94CA610E9455652EE83DE542
:1096900043E150E40E941A640E94B3648B010F5F9F
:1096A0001F4F1016110614F001E010E00F5F1F4F5E
:1096B000A8014C0D5D1D4930510514F048E050E003
:1096C0008E010F5F1F4F2C2DC501B4010E94FC5C61
:1096D000BC01C7010E949A3DC70128960FB6F894B5
:1096E000DEBF0FBECDBFDF91CF911F910F91FF90D5
:1096F000EF90DF90CF90BF90AF909F908F900895A4
:109700004F925F926F927F928F929F92AF92BF9291
:10971000CF92DF92EF92FF920F931F93CF93DF933D
:10972000CDB7DEB76E970FB6F894DEBF0FBECDBFD4
:109730008C016CE57FE0CE010D960E949A3D42DBE4
:1097400062E370E080E090E00E9459403BDB2983B7
:109750003A834B835C836D837E83C0903C14D090AE
:109760003D14E0903E14F0903F1469817A81072EF9
:10977000000C880B990B0E94CA61A70196010E94F8
:1097800029624B015C016D817E81072E000C880BE4
:10979000990B0E94CA61A70196010E9429622B01C0
:1097A0003C016B817C81072E000C880B990B0E9479
:1097B000CA61A70196010E94296280925715909272
:1097C0005815A0925915B0925A1560935B15709375
:1097D0005C1580935D1590935E1540925F155092D5
:1097E00060156092611570926215980121503109DF
:1097F0002330310508F07CC1A50194010E94C763A4
:109800002091430330914403409145035091460316
:109810000E9454636B017C0120E030E0A9010E94AA
:10982000C46187FD09C0C0925315D0925415E092CF
:109830005515F092561510C02BED3FE049EC50E461
:10984000C701B6010E945463609353157093541579
:109850008093551590935615C0905315D09054157C
:10986000E0905515F09056152BED3FE049EC50E493
:10987000C701B6010E940965181684F42BED3FE07C
:1098800049EC50E4C701B6010E945363609353153D
:1098900070935415809355159093561520E030E041
:1098A00044E353E46091531570915415809155151C
:1098B000909156150E9429622BED3FE049E450E457
:1098C0000E941A6460934F15709350158093511540
:1098D000909352150E94B3644AE0CE0143960E94D1
:1098E000673D62E87FE0CE0101960E949A3DBE018D
:1098F0006D5E7F4FCE0101960E94533C6CE87FE085
:109900000E943C3CBC0183E194E10E948D3CCE016D
:1099100001960E94DB3CCE0143960E94DB3CC09046
:109920004F15D0905015E0905115F090521520E051
:1099300030E044EB52E4C701B6010E94C46118163E
:1099400064F0C701B6010E94B3644AE0CE014396B9
:109950000E94673D63E97FE023C020E030E044E3FC
:1099600053E4C701B6010E94C46118163CF1A70177
:10997000960160E070E084E393E40E945363609397
:109980004F157093501580935115909352150E9466
:10999000B3644AE0CE0143960E94673D69E97FE0E7
:1099A000CE0101960E949A3DBE016D5E7F4FCE01B1
:1099B00001960E94533C66E97FE04AC020E030E017
:1099C00047E853E4C701B6010E94C4611816D4F0F9
:1099D00020E030E044E353E4C701B6010E94536342
:1099E00060934F15709350158093511590935215B5
:1099F0000E94B3644AE0CE0143960E94673D69E944
:109A00007FE019C0A701960160E070E084EB93E469
:109A10000E94536360934F157093501580935115B6
:109A2000909352150E94B3644AE0CE0143960E947F
:109A3000673D63E97FE0CE0101960E949A3DBE0139
:109A40006D5E7F4FCE0101960E94533C6CE97FE032
:109A50000E943C3CBC01CE010D960E948D3CCE0183
:109A600001960E94DB3CCE0143960E94DB3CACDDBC
:109A700060E080E00E94B7380E94914028EE33E019
:109A800040E050E00E94F662BA01A9012AE0CE014E
:109A900001960E943B3DBE016F5F7F4F87E094E1DE
:109AA0000E94A23CCE0101960E94DB3C69E175E078
:109AB00087E094E10E94643C67E074E1CE01019686
:109AC0000E94923DBE01635F7F4FCE0101960E94CE
:109AD000533CBC018EED94E10E94B53DCE01019650
:109AE0000E94DB3C64E170E080E090E00E9459401D
:109AF000C8010297029708F0A1C10E949140C0904E
:109B0000E60FD090E70FE090E80FF090E90F6C19A6
:109B10007D098E099F090E94C86120E030E04AE774
:109B200054E40E941A64AB01BC0122E0CE0101960C
:109B30000E94E03CBE016F5F7F4FCE0143960E94C2
:109B4000923D69E175E0CE0143960E943C3CBC0128
:109B500081E094E10E948D3CCE0143960E94DB3C63
:109B6000CE0101960E94DB3C61E074E1CE010196DA
:109B70000E94923D63E174E1CE0101960E94533C44
:109B8000BE01635F7F4F0E94533CBC01CE010D9626
:109B90000E948D3CCE0101960E94DB3C6FE97FE084
:109BA0008DE094E10E94783C4091571550915815F2
:109BB0006091591570915A1521E0CE0101960E94CD
:109BC000E03CBE016F5F7F4F8DE094E10E94723CEC
:109BD000CE0101960E94DB3C40915F1550916015CB
:109BE000609161157091621521E0CE0149960E9445
:109BF000E03C40915B1550915C1560915D15709152
:109C00005E1521E0CE0143960E94E03C60E87FE0D3
:109C1000CE0101960E949A3DBE016D5E7F4FCE013E
:109C200001960E94533C60E87FE00E943C3CBE01EC
:109C3000675E7F4F0E94533C6AEA7FE00E943C3C93
:109C4000BC018DE094E10E94723CCE0101960E941D
:109C5000DB3CCE0143960E94DB3CCE0149960E943C
:109C6000DB3C609157157091581580915915909172
:109C70005A1580905B1590905C15A0905D15B09082
:109C80005E15C0905F15D0906015E0906115F09062
:109C900062159B01AC010E9429622B013C01A501C8
:109CA0009401C501B4010E9429629B01AC01C3016A
:109CB000B2010E9454634B015C01A7019601C701E8
:109CC000B6010E9429629B01AC01C501B4010E944A
:109CD00054630E9418666B017C0160934B1570936E
:109CE0004C1580934D1590934E156EEA7FE08DE0F4
:109CF00094E10E94643C20E030E04AE754E4C7016C
:109D0000B6010E94C46187FF08C021E0B701A60127
:109D1000CE0101960E94E03C0BC0C701B6010E9433
:109D2000B364AB01BC012AE0CE0101960E943B3D29
:109D3000BE016F5F7F4FCE0143960E94923D6BEA5A
:109D40007FE0CE0143960E943C3CBC0183E194E15C
:109D50000E948D3CCE0143960E94DB3CCE010196D1
:109D60000E94DB3C20E030E64AE656E460914B1569
:109D700070914C1580914D1590914E150E94C461C3
:109D800087FF55C063E174E18DE094E10E94723C6D
:109D9000BE01635F7F4FCE0101960E94923D6BE54D
:109DA0007FE0CE0101960E943C3C6DE074E10E9490
:109DB000533CBC018DE094E10E948D3CCE010196A4
:109DC0000E94DB3C0330110571F46DE074E1CE01BB
:109DD00001960E94923DCE0101960E94022FCE0173
:109DE00001960E94DB3C61E080E00E94B73861E7A9
:109DF0007FE08EED94E10E94803E61E080E00E9471
:109E0000B73862EB7FE0CE0101960E949A3D63E194
:109E100074E1CE0101960E94533CBC018EED94E1A9
:109E20000E94B53DCE0101960E94DB3C07C0BE01F9
:109E3000635F7F4F8DE094E10E948D3C68E270E0AB
:109E400080E090E00E945940CE010D960E94DB3CDC
:109E50006E960FB6F894DEBF0FBECDBFDF91CF91E7
:109E60001F910F91FF90EF90DF90CF90BF90AF9038
:109E70009F908F907F906F905F904F9008956F921A
:109E80007F928F929F92AF92BF92CF92DF92EF928A
:109E9000FF920F931F93CF93DF9381E08093D214AF
:109EA0000E9491400091C2141091C3142091C414D7
:109EB0003091C514AB01BC01401B510B620B730BFD
:109EC0008091CE149091CF14A0E0B0E08417950754
:109ED000A607B70708F00AC1C0E08091CC14C817E4
:109EE00060F4E091C814F091C914EC0FF11D62E028
:109EF00080810E94D33FCF5FF0CF712C812C912CB9
:109F0000540183948091CD14781608F05FC0072D1A
:109F100010E0E091CA14F091CB14E00FF11F61E062
:109F200080810E94D33FE091CA14F091CB14E00FDE
:109F3000F11F60E080810E94A13FD501C401072C80
:109F400004C0880F991FAA1FBB1F0A94D2F76C0187
:109F50007C01E094F094612C8091CC146816F8F4A4
:109F6000C62DD0E0E091C814F091C914EC0FFD1F8C
:109F700080810E94773F2496CC0FDD1FCA59DB4EAB
:109F8000892B29F4888199818C299D2904C0888195
:109F900099818E219F21998388836394DDCFE091FD
:109FA000CA14F091CB14E00FF11F61E080810E9490
:109FB000A13F8091CA149091CB14FC01E00FF11FD6
:109FC00060E080810E94D33F73949CCFE2E8F4E18B
:109FD0008FEF9FEF23813481232B21F41082928312
:109FE00081831582369624E1EE3BF20799F710E063
:109FF00096E0F92E8091CC14181708F051C000E0BB
:10A00000C12FD0E0CC0FDD1FC259DB4E2091CD1403
:10A01000021708F043C068817981002E02C076954E
:10A0200067950A94E2F761707727129F90011124D7
:10A03000200F311DE091C614F091C714E20FF31FF9
:10A040004081E6E6F4E180E0A58DB68DA217B30766
:10A0500011F461701AC08F5F36968A30A9F7672BAA
:10A06000D9F0E2E8F4E180E090E0508151110FC0B6
:10A07000F89EF001F99EF00D1124EA59FB4E448F31
:10A08000368F258F10A2178E61E042DA05C0019647
:10A0900036968A30910549F70F5FB8CF1F5FAACF78
:10A0A00080E090E0C0E0FC01EA59FB4E21A12111C3
:10A0B000C1E006968C339105B1F70E949140609300
:10A0C000C2147093C3148093C4149093C514CC230A
:10A0D00069F080918714882349F0809185149091CC
:10A0E0008614019719F48091821403C01092D2143F
:10A0F00080E0DF91CF911F910F91FF90EF90DF9063
:10A10000CF90BF90AF909F908F907F906F90089569
:10A110008F929F92AF92BF92CF92DF92EF92FF9277
:10A120000F931F93CF93DF93DB01CD91DC91DC0183
:10A130001C96ED91FC911D97CE17DF070CF04AC0DD
:10A14000FE01EE0FFF1F1A968D919C911B97E80F51
:10A15000F91F80809180C170DD27B1E0CB27209767
:10A1600019F404E610E002C00CE91FEF79015A016E
:10A170006B01020F131FB801C4010E942443892BF5
:10A1800099F40E0D1F1DB801C4010E942443892BB0
:10A1900071F4B8016E0D7F1DC4010E942443892B08
:10A1A000E1F023E030E005C021E030E002C022E031
:10A1B00030E0F5018081918101968217930734F098
:10A1C00011821082F60180819181019691838083B2
:10A1D000CE0105C081E090E002C08FEF9FEFDF91DC
:10A1E000CF911F910F91FF90EF90DF90CF90BF9094
:10A1F000AF909F908F9008958091071490910814CC
:10A20000009711F00C941B5D60E070E0CB010895A5
:10A21000CF93DF93CDB7DEB7A5970FB6F894DEBF27
:10A220000FBECDBF789484B5826084BD84B5816053
:10A2300084BD85B5826085BD85B5816085BD809111
:10A240006E00816080936E00109281008091810089
:10A250008260809381008091810081608093810081
:10A26000809180008160809380008091B100846043
:10A270008093B1008091B00081608093B0008091A4
:10A280009100826080939100809191008160809321
:10A290009100809190008160809390008091A10056
:10A2A00082608093A1008091A10081608093A100D1
:10A2B0008091A00081608093A00080912101826044
:10A2C00080932101809121018160809321018091FF
:10A2D000200181608093200180917A0084608093C6
:10A2E0007A0080917A00826080937A0080917A006F
:10A2F000816080937A0080917A00806880937A00F0
:10A300001092C10020E042E060E18EED94E10E94F5
:10A310003D428EED94E10E94B7416AEB79E08EED0B
:10A3200094E10E94803E86E892E10E9412368CE41D
:10A3300091E10E94123660ED77E080E090E00E94AB
:10A34000594086E892E10E94553A782E83E77816C4
:10A3500009F46BC1109239101092381012EBE12EF3
:10A3600010E1F12E00E010E0C8010E94E062D70188
:10A370008D937D010F5F1F4F0A341105A9F780915E
:10A38000B2109091B310A091B410B091B510853671
:10A390009105A105B1050CF43AC180934703909350
:10A3A0004803A0934903B0934A038091B61090915B
:10A3B000B710A091B810B091B91080934303909357
:10A3C0004403A0934503B09346038091BA10909143
:10A3D000BB10A091BC10B091BD1080933F0390932F
:10A3E0004003A0934103B09342036EEC70E1CE01B1
:10A3F00001960E949A3DBE016F5F7F4F88ED94E108
:10A400000E94A23CCE0101960E94DB3C8091BE10CE
:10A410009091BF10A091C010B091C1108093AA0379
:10A420009093AB03A093AC03B093AD038091C210A3
:10A430009091C310A091C410B091C5108093A60351
:10A440009093A703A093A803B093A9038091C6108B
:10A450009091C710A091C810B091C9108093AE031D
:10A460009093AF03A093B003B093B1038091CA104F
:10A470009091CB10A091CC10B091CD108093B203ED
:10A480009093B303A093B403B093B5038091D61017
:10A490009091D710A091D810B091D91080938703D4
:10A4A00090938803A0938903B0938A038091DA1074
:10A4B0009091DB10A091DC10B091DD1080938303AC
:10A4C00090938403A0938503B09386038091DE105C
:10A4D0009091DF10A091E010B091E11080937F0384
:10A4E00090938003A0938103B09382038091E21044
:10A4F0009091E310A091E410B091E51080937B035C
:10A5000090937C03A0937D03B0937E038091E6102B
:10A510009091E710A091E810B091E91080933B036F
:10A5200090933C03A0933D03B0933E0340912303DB
:10A5300050912403A0902503B09026038090270318
:10A540009090280360918B0370918C0300912103FC
:10A550001091220340901F0350902003ECEBF3E096
:10A56000ACEEEA2EA0E1FA2EBBE2CB2EB3E0DB2E5E
:10A5700021E030E08091290390912A03821793070C
:10A5800074F1D7018D919D917D01D6018D939D939D
:10A590006D018430910519F48280938018C08A304F
:10A5A000910519F4A280B38012C08530910519F489
:10A5B0004281538110C08630910519F46281738104
:10A5C0000AC08730910519F40281138104C00B97EA
:10A5D00014F0428053802F5F3F4F3296CBCF1093C1
:10A5E0002203009321035092200340921F03709393
:10A5F0008C0360938B035093240340932303B09206
:10A600002603A0922503909228038092270380912D
:10A61000B2109091B310A091B410B091B5108536DE
:10A620009105A105B1050CF0FEC080914703909102
:10A630004803A0914903B0914A038093B2109093CC
:10A64000B310A093B410B093B510809143039091D0
:10A650004403A0914503B09146038093B6109093B4
:10A66000B710A093B810B093B91080913F039091A8
:10A670004003A0914103B09142038093BA1090939C
:10A68000BB10A093BC10B093BD108EEC90E1892B51
:10A69000E1F00091DC141091DD140115110519F49D
:10A6A0001092CE1012C00730110510F007E010E034
:10A6B0006091D8147091D914A8018EEC90E10E9499
:10A6C0001A69F801E253FF4E10828091AA0390911B
:10A6D000AB03A091AC03B091AD038093BE109093F7
:10A6E000BF10A093C010B093C1108091A6039091A9
:10A6F000A703A091A803B091A9038093C2109093DF
:10A70000C310A093C410B093C5108091AE03909174
:10A71000AF03A091B003B091B1038093C6109093A2
:10A72000C710A093C810B093C9108091B203909144
:10A73000B303A091B403B091B5038093CA10909372
:10A74000CB10A093CC10B093CD1080918703909143
:10A750008803A0918903B0918A038093D6109093C7
:10A76000D710A093D810B093D91080918303909103
:10A770008403A0918503B09186038093DA109093AF
:10A78000DB10A093DC10B093DD1080917F039091DB
:10A790008003A0918103B09182038093DE10909397
:10A7A000DF10A093E010B093E11080917B039091B3
:10A7B0007C03A0917D03B0917E038093E21090937F
:10A7C000E310A093E410B093E51080913B039091C7
:10A7D0003C03A0913D03B0913E038093E61090931B
:10A7E000E710A093E810B093E9102091290330916D
:10A7F0002A03A9E2B3E0EAEEF0E180E090E0281756
:10A80000390734F04D915D91419351930196F7CF03
:10A81000B3E77B1208C0109239101092381080E014
:10A8200090E00E943E366CE271E080E090E00E9491
:10A83000594068EC70E080E090E00E94594068EC7C
:10A8400070E080E090E00E945940F89482E08093AC
:10A85000B0008093B10094E69093B3001092B200E0
:10A8600080937000789480932F131092321380910C
:10A87000301360E00E94D33F0E94E44A60E080E031
:10A880000E94B7386BEC79E08EED94E10E94803E37
:10A8900061E080E00E94B73868ED74E1CE01019676
:10A8A0000E94923D65EF79E0CE0101960E943C3C0A
:10A8B000BC018EED94E10E94B53DCE0101960E944F
:10A8C000DB3C8E01035F1F4F64E175E0C8010E940D
:10A8D0009A3D68ED74E1C8010E94533C6BED79E04C
:10A8E0000E943C3CBC01CE0101960E94923DCE01EB
:10A8F00001960E94022FCE0101960E94DB3CC80106
:10A900000E94DB3C80913703909138030A97B1F4A1
:10A910008091390390913A030A9781F489EE91E18D
:10A920000E9412368CED95E0A0E0B0E08093ED112E
:10A930009093EE11A093EF11B093F01168EE73E0D5
:10A9400080E090E00E9459408DEF99E00E94E4344D
:10A950000E9493388CE09AE00E94E43480E090E01A
:10A96000A0E8BFE380933C1490933D14A0933E1461
:10A97000B0933F1469E17AE086E892E10E94803E5C
:10A9800060913F0370914003809141039091420395
:10A9900041E00E94BA3782E29AE00E94E43460917A
:10A9A0003F037091400380914103909142030E94C4
:10A9B000E7369093351080933410892B21F086EB85
:10A9C00095E00E94E43486E29AE00E94E43460E07C
:10A9D00070E082E090E00E94D63680E090E09093B4
:10A9E000351080933410892B21F086EB95E00E947E
:10A9F000E4340E94933864E670E080E090E00E94C6
:10AA0000594083E20E94CC3681E090E00E943936C2
:10AA10000E946F3683E0809325140E94933880ED66
:10AA20000E94DE39853509F074C58AEA0E943E39F4
:10AA300090932714809326148CEA0E943E399093B9
:10AA40002914809328148EEA0E943E3990932B1487
:10AA500080932A1480EB0E943E39909337148093A0
:10AA6000361482EB0E943E39909339148093381447
:10AA700084EB0E943E3990933B1480933A1486EB0A
:10AA80000E943E3990932D1480932C1488EB0E94E1
:10AA90003E3990932F1480932E148AEB0E943E39F6
:10AAA00090933114809330148CEB0E943E39909334
:10AAB0003314809332148EEB0E943E3990933514F8
:10AAC000809334140E9406450E94CA610E94B364B8
:10AAD0000E94CA6120E030E048EC52E40E941A640F
:10AAE000AB01BC0122E0CE0101960E94E03C68E38C
:10AAF0007AE0C8010E949A3DBE016F5F7F4FC80196
:10AB00000E94533C6DE675E00E943C3CBC018DE028
:10AB100094E10E948D3CC8010E94DB3CCE0101966D
:10AB20000E94DB3C6DE074E186E892E10E94703E99
:10AB300060914703709148038091490390914A03C3
:10AB40000E94CA6120E030E048EC52E40E941A649E
:10AB5000AB01BC0122E0CE0101960E94E03C6CE416
:10AB60007AE0C8010E949A3DBE016F5F7F4FC80125
:10AB70000E94533C6DE675E00E943C3CBC018DE0B8
:10AB800094E10E948D3CC8010E94DB3CCE010196FD
:10AB90000E94DB3C6DE074E186E892E10E94703E29
:10ABA0008CE59FE00E94E4340E94933860E08DE2DF
:10ABB0000E94A44760E18DE20E94A44768E08DE214
:10ABC0000E94A4474090541450905514609056141D
:10ABD0007090571449825A826B827C8280905814FC
:10ABE00090905914A0905A14B0905B148D829E825C
:10ABF000AF82B886C0905C14D0905D14E0905E1473
:10AC0000F0905F14C986DA86EB86FC8683E69AE0CC
:10AC10000E94E434FE0131961F01D1016D917D91B6
:10AC20008D919D911D0146E00E94BA3760E87FE05A
:10AC300086E892E10E94803E2016310671F78CE58D
:10AC40009FE00E94E43423E938E144E85FE3C30174
:10AC5000B2010E9429622B013C016D877E878F879C
:10AC6000988B22E430E645E85FE3C501B4010E9419
:10AC700029624B015C01698B7A8B8B8B9C8B25E85D
:10AC80003BEE41E95FE3C701B6010E9429626D8B8B
:10AC90007E8B8F8B988F40925414509255146092F3
:10ACA0005614709257148092581490925914A0928E
:10ACB0005A14B0925B1460935C1470935D1480938B
:10ACC0005E1490935F1481E79AE00E94E4348E0151
:10ACD000075E1F4FF10161917191819191911F0167
:10ACE00042E00E94BA3760E87FE086E892E10E9485
:10ACF000803E2016310671F78CE59FE00E94E43417
:10AD000040E654E166E070E082E30E943947C0907B
:10AD10006114D12CDC2CCC2480916014C82AE090E2
:10AD20006314F12CFE2CEE2480916214E82A009129
:10AD3000651410E0102F002780916414082B6EE733
:10AD40007AE086E892E10E94803E4AE050E0B60157
:10AD500086E892E10E94673E60E87FE086E892E143
:10AD60000E94803E4AE050E0B70186E892E10E94EE
:10AD7000673E60E87FE086E892E10E94803E4AE01C
:10AD800050E0B80186E892E10E94673E8CE59FE0C2
:10AD90000E94E434C1010E94F8476BE87AE086E83B
:10ADA00092E10E94803E8E010B5D1F4FD1016D919B
:10ADB0007D918D919D911D014AE00E94BA3760E816
:10ADC0007FE086E892E10E94803E2016310671F70E
:10ADD0008CE59FE00E94E43461E08DE10E94A4478D
:10ADE00064E97AE086E892E10E94803EA80161E091
:10ADF00070E08DE10E9439478DA190E00E94744778
:10AE000062E08EE10E94A44763E08FE10E94A447C4
:10AE100064E080E20E94A44768EA7AE086E892E172
:10AE20000E94803EA80161E070E08EE10E943947F7
:10AE3000ADA0B12CA80161E070E08FE10E9439471C
:10AE4000CDA0D12CA80161E070E080E20E943947DA
:10AE5000EDA0F12C4AE050E0B50186E892E10E94B5
:10AE6000673E60E87FE086E892E10E94803E4AE02B
:10AE700050E0B60186E892E10E94673E60E87FE01C
:10AE800086E892E10E94803E4AE050E0B70186E801
:10AE900092E10E94673E8CE59FE00E94E43465E009
:10AEA00081E20E94A44764EC7AE086E892E10E9485
:10AEB000803EA80161E070E081E20E9439478DA1E7
:10AEC00090E00E94744766E082E20E94A44767ED2A
:10AED0007AE086E892E10E94803EA80161E070E09D
:10AEE00082E20E9439478DA190E00E94744767E09A
:10AEF00083E20E94A4476FEE7AE086E892E10E9426
:10AF0000803EA80161E070E083E20E9439478DA194
:10AF100090E00E94744768E084E20E94A44765E0E4
:10AF20007BE086E892E10E94803EA80161E070E04B
:10AF300084E20E9439478DA190E00E94744769E045
:10AF400085E20E94A4476DE17BE086E892E10E94E1
:10AF5000803EA80161E070E085E20E9439478DA142
:10AF600090E00E9474476AE086E20E94A44767E38B
:10AF70007BE086E892E10E94803EA80161E070E0FB
:10AF800086E20E9439478DA190E00E9474476BE0F1
:10AF900088E20E94A4476DE47BE086E892E10E948B
:10AFA000803EA80161E070E088E20E9439478DA1EF
:10AFB00090E00E9474476CE089E20E94A44766E634
:10AFC0007BE086E892E10E94803EA80161E070E0AB
:10AFD00089E20E9439478DA190E00E9474476EE794
:10AFE0007BE086E892E10E94803E66E070E087E2C6
:10AFF0000E948A4790E00E94744765E97BE086E8FA
:10B0000092E10E94803E65E070E087E20E948A47FC
:10B0100090E00E9474476CEA7BE086E892E10E942F
:10B02000803E64E070E087E20E948A4790E00E94E0
:10B03000744763EC7BE086E892E10E94803E62E028
:10B0400070E087E20E948A4790E00E9474476CEDAE
:10B050007BE086E892E10E94803E61E070E087E25A
:10B060000E948A4790E00E94744765EF7BE086E883
:10B0700092E10E94803E60E070E087E20E948A4791
:10B0800090E00E9474476EE07CE086E892E10E94C6
:10B09000803E63E070E087E20E948A4790E00E9471
:10B0A000744741E067E070E087E20E94B94741E001
:10B0B00063E070E087E20E94B94741E063E070E03E
:10B0C0008AE20E94B9476FE17CE086E892E10E9443
:10B0D000803E63E070E08AE20E948A4790E00E942E
:10B0E000744740E063E070E08AE20E94B94768E399
:10B0F0007CE086E892E10E94803E63E070E08AE2B4
:10B100000E948A4790E00E94744741E062E070E04C
:10B110008AE20E94B94762E57CE086E892E10E94FB
:10B12000803E62E070E08AE20E948A4790E00E94DE
:10B13000744740E062E070E08AE20E94B9476EE640
:10B140007CE086E892E10E94803E62E070E08AE264
:10B150000E948A4790E00E94744741E061E070E0FD
:10B160008AE20E94B9476BE87CE086E892E10E949F
:10B17000803E61E070E08AE20E948A4790E00E948F
:10B18000744740E061E070E08AE20E94B94767EAF4
:10B190007CE086E892E10E94803E61E070E08AE215
:10B1A0000E948A4790E00E94744741E060E070E0AE
:10B1B0008AE20E94B94764EC7CE086E892E10E9452
:10B1C000803E60E070E08AE20E948A4790E00E9440
:10B1D000744740E060E070E08AE20E94B94760EEA8
:10B1E0007CE086E892E10E94803E60E070E08AE2C6
:10B1F0000E948A4790E00E94744741E066E070E058
:10B2000087E20E94B94741E065E070E087E20E9472
:10B21000B94741E064E070E087E20E94B94740E04E
:10B2200062E070E087E20E94B94740E061E070E0D0
:10B2300087E20E94B94740E060E070E087E20E9448
:10B24000B9476DEF7CE086E892E10E94803E66E0BF
:10B2500070E08BE20E948A4790E00E94744765E1AB
:10B260007DE086E892E10E94803E65E070E08BE23E
:10B270000E948A4790E00E94744763E37DE086E87D
:10B2800092E10E94803E64E070E08BE20E948A4777
:10B2900090E00E94744761E57DE086E892E10E94BB
:10B2A000803E62E070E08BE20E948A4790E00E945C
:10B2B00074476AE67DE086E892E10E94803E61E0A4
:10B2C00070E08BE20E948A4790E00E94744763E836
:10B2D0007DE086E892E10E94803E60E070E08BE2D3
:10B2E0000E948A4790E00E9474476CE97DE086E8FE
:10B2F00092E10E94803E63E070E08BE20E948A4708
:10B3000090E00E9474476FEA7DE086E892E10E9437
:10B31000803E64E070E08CE20E948A4790E00E94E8
:10B32000744740E064E070E08CE20E94B947A801F5
:10B3300061E070E08CE20E9439476DA1607F666039
:10B340008CE20E94A44764EC7DE086E892E10E94D2
:10B35000803EA80161E070E08CE20E9439476DA157
:10B360006F7070E066507109072E000C880B990B06
:10B370000E94CA619B01AC0160E070E080E090E453
:10B380000E94C86520E030E048EC50E40E94296249
:10B390000E94E94768ED7DE086E892E10E94803EE8
:10B3A000A80161E070E080E30E9439474DA150E0C0
:10B3B00060E070E02AE086E892E10E94D83D86E8ED
:10B3C00092E10E946D3E6FEE7DE086E892E10E9480
:10B3D000803E61E070E080E30E948A4790E00E9436
:10B3E000744767E07EE086E892E10E94803E61E07B
:10B3F00070E08FE20E948A4790E00E94744741E02B
:10B4000061E070E08FE20E94B94760E27EE086E88A
:10B4100092E10E94803E61E070E08EE20E948A47E5
:10B4200090E00E94744741E061E070E08EE20E948B
:10B43000B94740E067E070E081E30E94B94768E304
:10B440007EE086E892E10E94803E67E070E081E362
:10B450000E948A4790E00E9474476BE47EE086E891
:10B4600092E10E94803EA80161E070E080E00E94CD
:10B4700039478DA10E9468438CE59FE00E94E43427
:10B480008DE1E82EF12C62E57EE086E892E10E94F3
:10B49000803E40E150E0B70186E892E10E94673EBD
:10B4A00067E67DE086E892E10E94803EA80161E0C7
:10B4B00070E08E2D0E9439478DA10E9468438CE573
:10B4C0009FE00E94E434BFEFEB1AFB0AEAE3EE16BA
:10B4D000F104C9F668EE73E080E090E00E94594004
:10B4E00062E274E089E194E10E94783C81E090E0BE
:10B4F00090933710809336100E945E2C60ED77E0B9
:10B5000080E090E00E9459400E944F020E94263B3A
:10B51000FBCF65E57EE0CE0101960E949A3DCE010B
:10B5200001960E94022FCE0101960E94DB3C1092F0
:10B530001E03D0CF81E094E10E94DB3C87E094E1E0
:10B540000E94DB3C8DE094E10E94DB3C83E194E1CE
:10B550000E94DB3C89E194E10E94DB3C8FE194E1B5
:10B560000E94DB3C88ED94E10C94DB3C8F929F922F
:10B57000AF92BF92CF92DF92EF92FF92CF93109251
:10B580004F1110924E1188EE93E0A0E0B0E080934E
:10B59000501190935111A0935211B093531122ED79
:10B5A00033E030934D1120934C1145E351E050931B
:10B5B00059114093581144E351E050935B1140936B
:10B5C0005A1140E351E050935D1140935C1141E307
:10B5D00051E050935F1140935E1142E351E050936C
:10B5E00061114093601146E351E050936311409321
:10B5F00062111092651110926611109267111092EB
:10B6000068111092EC111092EB118093ED11909350
:10B61000EE11A093EF11B093F0113093EA11209343
:10B62000E91145ED50E05093F6114093F51144EDCA
:10B6300050E05093F8114093F71140ED50E05093D3
:10B64000FA114093F91141ED50E05093FC114093F1
:10B65000FB1142ED50E05093FE114093FD1146ED79
:10B6600050E0509300124093FF111092021210927A
:10B670000312109204121092051210928912109265
:10B68000881280938A1290938B12A0938C12B0939D
:10B690008D12309387122093861225EC30E0309380
:10B6A00093122093921224EC30E030939512209361
:10B6B000941220EC30E0309397122093961221ECF4
:10B6C00030E0309399122093981222EC30E03093BE
:10B6D0009B1220939A1226EC30E030939D12209317
:10B6E0009C1210929F121092A0121092A11210920E
:10B6F000A212109226131092251380932713909371
:10B700002813A0932913B0932A1384EE93E0909307
:10B710002413809323131092E1141092E01480E01C
:10B7200094E09093DF148093DE141092EE148FEF68
:10B730008093ED141092EC141092EF148FE3809329
:10B74000E9141092EA141092EB141092E81410927B
:10B75000E71484E08093F01482E08093F11481E098
:10B760008093F214C0E1C093F31480E28093F41448
:10B7700080E48093F51480E88093F61440E050E074
:10B7800063E08EED94E10E94E74068E47FE088ED9D
:10B7900094E10E949A3D88E18093D51481E18093E1
:10B7A000D614C093D71461E088E10E94D33F61E0D2
:10B7B0008091D5140E94A13F60E08091D6140E9430
:10B7C000D33F60E08091D7140E94D33F61E0809125
:10B7D000D6140E94A13F61E08091D7140E94A13F3E
:10B7E00061E08091D5140E94A13F109268141092DC
:10B7F0006C1410926B1410926D1486EF93E090937A
:10B8000067148093661480E090E0FC01EA59FB4ED7
:10B81000148E10A2178E11A206968C339105A9F7EB
:10B8200081E993E09093C9148093C8148DE893E064
:10B830009093CB148093CA1484E08093CC148093AB
:10B84000CD1485E993E09093C7148093C6148AE0E1
:10B8500090E09093CF148093CE1484EF91E0909376
:10B86000D1148093D0141092D4141092D314109247
:10B87000C2141092C3141092C4141092C5141092E2
:10B88000D21481E0809352141092531483EC9BEAFB
:10B89000A6E7BBE38093541490935514A0935614D9
:10B8A000B093571488ED9BE6A6E7BBE3809358144A
:10B8B00090935914A0935A14B0935B1482EF94EEB2
:10B8C000A4E6BBE380935C1490935D14A0935E1494
:10B8D000B0935F1480918B0390918C0390935114DB
:10B8E000809350148090870390908803A0908903E0
:10B8F000B0908A03209183033091840340918503A3
:10B9000050918603C501B401CED66B017C016093D2
:10B910004C1470934D1480934E1490934F14609177
:10B920007F037091800380918103909182036093E3
:10B930004014709341148093421490934314809266
:10B94000441490924514A0924614B092471420914A
:10B950007B0330917C0340917D0350917E03A3D6FD
:10B960009B01AC01C701B60165D760934814709381
:10B97000491480934A1490934B1480E090E0A0E81F
:10B98000BFE380933C1490933D14A0933E14B09376
:10B990003F146CE57FE08FE194E10E949A3D6CE5F5
:10B9A0007FE089E194E10E949A3D6CE57FE083E1CC
:10B9B00094E10E949A3D6CE57FE08DE094E10E9465
:10B9C0009A3D6CE57FE087E094E10E949A3D6CE54A
:10B9D0007FE081E094E10E949A3D87E080933013FC
:10B9E00010923113CF91FF90EF90DF90CF90BF90E6
:10B9F000AF909F908F900895EF920F931F93CF93E6
:10BA0000DF93E80147FD02C034E001C034E1E42FD8
:10BA1000440FFF0BF7FF03C0F195E195F109E32E09
:10BA2000022F2E2FAE01B5D0CE01DF91CF911F9105
:10BA30000F91EF9008956627772738C21F93FC0176
:10BA400099278827BC01E89411911032E9F3193045
:10BA500010F01E30C8F31B3249F01D3241F46894D7
:10BA600005C03ED0610F711D811D911D11911053B4
:10BA70001A30B8F33EF490958095709561957F4F9C
:10BA80008F4F9F4F1F9108954532510518F4423052
:10BA900008F004C0FB011082CB010895BB274A3097
:10BAA00031F4992322F4BDE2909581959F4F59C0BE
:10BAB0002532310518F4223008F004C0FA01108252
:10BAC000CA010895BB272A3051F4992342F4BDE2FC
:10BAD00090958095709561957F4F8F4F9F4F20C0B7
:10BAE000592F482F372F262F660F771F881F991F32
:10BAF000660F771F881F991F620F731F841F951F82
:10BB0000660F771F881F991F08952532310518F495
:10BB1000223008F004C0FA011082CA010895BB2740
:10BB2000FA01A62F6217710581059105330B30FBD1
:10BB300066F0AA27660F771F881F991FAA1FA217F2
:10BB400010F0A21B63953850A9F7A05DAA3308F046
:10BB5000A95DA19336F7B111B1931082CA0104C453
:10BB6000BB27FB015527AA27880F991FAA1FA417D7
:10BB700010F0A41B83955051B9F7A05DAA3308F0CB
:10BB8000A95DA193009779F7B111B1931192CB01FF
:10BB9000EBC34F925F926F927F929F92AF92BF9250
:10BBA000CF92DF92EF92FF920F931F93CF93DF9389
:10BBB000CDB7DEB729970FB6F894DEBF0FBECDBF65
:10BBC0006A01122FB02E2BE3201720F0FF24F394EC
:10BBD000F00E02C0BCE3FB2E0F2D27E0AE014F5F3D
:10BBE0005F4FCAD2AC018981982F9970913031F0A2
:10BBF000E1FC06C0E0FE06C090E205C09DE203C085
:10BC00009BE201C090E0EE2DE07183FF3CC09111FA
:10BC100002C083E001C084E0811718F4212F281BA3
:10BC200001C020E0E1110BC0F601822F30E2882331
:10BC300019F031938150FBCFC20ED11C20E0992323
:10BC400029F0D6019C93F60131966F01C601039647
:10BC5000E2FE0AC03EE4D6013C9341E411964C93C7
:10BC6000119712963C9306C03EE6F601308341E6FA
:10BC700041833283FC01322F40E2332309F442C076
:10BC800041933150FACF82FF44C0911102C083E04A
:10BC900001C084E0811718F4212F281B01C020E087
:10BCA000E1110BC0F601822F30E2882319F03193A5
:10BCB0008150FBCFC20ED11C20E0992329F0D60180
:10BCC0009C93F60131966F01C6010396E2FE0BC00C
:10BCD00039E4D6013C933EE411963C93119736E447
:10BCE00012963C9307C039E6F60130833EE6318375
:10BCF00036E63283FC01322F40E2332319F04193C0
:10BD00003150FBCFFC01E20FF11D10828EEF9FEF4F
:10BD1000B7C0F1E0911101C0F0E06F2F70E0141690
:10BD2000150624F49A012F5F3F4F02C021E030E056
:10BD3000260F371FBB2029F06B2D70E06F5F7F4F00
:10BD400002C060E070E0260F371F612F70E02617F9
:10BD500037071CF4121B212F01C020E03E2D387143
:10BD600059F4D601322F60E2332319F06D9331502C
:10BD7000FBCFC20ED11C20E0FF2331F0D6019C93F3
:10BD8000B6016F5F7F4F6B01E1110BC0F601922F7F
:10BD900030E3992319F031939150FBCFC20ED11C9F
:10BDA00020E09F2D940F3A81782F7071A72E84FF89
:10BDB00003C0313309F49150191624F4993018F066
:10BDC00098E001C091E0E42F852F57FF02C0E0E02A
:10BDD00080E06E2F782FE0E0F0E0AEE29A2E3A019C
:10BDE000691A71082A01461A570A0B2D10E011959D
:10BDF000019511096F3F8FEF780729F4D6019C92C6
:10BE0000C60101966C014617570784F0661677063F
:10BE10006CF47F01E40CF51CA1E0B0E0AC0FBD1F99
:10BE2000EA0EFB1ED7011196BC9002C090E3B92E1A
:10BE3000615071093196C60101967C016017710746
:10BE400024F0D601BC926C01D5CF6417750741F47C
:10BE5000363320F4353321F4A11002C081E3B82E2B
:10BE6000F601B082F701822F90E2882319F09193B6
:10BE70008150FBCFF701E20FF11D108280E090E0CE
:10BE800029960FB6F894DEBF0FBECDBFDF91CF91DC
:10BE90001F910F91FF90EF90DF90CF90BF90AF90E8
:10BEA0009F907F906F905F904F9008956F927F92D8
:10BEB0008F929F92AF92BF92CF92DF92EF92FF92BA
:10BEC0000F931F93CF93DF93EC017B0161157105F5
:10BED00019F0DB018D939C938E010F5F1F4F7880CB
:10BEE000872D90E021D2892B11F0E801F5CFBDE23A
:10BEF0007B1205C00F5F1F4F7980C1E008C0EBE2E5
:10BF00007E1204C08E010E5F1F4F7980C0E0680171
:10BF1000F1E0CF1AD10843E050E068EE71E0C601CD
:10BF20000BD2892BE9F4680122E0C20ED11C45E056
:10BF300050E063EE71E0C601FFD1892B21F4680166
:10BF400087E0C80ED11CE114F10419F0D701CD929D
:10BF5000DC92C111F9C060E070E080E89FE7FDC0AD
:10BF600043E050E060EE71E0C601E6D1892B51F468
:10BF7000E114F10409F4EDC00E5F1F4FF7011183C6
:10BF80000083E7C0680160E070E0CB0100E010E0F2
:10BF9000F601D0EDD70DDA3050F52C2F2260622E4D
:10BFA0002C2F2870C2FF05C0211127C00F5F1F4F23
:10BFB00024C0222311F001501109A5E0B0E09B013B
:10BFC000AC0130D34B015C01880C991CAA1CBB1C32
:10BFD000C501B4016D0F711D811D911D6839A9E95D
:10BFE0007A078A07A9E19A0740F0C66005C0DE3FDC
:10BFF00051F4C3FD44C0C8606C2EBFEFCB1ADB0AFE
:10C000007080C62DC5CF2D2F2F7D2531C1F54081E4
:10C010004D3211F4C06106C04B3221F0319621E05F
:10C0200030E006C03296D60111964C9122E030E005
:10C03000A0EDA40FAA3018F0E21BF30B20C040E0E3
:10C0400050E04038BCE05B075CF49A01220F331FDC
:10C05000220F331F420F531F440F551F4A0F511D0C
:10C060003196DF0111972C91A0EDA20FAA3048F371
:10C07000C4FF03C0519541955109040F151FC1FF1D
:10C0800007C0E114F10421F03197D701ED93FC933F
:10C090007FD1C370C33019F06B017C0106C06B0106
:10C0A0007C01F7FAF094F7F8F09420E030E0A90171
:10C0B000C701B60169D1882309F443C017FF06C040
:10C0C000119501951109CFEFD1E002C0C7E1D2E08F
:10C0D0005E01B8E1AB1AB1084601BE2DAF2D90E26A
:10C0E000E92EF12C0E151F057CF0FE0125913591EE
:10C0F00045915491B4018B2F9A2FABD14B01B82F9E
:10C10000A92F0E191F09EECF2497F594E794CA15AD
:10C11000DB0541F76401EB2EFA2E8E2D880F8F2D53
:10C12000881F8F3F41F020E030E0A901C701B60130
:10C130002BD1811106C082E290E090936415809328
:10C140006315C701B60109C060E070E080E89FEFA9
:10C1500004C060E070E080EC9FE7DF91CF911F9119
:10C160000F91FF90EF90DF90CF90BF90AF909F9096
:10C170008F907F906F900895283008F027E0332744
:10C18000DA01990F311D87FD9160009661057105F7
:10C1900039F432602E5F3D9330E32A95E1F708953C
:10C1A0009F3F30F080387105610509F03C5F3C5FCE
:10C1B0003D93913008F08068911DDF93CF931F93DA
:10C1C0000F93FF92EF92192F987F9695E92F9695EE
:10C1D0009695E90FFF27EB58FD4F99273327EE245B
:10C1E000FF24A701E70105900894079428F4360F6F
:10C1F000E71EF81E491F511D660F771F881F991FE4
:10C200000694A1F70590079428F4E70EF81E491F3D
:10C21000561FC11D770F881F991F661F0694A1F72F
:10C220000590079428F4F80E491F561FC71FD11D0B
:10C23000880F991F661F771F0694A1F70590079432
:10C2400020F4490F561FC71FD81F990F661F771F6D
:10C25000881F0694A9F784911095177041F0D69520
:10C26000C79557954795F794E7941A95C1F7EBE171
:10C27000F2E068941590159135916591959105902E
:10C280007FE27395E118F10A430B560BC90BD009F5
:10C29000C0F7E10CF11E431F561FC91FD01D7EF4CD
:10C2A000703311F48A95E6CFE894015030F0080F0E
:10C2B0000AF40027021708F4202F2395022F7A335F
:10C2C00028F079E37D932A95E9F710C07D932A95AC
:10C2D00089F6069497956795379517951794E11801
:10C2E000F10A430B560BC90BD00998F023957E91A8
:10C2F00073957A3308F070E37C932013B8F77E913E
:10C3000070617D9330F0839571E37D9370E32A959E
:10C31000E1F71124EF90FF900F911F91CF91DF91E2
:10C32000992787FD909508959111F6C0803219F0F4
:10C3300089508550D0F70895FB01DC0141505040F1
:10C3400088F08D9181341CF08B350CF4805E659102
:10C3500061341CF06B350CF4605E861B611171F367
:10C36000990B0895881BFCCFDC01FC01672F7191AC
:10C370007723E1F7329704C07C916D9370836291CB
:10C38000AE17BF07C8F3089540D008F481E00895C0
:10C39000E89409C097FB3EF490958095709561955F
:10C3A0007F4F8F4F9F4F9923A9F0F92F96E9BB2715
:10C3B0009395F695879577956795B795F111F8CF91
:10C3C000FAF4BB0F11F460FF1BC06F5F7F4F8F4FFC
:10C3D0009F4F16C0882311F096E911C0772321F0F2
:10C3E0009EE8872F762F05C0662371F096E8862F8A
:10C3F00070E060E02AF09A95660F771F881FDAF7E1
:10C40000880F9695879597F90895990F0008550F0D
:10C41000AA0BE0E8FEEF16161706E807F907C0F0CA
:10C4200012161306E407F50798F0621B730B840BD2
:10C43000950B39F40A2661F0232B242B252B21F4AC
:10C4400008950A2609F4A140A6958FEF811D811D4C
:10C4500008950BD07BC06CD028F071D018F09523D4
:10C4600009F05DC062C01124A5C081D0A0F3959FE2
:10C47000D1F3950F50E0551F629FF001729FBB27CB
:10C48000F00DB11D639FAA27F00DB11DAA1F649F77
:10C490006627B00DA11D661F829F2227B00DA11D2A
:10C4A000621F739FB00DA11D621F839FA00D611DB0
:10C4B000221F749F3327A00D611D231F849F600DD1
:10C4C000211D822F762F6A2F11249F5750408AF00A
:10C4D000E1F088234AF0EE0FFF1FBB1F661F771F96
:10C4E000881F91505040A9F79E3F510570F017C02A
:10C4F00061C05F3FECF3983EDCF3869577956795D6
:10C50000B795F795E7959F5FC1F7FE2B880F911DB3
:10C510009695879597F9089599278827089597F90B
:10C520009F6780E870E060E008959FEF80EC0895D9
:10C5300000240A9416161706180609060895002402
:10C540000A9412161306140605060895092E03947C
:10C55000000C11F4882352F0BB0F40F4BF2B11F4F0
:10C5600060FF04C06F5F7F4F8F4F9F4F089557FD4F
:10C570009058440F551F59F05F3F71F04795880F51
:10C5800097FB991F61F09F3F79F0879508951216E8
:10C5900013061406551FF2CF4695F1DF08C0161694
:10C5A00017061806991FF1CF869571056105089445
:10C5B0000895E894BB2766277727CB0197F908955C
:10C5C000F999FECF92BD81BDF89A992780B508955B
:10C5D000262FF999FECF1FBA92BD81BD20BD0FB69F
:10C5E000F894FA9AF99A0FBE01960895052E97FBD2
:10C5F00016F400940FD057FD05D024D007FC02D0CC
:10C6000046F408C050954095309521953F4F4F4FC7
:10C610005F4F089590958095709561957F4F8F4FEE
:10C620009F4F089531D0A59F900DB49F900DA49F6A
:10C63000800D911D11240895B7FFF4CFF3DF821B05
:10C64000930B0895A1E21A2EAA1BBB1BFD010DC07E
:10C65000AA1FBB1FEE1FFF1FA217B307E407F507B2
:10C6600020F0A21BB30BE40BF50B661F771F881F8E
:10C67000991F1A9469F760957095809590959B0124
:10C68000AC01BD01CF010895A29FB001B39FC001CD
:10C69000A39F700D811D1124911DB29F700D811DEE
:10C6A0001124911D08955058BB27AA270ED04ECFB4
:10C6B0003FDF30F044DF20F031F49F3F11F41EF4EF
:10C6C00034CF0EF4E095E7FB2ACFE92F50DF80F35B
:10C6D000BA17620773078407950718F071F49EF57F
:10C6E00068CF0EF4E0950B2EBA2FA02D0B01B901E7
:10C6F00090010C01CA01A0011124FF27591B99F0D8
:10C70000593F50F4503E68F11A16F040A22F232FE3
:10C71000342F4427585FF3CF469537952795A79533
:10C72000F0405395C9F77EF41F16BA0B620B730BDA
:10C73000840BBAF09150A1F0FF0FBB1F661F771F4B
:10C74000881FC2F70EC0BA0F621F731F841F48F400
:10C75000879577956795B795F7959E3F08F0B3CF86
:10C760009395880F08F09927EE0F97958795089570
:10C77000DFDE58F080E891E009F49EEFE0DE28F07B
:10C7800040E851E059F45EEF09C0CFCE12CFE92F57
:10C79000E078EDDE68F3092E052AC1F32617370786
:10C7A0004807590738F00E2E07F8E02569F0E02514
:10C7B000E0640AC0EF6307F8009407FADB01B901EF
:10C7C0009D01DC01CA01AD01EF9343D0BFDE0AD069
:10C7D0005F91552331F02BED3FE049E450FD49ECEA
:10C7E00063CF0895DF93DD27B92FBF7740E85FE37C
:10C7F0001616170648075B0710F4D92F0ED19F9322
:10C800008F937F936F9352D2E0E3F1E0DDD09EDE11
:10C810002F913F914F915F9128DEDD2349F0905891
:10C82000A2EA2AED3FE049EC5FE3D0785D274DDFD7
:10C83000DF918CCE0CD08ACE82DE40F079DE30F0F3
:10C8400021F45F3F19F06BCE5111B4CE6ECE8FDE66
:10C8500098F39923C9F35523B1F3951B550BBB27C7
:10C86000AA2762177307840738F09F5F5F4F220F74
:10C87000331F441FAA1FA9F333D00E2E3AF0E0E86D
:10C8800030D091505040E695001CCAF729D0FE2FB9
:10C8900027D0660F771F881FBB1F2617370748074B
:10C8A000AB07B0E809F0BB0B802DBF01FF27935801
:10C8B0005F4F2AF09E3F510568F031CE7BCE5F3F3F
:10C8C000ECF3983EDCF3869577956795B795F795E9
:10C8D0009F5FC9F7880F911D9695879597F90895E1
:10C8E000E1E0660F771F881FBB1F6217730784077D
:10C8F000BA0720F0621B730B840BBA0BEE1F88F78C
:10C90000E095089519F40EF00ACE53CE0ECE37DE20
:10C91000C8F39638C0F707F80F92E8942BE33AEA89
:10C9200048EB5FE7A4DD0F920F920F924DB75EB711
:10C930000F92FBD0EDE5F1E047D04F915F91EF9181
:10C94000FF91E595EE1FFF1F49F0FE57E068442771
:10C95000EE0F441FFA95E1F74195550B67D00F9004
:10C9600007FE5BC0089504D06894B11123CE0895EA
:10C9700006DE88F09F5790F0B92F9927B751A0F0A5
:10C98000D1F0660F771F881F991F1AF0BA95C9F763
:10C9900012C0B13081F00DDEB1E008950ACE672FEC
:10C9A000782F8827B85F39F0B93FCCF38695779513
:10C9B0006795B395D9F73EF49095809570956195FC
:10C9C0007F4F8F4F9F4F0895DF93CF931F930F9308
:10C9D000FF92EF92DF927B018C01689405C0DA2E02
:10C9E000EF0143DDFE01E894A59125913591459134
:10C9F0005591AEF3EF0169DEFE019701A801DA94CB
:10CA000079F7DF90EF90FF900F911F91CF91DF9119
:10CA10000895FBDC08F48FEF08959B01AC0160E002
:10CA200070E080E89FE306CF7ACD47C1A8DDE8F348
:10CA30009923D9F3940F511DBBF39150504094F0BA
:10CA400059F0882332F0660F771F881F91505040AD
:10CA5000C1F79E3F510544F7880F911D9695879524
:10CA600097F908955F3FACF0983E9CF0BB27869500
:10CA700077956795B79508F4B1609395C1F7BB0FAB
:10CA800058F711F460FFE8CF6F5F7F4F8F4F9F4FD4
:10CA9000E3CF90CD0AD029ED3BE54EED5EE3D9CC56
:10CAA0000EF00BC142CD68943ACD69DDC8F39923ED
:10CAB000D1F3C6F3DF93CF931F930F93FF92C92F48
:10CAC000DD2788232AF02197660F771F881FDAF762
:10CAD00020E030E040E85FEB9FE3883920F0803EC3
:10CAE00030F021968F77E0DDE5E8F1E003C0DCDD92
:10CAF000E2EBF1E069DF8B01BE01EC01FB2E6F5729
:10CB000071097595771F880B990B44DC28E132E792
:10CB100041E35FE3AADCAF2D9801AE01FF900F91D6
:10CB20001F91CF91DF91D1DD11CDFA01DC01AA0F68
:10CB3000BB1F9B01AC01BF5728F422273327442792
:10CB400050781FC0B75188F4AB2F00244695379515
:10CB50002795011CA395D2F3002069F0220F331F03
:10CB6000441FB395DAF30DD09ECD61307105A0E876
:10CB70008A07B94630F49B01AC01662777278827DE
:10CB80009078309621F02083318342835383089537
:10CB9000FA01EE0FFF1F30962105310599F161155D
:10CBA000710561F48038BFE39B0749F168949038C0
:10CBB000810561F08038BFEF9B0741F0992342F572
:10CBC000FF3FE1053105210511F1E8940894E7954F
:10CBD000D901AA2329F4AB2FBE2FF85FD0F310C0E0
:10CBE000FF5F70F4A695E0F7F73950F019F0FF3ABF
:10CBF00038F49F779F930CD00F9007FC90580895BE
:10CC00003EF093CC60E070E080E89FE308954FE74A
:10CC10009F775F934F933F932F9347DF2F913F91E0
:10CC20004F915F9116DC73CE11F40EF47ECC45C0AB
:10CC3000A6DCD0F39923D9F3CEF39F57550B87FF8A
:10CC40004AD00024A0E640EA900180585695979576
:10CC500028F4805C660F771F881F20F0261737079F
:10CC6000480730F4621B730B840B202931294A2BAF
:10CC7000A69517940794202531254A2758F7660F63
:10CC8000771F881F20F026173707480730F4620BFC
:10CC9000730B840B200D311D411DA09581F7B90147
:10CCA000842F9158880F9695879508959B01AC0124
:10CCB000D0CBABDB880B990B08959F3F31F091509F
:10CCC00020F4879577956795B795880F911D969570
:10CCD000879597F9089591505040660F771F881FE8
:10CCE000D2F70895DB018F939F939CDCBF91AF91A6
:10CCF000A29F800D911DA39F900DB29F900D1124B6
:10CD0000089597FB072E16F4009406D077FD08D0FF
:10CD10004AD007FC05D03EF4909581959F4F089529
:10CD2000709561957F4F0895EE0FFF1F881F8BBF91
:10CD30000790F691E02D19940F93083090F0982FFA
:10CD4000872F762F652F542F432F322F22270850FD
:10CD5000F4CF220F331F441F551F661F771F881FF4
:10CD6000991F0A95B2F70F91089597FB10F8169442
:10CD700000080F93083098F00850232F342F452FC8
:10CD8000562F672F782F892F902DF4CF05949795E4
:10CD900087957795679557954795379527950A9580
:10CDA000AAF70F910895AA1BBB1B51E107C0AA1F48
:10CDB000BB1FA617B70710F0A61BB70B881F991F3C
:10CDC0005A95A9F780959095BC01CD010895CF9310
:10CDD000DF938230910510F482E090E0E0916715D6
:10CDE000F091681520E030E0C0E0D0E0309711F11C
:10CDF0004081518148175907C0F04817590761F41D
:10CE000082819381209719F09B838A832BC0909312
:10CE100068158093671526C02115310519F0421752
:10CE2000530718F49A01BE01DF01EF010280F3817C
:10CE3000E02DDCCF2115310509F1281B390B2430F9
:10CE4000310590F412968D919C911397611571059F
:10CE500021F0FB019383828304C090936815809333
:10CE60006715FD01329644C0FD01E20FF31F819367
:10CE70009193225031092D933C933AC0209165152E
:10CE800030916615232B41F42091B8033091B903FA
:10CE900030936615209365152091B6033091B70342
:10CEA0002115310541F42DB73EB74091BA03509199
:10CEB000BB03241B350BE0916515F0916615E21755
:10CEC000F307A0F42E1B3F0B2817390778F0AC01AD
:10CED0004E5F5F4F2417350748F04E0F5F1F50938A
:10CEE0006615409365158193919302C0E0E0F0E0F0
:10CEF000CF01DF91CF9108950F931F93CF93DF93CD
:10CF0000009709F48CC0FC013297138212820091C1
:10CF10006715109168150115110581F42081318183
:10CF2000820F931F209165153091661528173907D8
:10CF300079F5F0936615E093651571C0D80140E06E
:10CF400050E0AE17BF0750F412962D913C91139705
:10CF5000AD012115310509F1D901F3CF9D01DA01A8
:10CF60003383228360817181860F971F8217930715
:10CF700069F4EC0128813981260F371F2E5F3F4F5E
:10CF8000318320838A819B8193838283452B29F47B
:10CF9000F0936815E093671542C01396FC93EE93E7
:10CFA0001297ED01499159919E01240F351FE21707
:10CFB000F30771F480819181840F951F0296119679
:10CFC0009C938E938281938113969C938E93129758
:10CFD000E0E0F0E0D80112968D919C9113970097B4
:10CFE00019F0F8018C01F6CF8D919C9198012E5F7C
:10CFF0003F4F820F931F20916515309166152817BA
:10D00000390769F4309729F4109268151092671562
:10D0100002C0138212821093661500936515DF918A
:10D02000CF911F910F9108956F927F928F929F924F
:10D03000AF92BF92CF92DF92EF92FF920F931F9326
:10D04000CF93DF93EC01009781F4CB01DF91CF9177
:10D050001F910F91FF90EF90DF90CF90BF90AF9016
:10D060009F908F907F906F90B2CEFC01E60FF71FDC
:10D070009C0122503109E217F30708F4A8C0D90136
:10D080000D911C91119706171707A8F0053011058F
:10D0900008F49BC0C80104978617970708F495C049
:10D0A00002501109061B170B019311936D937C938A
:10D0B000CF0122DF8AC05B01A01AB10A4C01800EA9
:10D0C000911EA0916715B091681540E050E0E12CE9
:10D0D000F12C109709F44AC0A815B905D1F56D9047
:10D0E0007C901197630182E0C80ED11CCA14DB0446
:10D0F00080F1A3014A195B096A0182E0C80ED11CC4
:10D100001296BC9012971396AC91B5E0CB16D10451
:10D1100040F0B282A38351834083D9016D937C9305
:10D120000AC00E5F1F4FC301800F911FF901918349
:10D130008083EB2DFA2FE114F10431F0D70113961F
:10D14000FC93EE93129741C0F0936815E093671536
:10D150003CC08D919C9111974817590708F4AC0178
:10D160007D0112960D90BC91A02DB3CF80916515D5
:10D170009091661588159905E1F446175707C8F48C
:10D180008091B6039091B703009741F48DB79EB795
:10D190004091BA035091BB03841B950BE817F90724
:10D1A000B0F4F0936615E0936515F901718360831F
:10D1B0000CC0CB010CDE7C01009749F0A801BE0138
:10D1C0001BD0CE0199DEC70104C0CE0102C080E0B1
:10D1D00090E0DF91CF911F910F91FF90EF90DF9042
:10D1E000CF90BF90AF909F908F907F906F90089559
:10D1F00081E090E0F89447C0FB01DC0102C001909F
:10D200000D9241505040D8F70895FB01DC01019088
:10D210000D920020E1F70895FB01DC0141505040E0
:10D2200030F08D910190801919F40020B9F7881B16
:10D23000990B0895FB01DC014150504048F00190EA
:10D240000D920020C9F701C01D9241505040E0F7F7
:10D250000895FB0151915523A9F0BF01DC014D91C7
:10D2600045174111E1F759F4CD010190002049F033
:10D270004D9140154111C9F3FB014111EFCF81E000
:10D2800090E00197089512E0CCE1D2E000E005C003
:10D29000802FFE0149DD2196011DCD31D10780E0AF
:08D2A0000807B1F7F894FFCF75
:10D2A8000000F0410AD7C3BF9A99F93F0000204116
:10D2B800756E646566696E65640000000000005460
:10D2C800656D702B48756D00000000000000495224
:10D2D80020466C616D650000000000000047617326
:10D2E8000000000000000000000000005475726299
:10D2F800696469747900000000000070480000004B
:10D3080000000000000000000000434F3200000051
:10D318000000000000000000004F32000000000084
:10D32800000000000000000049522054656D7000A4
:10D338000000000000000049522054656D70000094
:10D34800000000000000504D000000000000000038
:10D358000000000000434834000000000000000006
:10D3680000000000416C636F686F6C0000000000F3
:10D37800000000434F000000000000000000000013
:10D38800000048320000000000000000000000001B
:10D39800004F7A6F6E65000000000000000000007A
:10D3A8004832530000000000000000000000004E5A
:10D3B80048330000000000000000000000000139B0
:10D3C800003D003F0008003E000800010002000385
:10D3D80000050004000600080009000000A84166D6
:10D3E80066A63FA167333D7C8C010062BE3C399341
:10D3F800522A409352AA4017D900418C968141B7CE
:10D408003AC9418B899D3E0000A04100002042009E
:10D41800007042133BF142ECC43A430000804027BD
:10D42800882640643B5F3E21B0B23E3D002E30323C
:10D43800342F313335313233413435364237383988
:10D44800432A3023440100803B450000803F0AD72F
:10D458008B40CDCC2C4000006915800008003700B7
:10D46800380039003F003E003D0011001000000068
:10D478000000BF3A023A463A053B773A553A693ACC
:10D4880000000000C72B972B942B12418B2B772B76
:10D498001341000000002241D03F9F3F00000000E0
:10D4A800FB40023A942B932B3D42E740964177414B
:10D4B80007002D37002D34002D35002D33002D3277
:10D4C800002D310073657269616C3A200042543A4C
:10D4D8002000530041004200736574005345540016
:10D4E80023506172616D65746572730023536561C1
:10D4F8002D6C6576656C2050726573737572653D29
:10D5080000234D61676E65746963206465636C69A7
:10D518006E6174696F6E20416E676C653D002343D0
:10D528006F6D70617373205363616C653D002354A4
:10D53800757262696469747920766F6C7461676565
:10D54800733A005640004E54552C20004E54552036
:10D558000023426C7565746F6F7468204E616D6549
:10D568003D0023434F32207A65726F20766F6C74CA
:10D57800616765280070706D293D005620002343BF
:10D588004F32206D617820766F6C74616765202852
:10D59800002343616C69627261746564204F3220B4
:10D5A800636F6E63203D0020766F6C252000237327
:10D5B8006C6F742023002920697320002354696D3F
:10D5C8006520696E74657276616C3D002354696DDF
:10D5D80065206475726174696F6E3D004769766590
:10D5E8006E20736561206C6576656C20503D005037
:10D5F8006120697320756E6C696B656C79210053C5
:10D608006561206C6576656C20503D00206850612E
:10D6180000736C6F743D00534C4F543D0042543DB1
:10D628000062743D0041542B4E414D450043533D2B
:10D638000063733D00234572726F7220746F20730C
:10D648006574206E657720636F6D706173732073E6
:10D6580063616C653D00456E746572656420736333
:10D66800616C6520776173206E6F742076616C69D8
:10D67800642C2076616C6964206761757373207609
:10D68800616C756573206172653A20302E38382CCC
:10D6980020312E332C20312E392C20322E352C20BF
:10D6A800342E302C20342E372C20352E362C203892
:10D6B8002E310023436F6E74696E756F7573204D3C
:10D6C8006F6465204572726F7220746F2073657481
:10D6D800206E657720636F6D70617373207363616B
:10D6E8006C653D00234E657720636F6D70617373C1
:10D6F800207363616C653D0050494E3D0070696E52
:10D708003D0041542B50494E00706800704800504D
:10D7180048007068340070483400566F6C74616754
:10D72800652870483D34293A0070683130007048E7
:10D73800313000566F6C746167652870483D313030
:10D74800293A0074696D65693D0074696D65643DC9
:10D758000054423100746231005475726269646920
:10D768007479204C6F776572204C696D6974205606
:10D77800313A2000235442285631293D004F324384
:10D78800414C006F3263616C004F322063616C69F9
:10D7980062726174696F6E3A2000234F3220766F8F
:10D7A8006C253D00434F325A00636F327A00434F75
:10D7B80032207A65726F20766F6C74202800707042
:10D7C8006D293A200023434F3220566F3D00560002
:10D7D800434F324D00636F326D00434F32204D414D
:10D7E8005820766F6C7420280023434F3220566DE2
:10D7F8003D0054424900746269005475726269645C
:10D80800697479204C6F776572204C696D69742052
:10D8180056696E663A20002354422856696E662976
:10D828003D0054424C0074626C0054757262696425
:10D83800697479204C6F776572204C696D69743A08
:10D84800200020766F6C746167653D002354422880
:10D8580056293D0054425500746275005475726231
:10D868006964697479205570706572204C696D69B6
:10D87800743A20006B65793D00616E6F746865725B
:10D8880020495220696E7075743D007265706C692C
:10D8980065733D0073204F3220436F6E6300566FEF
:10D8A8006C25007320434F3220436F6E6300434F53
:10D8B800323D0070706D004D6561737572696E67F9
:10D8C80020504D322E350020504D313A322E353A07
:10D8D800313000504D28312E302C322E352C31303D
:10D8E800293D00206E672F4C0042543A00313A54CB
:10D8F800656D702048756D696469747900323A54B1
:10D90800656D7020507265737375726500323A6187
:10D918006E642048656967687400333A4C696768C3
:10D928007420496E742E00343A495220466C616D59
:10D938006500353A476173204C6576656C00363A68
:10D948004D61676E65746963206669656C6400374C
:10D958003A49522054656D7000383A704820766113
:10D968006C756500393A496E636C2E20616E672EBE
:10D9780000393A6F7220334420616363656C2E006E
:10D9880044313A5475726269646974790044323A70
:10D99800504D28313A322E353A3130290044333A45
:10D9A800434F3220636F6E632E0044343A4F322067
:10D9B800636F6E632E002A3A546869732048656C59
:10D9C8007000233A53686F77204C4344006F43201C
:10D9D800413D006F432020004C6967687420496E00
:10D9E80074656E73697479007320202000206C7848
:10D9F800004C3D00206C7820004C6576656C3D003D
:10DA0800495220466C616D652000476173206C6542
:10DA180076656C3D00536561726368204469726580
:10DA28006374696F6E00482D6669656C64007320C5
:10DA380020004952204661696C65640049522054AF
:10DA4800656D703D006F430070483D004E6F20705B
:10DA5800482073656E736F72210057656C636F6D34
:10DA68006520746F20456455484B00456455484B04
:10DA7800205345534C6F6767657200206D6F62696C
:10DA88006C65206C6F67676572207374617274656A
:10DA98006420616E642072656164792100493243B3
:10DAA80020696E746572666163652E006E65772005
:10DAB800484D43353838334C007363616C65203DFD
:10DAC8002000204761006D6F646520746F20636FCC
:10DAD8006E74696E6F75730023536561206C65768B
:10DAE800656C20502863616C63293D002343616C99
:10DAF8006962726174696F6E2050726573737572B2
:10DB0800653D006761696E735F6F7269675B5D3A57
:10DB180000736574206761696E735B5D3A005859DC
:10DB28005A20434F554E54533A200058595A2047CB
:10DB3800733A20006765745461705468726573683D
:10DB48006F6C6428293A2000676574417869734FBF
:10DB580066667365742826782C2026792C20267A08
:10DB6800293A20006765745461704475726174695C
:10DB78006F6E28293A2000676574446F75626C657A
:10DB88005461704C6174656E637928293A20006786
:10DB98006574446F75626C6554617057696E646F23
:10DBA80077282920006765744163746976697479F8
:10DBB8005468726573686F6C6428292000676574FF
:10DBC800496E6163746976697479546872657368BB
:10DBD8006F6C642829200067657454696D65496E07
:10DBE800616374697669747928293A2000676574D5
:10DBF8004672656546616C6C5468726573686F6CD3
:10DC08006428293A20006765744672656546616C28
:10DC18006C4475726174696F6E28293A20006973C3
:10DC2800416374697669747958456E61626C65649C
:10DC380028293A20006973416374697669747959AF
:10DC4800456E61626C656428293A200069734163F6
:10DC58007469766974795A456E61626C65642829BD
:10DC68003A20006973496E616374697669747958FA
:10DC7800456E61626C656428293A20006973496EB3
:10DC8800616374697669747959456E61626C65641B
:10DC980028293A20006973496E616374697669744A
:10DCA800795A456E61626C656428293A2000697367
:10DCB8004163746976697479416328293A20006759
:10DCC8006574537570707265737342697428293B63
:10DCD80020747275653F20006765745375707072A3
:10DCE80065737342697428293B2066616C73653FCC
:10DCF80020006973546170446574656374696F6E5C
:10DD08004F6E5828293B20747275653F200069734F
:10DD1800546170446574656374696F6E4F6E5828FA
:10DD2800293B2066616C73653F20006973546170FC
:10DD3800446574656374696F6E4F6E5928293B207A
:10DD4800747275653F200069735461704465746529
:10DD58006374696F6E4F6E5928293B2066616C7336
:10DD6800653F200069735461704465746563746924
:10DD78006F6E4F6E5A28293B20747275653F2000DC
:10DD88006973546170446574656374696F6E4F6E2E
:10DD98005A28293B2066616C73653F2000697341EE
:10DDA80063746976697479536F757263654F6E58D9
:10DDB80028293A2000616363656C2E697341637496
:10DDC8006976697479536F757263654F6E5928293E
:10DDD8003A2000616363656C2E69734163746976E8
:10DDE800697479536F757263654F6E5A28293A20A2
:10DDF80000616363656C2E6973546170536F75724B
:10DE080063654F6E5828293A2000616363656C2E5C
:10DE18006973546170536F757263654F6E59282921
:10DE28003A2000616363656C2E6973546170536FA7
:10DE3800757263654F6E5A28293A200061636365DD
:10DE48006C2E697341736C65657028293A200061EE
:10DE58006363656C2E69734C6F77506F77657228B2
:10DE6800293A20006765745261746528293A20337D
:10DE78002E31343135393F00676574496E746572E7
:10DE880072757074536F7572636528293A2000673C
:10DE98006574496E74657272757074536F757263C8
:10DEA800652831293A2000676574496E7465727275
:10DEB8007570744D617070696E672831293A200059
:10DEC8006973496E74657272757074456E61626CBF
:10DED80065642831293A200067657453656C665477
:10DEE80065737442697428293A2000307830303AD2
:10DEF8002000307800234572726F723A7072657331
:10DF08007375726520424D503038352C2063686532
:10DF1800636B20776972696E67210054656D7020A4
:10DF280048756D6964697479202020007320202069
:10DF380020006F4320483D00432000252020004951
:10DF4800742773207665727920686F7421200049E0
:10DF580074277320717569746520686F742100498E
:10DF680073206169722D636F6E64206F6E3F005479
:10DF7800656D702069732066696E652120200049EF
:10DF880074277320746F6F20636F6F6C2120004FAC
:10DF98006666206169722D636F6E642120200061BE
:10DFA80028782C792C7A292F673A20007320613D34
:10DFB80000206700496E636C2E20616E672E2878FA
:10DFC8002079207A292F6465673A20007320496EEA
:10DFD800636C2E20416E672E007320617A3D0067C6
:10DFE80020006B6579323D005343493531006E613D
:10DFF8006E00696E66006F7666000D0A0073205425
:10E0080075726269646974790054423D004E5455D2
:10E018000020202020202020202020202020202018
:10E028002000436F6D706173733A20002864656740
:10E038002920004E2000204500532000205700488A
:10E048002D6669656C643A202800296D4700203DDB
:0CE058003E00482D6669656C643D0000C8
:020000023000CC
:10E000000D9489F10D94B2F10D94B2F10D94B2F129
:10E010000D94B2F10D94B2F10D94B2F10D94B2F1F0
:10E020000D94B2F10D94B2F10D94B2F10D94B2F1E0
:10E030000D94B2F10D94B2F10D94B2F10D94B2F1D0
:10E040000D94B2F10D94B2F10D94B2F10D94B2F1C0
:10E050000D94B2F10D94B2F10D94B2F10D94B2F1B0
:10E060000D94B2F10D94B2F10D94B2F10D94B2F1A0
:10E070000D94B2F10D94B2F10D94B2F10D94B2F190
:10E080000D94B2F10D94B2F10D94B2F10D94B2F180
:10E090000D94B2F10D94B2F10D94B2F10D94B2F170
:10E0A0000D94B2F10D94B2F10D94B2F10D94B2F160
:10E0B0000D94B2F10D94B2F10D94B2F10D94B2F150
:10E0C0000D94B2F10D94B2F10D94B2F10D94B2F140
:10E0D0000D94B2F10D94B2F10D94B2F10D94B2F130
:10E0E0000D94B2F141546D656761323536300041AF
:10E0F000726475696E6F206578706C6F72657220DE
:10E1000073746B3530305632206279204D4C530099
:10E11000426F6F746C6F616465723E004875683F52
:10E1200000436F6D70696C6564206F6E203D200048
:10E130004350552054797065202020203D20005FF9
:10E140005F4156525F415243485F5F3D2000415658
:10E1500052204C696243205665723D20004743437C
:10E160002056657273696F6E203D20004350552024
:10E1700049442020202020203D20004C6F7720663D
:10E18000757365202020203D20004869676820665F
:10E190007573652020203D200045787420667573D6
:10E1A00065202020203D20004C6F636B2066757336
:10E1B000652020203D20004D617220203720323024
:10E1C000313300312E362E3800342E332E350056A2
:10E1D00023202020414444522020206F7020636F70
:10E1E00064652020202020696E73747275637469E1
:10E1F0006F6E2061646472202020496E74657272B3
:10E20000757074006E6F20766563746F7200726A49
:10E210006D702020006A6D70200057686174207056
:10E220006F72743A00506F7274206E6F7420737541
:10E2300070706F72746564004D7573742062652030
:10E2400061206C6574746572002000577269747483
:10E25000696E672045450052656164696E672045B7
:10E26000450045452065727220636E743D00504F35
:10E27000525400303D5A65726F2061646472003FF1
:10E280003D43505520737461747300403D454550C3
:10E29000524F4D207465737400423D426C696E6B41
:10E2A000204C454400453D44756D70204545505215
:10E2B0004F4D00463D44756D7020464C415348001B
:10E2C000483D48656C70004C3D4C69737420492F83
:10E2D0004F20506F72747300513D51756974005234
:10E2E0003D44756D702052414D00563D73686F7707
:10E2F00020696E7465727275707420566563746FF0
:10E30000727300593D506F727420626C696E6B00BD
:10E310002A0011241FBECFEFD1E2DEBFCDBF01E046
:10E320000CBF12E0A0E0B2E0EEE1FDEF03E00BBFB6
:10E3300002C007900D92A030B107D9F712E0A0E01B
:10E34000B2E001C01D92AE30B107E1F70F9460F367
:10E350000D948DFE01E20EBF0FEF0DBF11241FBE05
:10E360000D9460F30D9400F020E030E040ED57E0B4
:10E3700005C0FA013197F1F72F5F3F4F2817390792
:10E38000C0F308959C01260F311DC901A0E0B0E043
:10E390002F5F3F4FABBFFC018791882361F08093D3
:10E3A000C6008091C00086FFFCCF8091C0008064D1
:10E3B0008093C000EACF08958DE08093C6008091DD
:10E3C000C00086FFFCCF8091C00080648093C000B5
:10E3D0008AE08093C6008091C00086FFFCCF8091C8
:10E3E000C00080648093C00008950F94C2F10F9420
:10E3F000DCF10895FC019081992359F09093C600B7
:10E400008091C00086FFFCCF8091C0008064809323
:10E41000C0003196992379F70895282F982F929567
:10E420009F70892F805D8A3308F0895F8093C600D2
:10E430008091C00086FFFCCF8091C00080648093F3
:10E44000C000822F8F70982F905D9A3308F0995FEB
:10E450009093C6008091C00086FFFCCF8091C000E1
:10E4600080648093C00008959C01FB01853691056E
:10E470001CF46330710594F0C90164E670E00F94F8
:10E480002EFE605D7F4F6093C6008091C00086FFC6
:10E49000FCCF8091C00080648093C0002B30310598
:10E4A00014F43297B4F0C90164E670E00F942EFEC4
:10E4B0006AE070E00F942EFE605D7F4F6093C600AF
:10E4C0008091C00086FFFCCF8091C0008064809363
:10E4D000C000C9016AE070E00F942EFEC0968093E0
:10E4E000C6008091C00086FFFCCF8091C000806490
:10E4F0008093C00008951F93182F8EE692EE60E07F
:10E500000F94C2F11093C6008091C00086FFFCCF2B
:10E510008091C00080648093C0000F94DCF11F9153
:10E5200008952F923F924F925F926F927F928F92B7
:10E530009F92AF92BF92CF92DF92EF92FF920F9392
:10E540001F93DF93CF93CDB7DEB762970FB6F894E2
:10E55000DEBF0FBECDBF382E622ECA01DB015C01CB
:10E560006D01772420E2222E2E010894411C511CBB
:10E570008BC081E0A81680E0B80681E0C80680E084
:10E58000D80628F0C601AA27BB270F940DF2BB2797
:10E59000AD2D9C2D8B2D0F940DF28A2D0F940DF225
:10E5A0002092C6008091C00086FFFCCF8091C00001
:10E5B00080648093C0009DE29093C6008091C0006B
:10E5C00086FFFCCF8091C00080648093C0002092C1
:10E5D000C6008091C00086FFFCCF8091C00080649F
:10E5E0008093C00019828601750188249924A1E0D6
:10E5F0003A1651F03A1620F0B2E03B1661F409C029
:10E600000BBFF701779007C0C7010F9477FE782EF4
:10E6100002C0F7017080872D0F940DF22092C60082
:10E620008091C00086FFFCCF8091C0008064809301
:10E63000C000872D8052F401EF70F0708F3520F408
:10E64000E40DF51D708204C0E40DF51D8EE280839B
:10E650000894E11CF11C011D111D0894811C911CE2
:10E6600090E18916910409F0C2CF80E190E0A0E02A
:10E67000B0E0A80EB91ECA1EDB1E198AC2010F9493
:10E68000FAF10F94DCF16A94662009F072CF629679
:10E690000FB6F894DEBF0FBECDBFCF91DF911F91B3
:10E6A0000F91FF90EF90DF90CF90BF90AF909F9031
:10E6B0008F907F906F905F904F903F902F90089534
:10E6C0002F923F924F925F926F927F928F929F9282
:10E6D000AF92BF92CF92DF92EF92FF920F931F9370
:10E6E000DF93CF93CDB7DEB7CD53D1400FB6F894BB
:10E6F000DEBF0FBECDBF01E20EBF0FEF0DBF94B75F
:10E70000F894A89514BE80916000886180936000A1
:10E7100010926000789493FF05C0E0910002F091A0
:10E7200001021995279A2F9A8091C00082608093E8
:10E73000C00080E18093C40088E18093C1000000A4
:10E74000EE24FF24870144E0A42EB12CCC24DD2448
:10E7500024C0C5010197F1F70894E11CF11C011DCB
:10E76000111D21E2E2162EE4F20620E0020720E06D
:10E77000120718F031E0C32ED12CC801B70127ECE5
:10E780003BE140E050E00F9441FE611571058105C9
:10E79000910519F485B1805885B98091C00087FD35
:10E7A00003C0C114D104A9F2A6014F5F5F4FC25E3E
:10E7B000DE4F59834883CE51D140C25EDE4F8881FF
:10E7C0009981CE51D140019711F00D9410FEC05D9A
:10E7D000DE4F19821882C053D14060E0C15DDE4F28
:10E7E0001882CF52D14088249924C35DDE4F19820C
:10E7F0001882CD52D140C05EDE4F188219821A8233
:10E800001B82C052D140CE5CDE4F188219821A8220
:10E810001B82C253D140EE24FF2487010BBFF701B6
:10E8200007911691C45CDE4F19830883CC53D14005
:10E830000D940BFEC25EDE4F28813981CE51D1404E
:10E840002130310509F52091C600C25EDE4F1982E4
:10E850001882CE51D14022C02F5F3F4F4F4F5F4FA4
:10E86000213082E138078AE7480780E0580780F0C6
:10E87000C45CDE4FE881F981CC53D140EF5FFF4F9C
:10E8800019F0EE27FF27099420E030E040E050E047
:10E890008091C00087FFE0CF2091C600C35DDE4FAE
:10E8A00048815981CD52D1404F5F5F4FC35DDE4FEC
:10E8B00059834883CD52D140213209F063C64A3092
:10E8C000510508F05FC60894811C911C53E0851621
:10E8D000910409F059C600E010E018C081E280936D
:10E8E000C6008091C00086FFFCCF8091C00080648C
:10E8F0008093C0002F5F3F4F2931310579F70F9486
:10E90000DCF10F5F1F4F0530110519F020E030E0FA
:10E91000E5CF10920A0210920B0210920C02109294
:10E920000D02109206021092070210920802109235
:10E930000902109202021092030210920402109235
:10E9400005028FEE90EE60E00F94F5F180E191EE1C
:10E9500060E00F94C2F18091C00087FFFCCF9091DE
:10E96000C600903608F09F759032B8F09093C600BC
:10E970008091C00086FFFCCF8091C00080648093AE
:10E98000C000A0E2A093C6008091C00086FFFCCF2B
:10E990008091C00080648093C000983409F4D7C18E
:10E9A0009934B8F4923409F459C1933458F490333B
:10E9B00019F1903308F4E3C59F33A1F1903409F0C5
:10E9C000DEC5BDC0953409F470C1963409F0D7C5D1
:10E9D00098C1923509F42BC2933538F49C3409F46C
:10E9E000F5C1913509F0CBC518C2963509F445C279
:10E9F000993509F0C4C567C483E792EE62E00F94CD
:10EA0000F5F110920602109207021092080210927D
:10EA1000090210920A0210920B0210920C0210923C
:10EA20000D0213C18FE792EE62E00F94F5F18FEEC5
:10EA300090EE60E00F94F5F181E291EE60E00F94CA
:10EA4000C2F187EB91EE60E00F94F5F180E391EE77
:10EA500060E00F94C2F184EE90EE60E00F94F5F167
:10EA60008FE391EE60E00F94C2F186E090E061E008
:10EA700070E00F9434F20F94DCF18DE591EE60E0DC
:10EA80000F94C2F189EC91EE60E00F94F5F18EE401
:10EA900091EE60E00F94C2F183EC91EE60E00F9490
:10EAA000F5F18CE691EE60E00F94C2F18EE10F94E7
:10EAB0000DF288E90F940DF281E00F940DF20F949E
:10EAC000DCF18BE791EE60E00F94C2F119E0E0E039
:10EAD000F0E010935700E4918E2F0F940DF20F94F5
:10EAE000DCF18AE891EE60E00F94C2F1E3E0F0E03F
:10EAF00010935700E4918E2F0F940DF20F94DCF1D8
:10EB000089E991EE60E00F94C2F1E2E0F0E0109349
:10EB10005700E4918E2F0F940DF20F94DCF188EAE8
:10EB200091EE60E00F94C2F1E1E0F0E01093570045
:10EB30001491812F0F940DF20F94DCF107CF8BE825
:10EB400092EE62E00F94F5F18BE492EE60E00F94A8
:10EB5000F5F10F94DCF100E010E019C0C8016F2D51
:10EB60000F947FFEFF2031F489E492EE60E00F9471
:10EB7000C2F10BC0F092C6008091C00086FFFCCFAE
:10EB80008091C00080648093C0000F5F1F4FC80158
:10EB900081519F41A0E0B0E0ABBFFC01F790BAE229
:10EBA000FB1621F0E2E000301E07C1F60F94DCF105
:10EBB0000F94DCF187E592EE60E00F94F5F10F948D
:10EBC000DCF1CC24DD2400E010E01EC0C8010F946D
:10EBD00077FEF82E882331F489E492EE60E00F94FA
:10EBE000C2F10BC08093C6008091C00086FFFCCFAD
:10EBF0008091C00080648093C000FE1419F00894D6
:10EC0000C11CD11C0F5F1F4FC80181519F41A0E063
:10EC1000B0E0ABBFFC01E790FAE2EF1621F022E092
:10EC20000030120799F60F94DCF10F94DCF182E6C4
:10EC300092EE60E00F94C2F1C60161E070E00F94C3
:10EC400034F20F94DCF10F94DCF110920202109276
:10EC50000302109204021092050278CE89E992EE26
:10EC600062E00F94F5F1279A2F9A16C02F9880E052
:10EC700090E0E0EDF7E03197F1F7019684369105E9
:10EC8000C1F72F9A80E090E0E0EDF7E03197F1F7DF
:10EC9000019684369105C1F78091C00087FFE6CFC9
:10ECA0008091C00087FFFCCF64C485EA92EE62E0E9
:10ECB0000F94F5F140910202509103026091040219
:10ECC0007091050281E020E10F9491F2809102029F
:10ECD00090910302A0910402B091050280509F4FD1
:10ECE000AF4FBF4F8093020290930302A0930402A0
:10ECF000B093050280509041A040B04008F426CE69
:10ED0000A4CF83EB92EE62E00F94F5F140910602FE
:10ED100050910702609108027091090280E020E1A1
:10ED20000F9491F28091060290910702A09108023F
:10ED3000B091090280509F4FAF4FBF4F80930602A2
:10ED400090930702A0930802B0930902FFCD80ECD4
:10ED500092EE62E00F94F5F183E792EE60E00F949B
:10ED6000F5F18FE792EE60E00F94F5F18BE892EE0B
:10ED700060E00F94F5F189E992EE60E00F94F5F10F
:10ED800085EA92EE60E00F94F5F183EB92EE60E09D
:10ED90000F94F5F180EC92EE60E00F94F5F187ECC2
:10EDA00092EE60E00F94F5F188ED92EE60E00F9442
:10EDB000F5F18FED92EE60E00F94F5F18AEE92EEB0
:10EDC00060E00F94F5F183E093EEBDCD87EC92EE19
:10EDD00062E00F94F5F181E40F947BF282E40F94EA
:10EDE0007BF283E40F947BF284E40F947BF285E45E
:10EDF0000F947BF286E40F947BF287E40F947BF20E
:10EE000088E40F947BF28AE40F947BF28BE40F94F6
:10EE10007BF28CE40F947BF299CD88ED92EE62E068
:10EE20000F94F5F1772473948824992409C48FED05
:10EE300092EE62E00F94F5F140910A0250910B02BC
:10EE400060910C0270910D0282E020E10F9491F22A
:10EE500080910A0290910B02A0910C02B0910D02D8
:10EE600080509F4FAF4FBF4F80930A0290930B0289
:10EE7000A0930C02B0930D0269CD8AEE92EE62E08F
:10EE80000F94F5F184EE90EE60E00F94F5F18FECC5
:10EE900091EE60E00F94F5F1662477244301CC5D98
:10EEA000DE4F19821882C452D140D401C301B695F5
:10EEB000A79597958795CA5DDE4F88839983AA8326
:10EEC000BB83C652D140CC5DDE4FA881B981C4520C
:10EED000D1401196CC5DDE4FB983A883C452D14096
:10EEE000CD0162E070E00F9434F2B0E2B093C6005E
:10EEF0008091C00086FFFCCF8091C0008064809329
:10EF0000C000EDE2E093C6008091C00086FFFCCF18
:10EF10008091C00080648093C000F0E2F093C6004E
:10EF20008091C00086FFFCCF8091C00080648093F8
:10EF3000C000CA5DDE4FE880F9800A811B81C6529D
:10EF4000D140BB27A12F902F8F2D0F940DF2CA5DBA
:10EF5000DE4F8881C652D1400F940DF2B0E2FB2EF5
:10EF6000F092C6008091C00086FFFCCF8091C00067
:10EF700080648093C0000DE30093C6008091C000C0
:10EF800086FFFCCF8091C00080648093C00010E2B7
:10EF90001093C6008091C00086FFFCCF8091C00016
:10EFA00080648093C0008BBEF3012791C65DDE4F65
:10EFB0002883CA52D140A22EBB24CC24DD2408943D
:10EFC000611C711C811C911C8BBEF3018791282E42
:10EFD0003324442455240894611C711C811C911C09
:10EFE0008BBEF3013791C55DDE4F3883CB52D140E4
:10EFF0000894611C711C811C911C8BBEF30147910C
:10F00000C45DDE4F4883CC52D140ADEFEA2EAFEF66
:10F01000FA2EAFEF0A2FAFEF1A2F6E0C7F1C801E57
:10F02000911E142D032DF22CEE24EA0CFB1C0C1D5A
:10F030001D1D0F940DF220E22093C6008091C000A8
:10F0400086FFFCCF8091C00080648093C000C65DC5
:10F05000DE4F8881CA52D1400F940DF230E23093D6
:10F06000C6008091C00086FFFCCF8091C000806404
:10F070008093C000C45DDE4F8881CC52D1400F9494
:10F080000DF240E24093C6008091C00086FFFCCFA5
:10F090008091C00080648093C000C55DDE4F888190
:10F0A000CB52D1400F940DF250E25093C6008091A4
:10F0B000C00086FFFCCF8091C00080648093C000B8
:10F0C0008FEFE8168FEFF80680E0080780E018075A
:10F0D00031F484E092EE60E00F94C2F1DFC0D80119
:10F0E000C7018070907CA070B0708050904CA040A0
:10F0F000B040D1F52FEF3FE340E050E0E222F322B1
:10F1000004231523CA5DDE4FA880B980CA80DB8046
:10F11000C652D140AE0CBF1CC01ED11EAA0CBB1CD7
:10F12000CC1CDD1C8EE092EE60E00F94C2F1BB2798
:10F13000A12F902F8F2D0F940DF28E2D0F940DF285
:10F1400030E23093C6008091C00086FFFCCF8091F2
:10F15000C00080648093C0004EE34093C60080915D
:10F16000C00086FFFCCF87C08EE09EEFA0E0B0E03D
:10F17000E822F9220A231B239CE0E91694E9F90608
:10F1800090E0090790E0190709F088C0C45DDE4FE0
:10F19000A881CC52D140EA2EFF2400E010E0102FCD
:10F1A0000F2DFE2CEE24C55DDE4FB881CB52D14031
:10F1B000EB0EF11C011D111DD601C501817090706F
:10F1C000A070B070DC0199278827E80EF91E0A1F8D
:10F1D0001B1F20EF30E040E050E0A222B322C42207
:10F1E000D52241E1AA0CBB1CCC1CDD1C4A95D1F7F1
:10F1F000EA0CFB1C0C1D1D1D81E090E0A0E0B0E0BE
:10F20000282239224A225B2235E1220C331C441C7D
:10F21000551C3A95D1F7E20CF31C041D151D57013E
:10F220006801AA0CBB1CCC1CDD1C85E192EE60E0E1
:10F230000F94C2F1C801AA27BB270F940DF2BB2778
:10F24000A12F902F8F2D0F940DF28E2D0F940DF274
:10F2500090E29093C6008091C00086FFFCCF809121
:10F26000C00080648093C000AEE3A093C60080918C
:10F27000C00086FFFCCF8091C00080648093C000F6
:10F28000C601AA27BB270F940DF2BB27AD2D9C2DDD
:10F290008B2D0F940DF28A2D0F940DF20F94DCF14B
:10F2A000CC5DDE4FE881F981C452D140F99709F471
:10F2B0004DCBF4E0EF2EF12C012D112D6E0C7F1CA7
:10F2C000801E911EF2CD83E093EE62E00F94F5F183
:10F2D0008AE192EE60E00F94C2F18091C00087FF56
:10F2E000FCCF1091C6001F751093C6008091C0001E
:10F2F00086FFFCCF8091C00080648093C0000F9493
:10F30000DCF1812F81548A3108F036C1163409F4BA
:10F3100095C0173490F4133409F44EC0143430F40B
:10F320001134F1F0123409F01DC130C0143409F465
:10F3300059C0153409F016C16BC01A3409F4C4C0A1
:10F340001B3438F4173409F48FC0183409F00AC19B
:10F35000A1C01B3409F4D2C01C3409F003C1E8C0B9
:10F360008FEF81B90DC082B1809582B980E090E0C5
:10F37000E0EDF7E03197F1F70196883C9105C1F790
:10F380008091C00087FFEFCF12B8EFC08FEF84B934
:10F390000DC085B1809585B980E090E0E0EDF7E0A3
:10F3A0003197F1F70196883C9105C1F78091C00033
:10F3B00087FFEFCF15B8D9C08FEF87B90DC088B1DF
:10F3C000809588B980E090E0E0EDF7E03197F1F7C3
:10F3D0000196883C9105C1F78091C00087FFEFCF6F
:10F3E00018B8C3C08FEF8AB90DC08BB180958BB9A7
:10F3F00080E090E0E0EDF7E03197F1F70196883C8E
:10F400009105C1F78091C00087FFEFCF1BB8ADC059
:10F410008FEF8DB90DC08EB180958EB980E090E0F0
:10F42000E0EDF7E03197F1F70196883C9105C1F7DF
:10F430008091C00087FFEFCF1EB897C08FEF80BBD1
:10F440000DC081B3809581BB80E090E0E0EDF7E0F6
:10F450003197F1F70196883C9105C1F78091C00082
:10F4600087FFEFCF11BA81C08FEF83BB0DC084B38C
:10F47000809584BB80E090E0E0EDF7E03197F1F714
:10F480000196883C9105C1F78091C00087FFEFCFBE
:10F4900014BA6BC08FEF809301010FC080910201FD
:10F4A00080958093020180E090E0E0EDF7E03197F5
:10F4B000F1F70196883C9105C1F78091C00087FF64
:10F4C000EDCF1092020151C08FEF809304010FC065
:10F4D0008091050180958093050180E090E0E0ED4A
:10F4E000F7E03197F1F70196883C9105C1F78091DB
:10F4F000C00087FFEDCF1092050137C08FEF8093DA
:10F5000007010FC08091080180958093080180E079
:10F5100090E0E0EDF7E03197F1F70196883C910536
:10F52000C1F78091C00087FFEDCF109208011DC088
:10F530008FEF80930A010FC080910B01809580931B
:10F540000B0180E090E0E0EDF7E03197F1F70196F4
:10F55000883C9105C1F78091C00087FFEDCF1092E4
:10F560000B0103C085E292EEEEC98091C00087FFD7
:10F57000FCCF8091C600EAC988E392EEE4C98CE131
:10F5800091EEE1C988249924933011F1943028F444
:10F59000913089F09230B8F408C0953061F195301F
:10F5A000F0F0963009F048C043C02B3109F042C951
:10F5B00091E06BE13FC96227C15DDE4F2883CF52E6
:10F5C000D14092E037C9B22FA0E0622793E032C960
:10F5D000822F90E0A82BB92B622794E02BC92E3004
:10F5E00009F039C3622795E0C05DDE4F19821882A9
:10F5F000C053D1401FC9E1E0F0E0EC0FFD1FC05D3A
:10F60000DE4F08811981C053D140E00FF11F2083E4
:10F610000F5F1F4FC05DDE4F19830883C053D14079
:10F6200062270A171B0709F005C9D80196E002C92D
:10F63000261709F010C303C0973009F0FBC87724E0
:10F640009981933109F412C19431C8F4963009F4C8
:10F65000D8C0973050F4923009F406C1933009F4C1
:10F660006DC0913009F059C253C0913109F477C08F
:10F67000923108F0BBC0903109F04FC2F5C098310B
:10F6800009F487C0993150F4953109F4EFC09531F0
:10F6900008F4C6C1963109F040C2C2C19A3109F4DA
:10F6A0006CC09A3108F491C09B3109F45BC09D3164
:10F6B00009F033C29D81903359F48F81882311F46E
:10F6C0009EE11CC0813011F091E018C098E916C08D
:10F6D000892F807591F0903539F4E0E0F0E089E011
:10F6E0008093570094910AC0983539F4E3E0F0E034
:10F6F00089E080935700949101C090E01A821B82A8
:10F700008D818C831D829E831F8227E030E009C299
:10F710001A8288E08B8381E48C8386E58D8382E581
:10F720008E8389E48F8383E5888780E589878FE5E9
:10F730008A8782E38B872BE030E0F3C18A818139AD
:10F7400041F0823941F0803911F48FE005C080E04A
:10F7500003C082E001C08AE01A828B8344C0772410
:10F76000739482C08D81882311F48EE12CC0813086
:10F7700011F081E028C088E926C01A82E1E0F0E0BB
:10F7800089E08093570084918B831C8224E030E0D1
:10F79000C8C18B81803589F48C81883039F4E2E0EE
:10F7A000F0E089E08093570084910DC0E0E0F0E044
:10F7B00089E080935700849106C0E3E0F0E089E09F
:10F7C0008093570084911A82DFCF8D81836C99E0FA
:10F7D000E1E0F0E0082E90935700E89507B600FCB2
:10F7E000FDCF1A821B8223E030E09BC180EC8A832C
:10F7F000CE5CDE4F188219821A821B82C253D1401E
:10F800008EC18A8190E0A0E0B0E0582F44273327D2
:10F8100022278B8190E0A0E0B0E0DC0199278827C7
:10F82000282B392B4A2B5B2B8D8190E0A0E0B0E098
:10F83000282B392B4A2B5B2B8C8190E0A0E0B0E089
:10F84000BA2FA92F982F8827282B392B4A2B5B2BCF
:10F85000220F331F441F551FC05EDE4F288339839C
:10F860004A835B83C052D1401A8259C13A81C95C34
:10F87000DE4F3883C753D140CA5CDE4F1882C6536F
:10F88000D1408B81C82EDD24CA5CDE4F488159816E
:10F89000C653D140C42AD52A933109F082C0CE5C28
:10F8A000DE4F88819981AA81BB81C253D1408050AB
:10F8B000904CA340B04030F583E0CE5CDE4FE88052
:10F8C000F9800A811B81C253D140F70100935B008C
:10F8D00080935700E89507B600FCFDCFCE5CDE4F65
:10F8E000088119812A813B81C253D14000501F4FAA
:10F8F0002F4F3F4FCE5CDE4F088319832A833B8313
:10F90000C253D140C05EDE4F488159816A817B81FC
:10F91000C052D140DE011B9631E08C9111962C91A2
:10F9200011971296C75CDE4F2883C953D140C85C3B
:10F93000DE4F1882C853D14090E0C85CDE4FE881AA
:10F94000F981C853D1408E2B9F2B0C01FA01609393
:10F950005B0030935700E89511244E5F5F4F6F4F67
:10F960007F4F0EEFE02E0FEFF02ECE0CDF1CC114F8
:10F97000D10499F685E0C05EDE4F088119812A81A5
:10F980003B81C052D140F80120935B008093570027
:10F99000E89507B600FCFDCF81E180935700E8951C
:10F9A00035C0C05EDE4F88819981AA81BB81C0527B
:10F9B000D140B695A795979587957C018601ABE0D8
:10F9C000AA2EB12CAC0EBD1E0BC0D5016D915D01F0
:10F9D000C7010F947FFE0894E11CF11C01501040F8
:10F9E0000115110591F7A60160E070E0440F551F65
:10F9F000661F771FC05EDE4FE880F9800A811B8199
:10FA0000C052D1404E0D5F1D601F711F1A82C05E33
:10FA1000DE4F488359836A837B83C052D1407FC0C5
:10FA2000FA80C55CDE4FF882CB53D140C65CDE4F16
:10FA30001882CA53D1408B81C82EDD24C65CDE4FAC
:10FA400008811981CA53D140C02AD12A1A828981DA
:10FA5000BE016D5F7F4F843121F59601C05EDE4FA0
:10FA6000E880F9800A811B81C052D1400BBFF701A9
:10FA700087919691DB018C9311969C936E5F7F4FDB
:10FA8000D801C7010296A11DB11DC05EDE4F88835B
:10FA90009983AA83BB83C052D14022503040F1F6F3
:10FAA00036C0C05EDE4F288139814A815B81C052F9
:10FAB000D1400894C108D108760100E010E0089414
:10FAC000C11CD11C0894E11CF11C011D111DE20E8A
:10FAD000F31E041F151F21BDBB27A52F942F832FB5
:10FAE00082BD2F5F3F4F4F4F5F4FF89A80B5DB01CC
:10FAF0008D93BD012E153F054007510761F7C05E8C
:10FB0000DE4F288339834A835B83C052D1409601FC
:10FB10002D5F3F4FFB01108204C080EC8A8322E0FE
:10FB200030E08BE18093C6008091C00086FFFCCF5F
:10FB30008091C00080648093C000C15DDE4FF88179
:10FB4000CF52D140F093C6008091C00086FFFCCF19
:10FB50008091C00080648093C000432F3093C60022
:10FB60008091C00086FFFCCF8091C00080648093AC
:10FB7000C000922F2093C6008091C00086FFFCCF6A
:10FB80008091C00080648093C0008EE08093C600A6
:10FB90008091C00086FFFCCF8091C000806480937C
:10FBA000C00065E1C15DDE4FE880CF52D1406E25D7
:10FBB00069276427FE01319610C090819093C6009A
:10FBC0008091C00086FFFCCF31968091C000806498
:10FBD0008093C0006927215030402115310569F715
:10FBE0006093C6008091C00086FFFCCF8091C0006A
:10FBF00080648093C00085B1805885B9772081F4F6
:10FC0000C15DDE4F0881CF52D1400F5FC15DDE4F35
:10FC10000883CF52D14090E0A0E0B0E00D941AF4F8
:10FC200027982F9880E090E020ED37E0F901319798
:10FC3000F1F7019684369105C9F700008091C00064
:10FC40008D7F8093C00081E180935700E895EE2777
:10FC5000FF270994FFCF90E00D941AF497FB092E2B
:10FC600007260AD077FD04D02ED006D000201AF443
:10FC7000709561957F4F0895F6F7909581959F4F08
:10FC80000895A1E21A2EAA1BBB1BFD010DC0AA1FDD
:10FC9000BB1FEE1FFF1FA217B307E407F50720F0F5
:10FCA000A21BB30BE40BF50B661F771F881F991F70
:10FCB0001A9469F760957095809590959B01AC01B9
:10FCC000BD01CF010895AA1BBB1B51E107C0AA1FAC
:10FCD000BB1FA617B70710F0A61BB70B881F991FED
:10FCE0005A95A9F780959095BC01CD010895F99991
:10FCF000FECF92BD81BDF89A992780B50895262F31
:10FD0000F999FECF1FBA92BD81BD20BD0FB6F89400
:0EFD1000FA9AF99A0FBE01960895F894FFCF63
:040000033000E000E9
:00000001FF
